:1000000000800020BD010000DD620000A962000048
:10001000A9620000A9620000A9620000A9620000B4
:10002000A9620000A9620000A9620000DD62000070
:10003000DD620000A9620000DD620000996200003C
:10004000DD620000DD620000DD620000DD620000B4
:10005000DD620000DD620000DD620000DD620000A4
:10006000DD620000DD620000DD620000DD62000094
:10007000DD620000DD620000DD620000DD62000084
:10008000DD620000DD620000DD620000DD62000074
:10009000DD620000DD620000DD620000DD62000064
:1000A000DD620000DD620000DD620000DD62000054
:1000B000DD620000DD620000DD620000DD62000044
:1000C000DD620000DD620000DD620000DD62000034
:1000D000DD620000DD620000DD620000DD62000024
:1000E000DD620000DD620000DD620000DD62000014
:1000F000DD620000816F0000DD6200003D750000E0
:10010000DD620000197A0000DD620000DD6200009F
:10011000DD620000DD620000DD620000DD620000E3
:10012000DD620000AD0800004D0C0000DD62000043
:10013000DD620000DD620000DD620000DD620000C3
:10014000DD620000DD620000DD620000DD620000B3
:10015000558900006D890000858900009D89000097
:10016000DD620000217D0000DD620000DD62000034
:10017000DD620000DD620000DD620000DD62000083
:10018000DD620000DD620000DD620000C55B000092
:10019000DD620000DD620000DD620000DD62000063
:1001A000DD620000DD620000DD620000DD62000053
:1001B000DD620000DD620000DD620000564B4CF2A3
:1001C000205210B51A804DF628121A8000BF00BFC9
:1001D00006F088F8514B4FF010621A60504A9A604E
:1001E000504ADA60A3F53043203B1A6812F480725B
:1001F00004D14D490A604FF4A8521A604B4B1A784B
:10020000110703D51A7842F008021A70484B2A22C7
:100210001A700023474A48499818884204D247492F
:10022000595899500433F5E7454A464B9A424FF0E6
:10023000000302D242F8043BF7E74349434A5958C6
:1002400099500433B3F5DE7FF7D1414B802103F899
:10025000011B40498B42F9D13F4B1A603F4B0A22A8
:100260001A70A3F5805324225A70A0221A709A792A
:100270009207FCD59A79D406FCD4394B9A7902F0CE
:100280000C02082AF9D103221A7140225A719A7974
:100290009006FCD5324B9A795106FBD5314A32494A
:1002A00011600221516020221A702D4B9B7903F0BE
:1002B0000C030C2BF9D12D4B2D4A1A602D4B2E4AD5
:1002C0001A6000225A60072243F8042C2B4AC3F814
:1002D0000C2D62B606F0B0FB134B1B68DA0705D590
:1002E000274806F0B9F9274B274A1A60274B1B7895
:1002F0005B0609D5234C244A2368934204D1204845
:1003000006F0AAF90023236009F0C2FC05F0F0FF13
:1003100008F001FCFEE700BF0E20054030800440DD
:10032000823F04000100002B14D0034002D007409C
:1003300000E007406087FF1F7C88FF1F74D100002A
:100340007C88FF1F0092FF1F000000000082FF1F3B
:1003500000E400E05FE400E008ED00E0005006404B
:100360000040064044800440000003010480044033
:10037000C010050014E000E0FF760100000020201E
:1003800000DD68501CE00340A5C3945A00F007400C
:10039000FFFFFFFFFFFFFFFFFFFFFFFFFFFFFFFF6D
:1003A000FFFFFFFFFFFFFFFFFFFFFFFFFFFFFFFF5D
:1003B000FFFFFFFFFFFFFFFFFFFFFFFFFFFFFFFF4D
:1003C000FFFFFFFFFFFFFFFFFFFFFFFFFFFFFFFF3D
:1003D000FFFFFFFFFFFFFFFFFFFFFFFFFFFFFFFF2D
:1003E000FFFFFFFFFFFFFFFFFFFFFFFFFFFFFFFF1D
:1003F000FFFFFFFFFFFFFFFFFFFFFFFFFFFFFFFF0D
:10040000FFFFFFFFFFFFFFFFFFFFFFFFFEFFFFFFFD
:1004100010B5054C237833B9044B13B10448AFF33E
:1004200000800123237010BD7C88FF1F00000000A6
:1004300074D1000008B5064B1BB106480649AFF35E
:1004400000800648036813B1054B03B1984708BD07
:100450000000000074D100008088FF1F7C88FF1F0F
:10046000000000002DE9F34101210D2006F09CF968
:100470006F4B704C704E20221A600C2005F0EAFC85
:10048000082005F011FDC02008F04DFB054602F0E4
:10049000A7FE2846256002F028FEFE2811D14FF461
:1004A0007A6006F0B3FA902008F03DFB63490446F9
:1004B0004FF4E13201F0EAF93460306802F0B4FB45
:1004C000FBE723685E4993F8700006F0D5F82368CF
:1004D000012193F8700006F067F92368C42193F8AE
:1004E000700006F091F94FF4FA7006F08FFA206868
:1004F00002F0CEFD430803F1376303F5D833B3FBB5
:10050000F0F006F0E7FA206802F0D3FD20B123688E
:1005100093F86E0006F08AFB206802F0D4FD4308D1
:1005200003F1376303F5D833B3FBF0F006F0BCFDFD
:10053000206802F0D1FD430803F1B76303F5584387
:10054000B3FBF0F007F08EF8206802F0BCFD054622
:100550005C2008F0E8FA2A463A493B4D074604F089
:1005600047FB20682F6002F093FD8046682008F06A
:10057000DAFA42463549074603F03AFE344B542036
:100580001F6008F0D0FA074600F0A4FD314B324955
:100590001F60384600F02CFF902008F0C4FA27496D
:1005A0004FF4E132074601F071F92068376002F03C
:1005B00093FD0746902008F0B6FA27493A460646CA
:1005C00001F064F9254B1E60254E3368B3F57A6F50
:1005D000FAD32868234B01221A7003689B6A984754
:1005E000286803681B6A984728683768036807F219
:1005F000FA575B6ABFB298473368BB4203D2286898
:1006000003681B6AF7E76022009213462068002106
:1006100002F0F5FC00F008F923681B7C2BB10120E7
:1006200002B0BDE8F04105F0CDB902B0BDE8F081FF
:1006300084F00F40B088FF1F9888FF1FC891FF1FEC
:100640000000A0419091FF1FB888FF1F8091FF1FFD
:10065000AC88FF1FA488FF1FA091FF1FB488FF1F55
:10066000CC89FF1FA088FF1F114B1B6893F88530B2
:10067000EBB1104B1A68002A08DA0F4908780128F4
:100680000DD00120087020200C4907E007D00A494E
:10069000087820B100200870094920200860013244
:1006A0004FF6E8518A42C8BF4FF0FF321A607047D8
:1006B000B088FF1F9C88FF1F6487FF1F84F00F40D6
:1006C00088F00F402DE9F3474E4C4F4D236893F8C7
:1006D0008060002E69D14D4BDFF840A11868DFF82B
:1006E000409102F0A1FA4A4B186802F09DFA494B7A
:1006F000186804F01BF8286803681B6A9847DAF842
:100700000020B9F80030D31A9BB2B3F57A7F46D9EE
:100710002068DFF8108103F083F998F800309842E0
:100720002AD03D4F4BB1206803F065F9206802F0F4
:1007300098FC3E7088F800602DE03A78042A0AD8C8
:100740003322009220680121992202F058FC3B7864
:1007500001333B701FE0052A1DD1286803689B6A9E
:100760009847286803685B6A9847206802F079FC1C
:10077000012388F800300EE0206803F041F938B119
:10078000009620680121FF22334602F038FC02E087
:10079000206802F066FCDAF80030A9F80030206822
:1007A00003F07CF8FFF760FF8EE700F067F823683E
:1007B0001B7C0BB105F078FA00F05AFB2368002689
:1007C00083F8806000F030F823681B7C13B130465A
:1007D00005F0F8F8206802F0FBFF4FF47A6006F0AD
:1007E00015F9286803689B6A9847286803681B6A9C
:1007F0009847286803685B6A9847206802F031FCD4
:1008000062E700BFB088FF1FB888FF1F9888FF1FEE
:10081000B488FF1FAC88FF1FA888FF1FCC89FF1F6B
:10082000A288FF1FA088FF1F08B50F4B0F494FF08C
:1008300000721A604FF080621A600D4B1B68587A84
:100840001A7A51F83010022A4FF001020CBF81F8D9
:10085000802081F80021587E064B187005F0BEFB01
:10086000054B01221A7008BD04E100E0F0CC000045
:10087000B088FF1FBC88FF1FBE88FF1F084B4FF0CA
:1008800000721A604FF080621A60064B1B685A7A39
:10089000054B53F83230012283F80021704700BF26
:1008A00084E100E0B088FF1FF0CC00002DE9F041AA
:1008B000A64C23780F2B00F2BD81DFE813F0200057
:1008C00036004C00620078008E00A400BA00D1000F
:1008D000E8002D0151010F017F01690110009C4DBD
:1008E000287805F0C3FB9B4B1B68B3F878200521E3
:1008F00000EB8200B0FBF1F2A3F87820E8E0944D21
:10090000287805F0B3FB934B1B685A8C452192B2B3
:1009100001FB02004626B0FBF6F292B2587E5A84E2
:10092000287005F05BFB01237AE1894D287805F0FA
:100930009DFB884B1B689A8C452192B201FB0200FB
:100940004626B0FBF6F292B2987E9A84287005F0A3
:1009500045FB022364E17E4D287805F087FB7D4B43
:100960001B68DA8C452192B201FB02004626B0FBDF
:10097000F6F292B2D87EDA84287005F02FFB0323BA
:100980004EE1734D287805F071FB724B1B681A8D90
:10099000452192B201FB02004626B0FBF6F292B26C
:1009A000187F1A85287005F019FB042338E1684D7B
:1009B000287805F05BFB674B1B685A8D452192B286
:1009C00001FB02004626B0FBF6F292B2587F5A8530
:1009D000287005F003FB052322E15D4D287805F022
:1009E00045FB5C4B1B689A8D452192B201FB0200CE
:1009F0004626B0FBF6F292B2987F9A85287005F0F1
:100A0000EDFA06230CE1524D287805F02FFB514BEF
:100A10001B68DA8D452192B201FB02004626B0FB2D
:100A2000F6F292B2D87FDA85287005F0D7FA07235C
:100A3000F6E0474D287805F019FB464B1B681A8EE7
:100A4000452192B201FB02004626B0FBF6F292B2BB
:100A500093F820001A86287005F0C0FA0823DFE01A
:100A60003B4D287805F002FB3A4B1B685A8E452116
:100A700092B201FB02004626B0FBF6F292B293F866
:100A800021005A86287005F0A9FA0923C8E0304DE4
:100A9000287805F0EBFA2F4B1B689A8E452192B20D
:100AA00001FB02004626B0FBF6F292B29A862A4A71
:100AB000117809290AD9002111701A7A012A24D142
:100AC000987A287005F08AFA0C23A9E00131117098
:100AD000187E287005F082FA0023A1E01C4D2878CA
:100AE00005F0C4FA1B4B1B689A89632192B201FB83
:100AF00002006426B0FBF6F292B2597A9A81174A44
:100B000052F83120012182F8801093F86900287092
:100B100005F064FA0A2383E00D4D287805F0A6FA63
:100B20000C4B1B68B3F86C2092B202EBC20210446B
:100B30000A21B0FBF1F292B293F86800A3F86C209E
:100B4000287005F04BFA0B236AE000BFBE88FF1F38
:100B5000BC88FF1FB088FF1FBD88FF1FF0CC0000BE
:100B6000374D287805F082FA364B1B68B3F86A20B7
:100B700092B202EBC20210440A21B0FBF1F292B22F
:100B80001879A3F86A20287005F028FA0E2347E0A8
:100B90002B4D287805F06AFA2A4B1B68DA881D214C
:100BA00092B201FB02001E26B0FBF6F292B2987AD6
:100BB000DA80287005F012FA0D2331E0214B204D28
:100BC0001E68377A012F984615D1287805F04EFA1D
:100BD000D8F80030DA89632192B201FB0200642662
:100BE000B0FBF6F292B2DA815A7A174B53F83230F0
:100BF00083F8007109E0022F05D1287805F036FA54
:100C000080B2F08101E00023F381D8F8003093F83E
:100C1000776046B193F87600287005F0DFF90F236E
:100C20002370BDE8F081187E287005F0D7F9267092
:100C3000BDE8F0810220BDE8F04104F043BB00BFF5
:100C4000BC88FF1FB088FF1FF0CC0000FFF72EBE4E
:100C50002DE9F3477B4E06F09BFA96F800900025AD
:100C600009F001092F46784C802300220093206868
:100C70001346012102F0C3F9337813F0010FA046A7
:100C800023D104F005FEB7F5966F0FD175B9206832
:100C900002F019FA430803F1376303F5D833B3FBC5
:100CA000F0F002B0BDE8F04706F0FEB9FFF7BCFD7A
:100CB0003378D90706D4FFF7D7FCD8F8000002F044
:100CC000EDFDF5E7FFF7DAFD02E0B9F1000F6BD1BA
:100CD0003378DA0768D54FF4FA70DFF890915A4DFF
:100CE00005F094FE2068D9F8007002F00AFA57491E
:100CF00003463A46564807F051FF206802F0F5F9DE
:100D0000032800F38580286802F08AFE514B524A7E
:100D10005249002818BF1A464D4807F03FFF4C487B
:100D20004F4907F03BFF206802F07AFE18B94848A7
:100D30004C4907F033FF07F0B3FB00287DD0317832
:100D400011F001014FF000052ED0AA227723009563
:100D5000206802F054F929460A2005F025FD206894
:100D600002F002FD206802F0C0F90328D4BF4FF45E
:100D70007A7040F2E24005F049FE0A20012105F0B8
:100D800013FD01210A2005F0EFFC206802F00EFAA5
:100D9000206802F066F9192005F038FE0A20D9F81B
:100DA000001004F045FD002596F8009009F00109B7
:100DB00007F076FB88B107F031FB80230093824671
:100DC0000121D8F80000FF22002302F018F95FFA91
:100DD0008AF0013504F0A2FDEAE704F075FD88B160
:100DE00004F082FD8023009382460121D8F80000A0
:100DF0000022FF2302F003F91548026851461268E9
:100E00009047EAE7206802F049FDFFF72DFC2AE74A
:100E1000286802F025FD8246286802F021FD0A2399
:100E200090FBF3F19AFBF3F201FB130312B20E49AC
:100E300007481BB207F0B2FE71E73378DB077FF596
:100E40007EAF78E77C91FF1FB088FF1FB1AC000038
:100E5000C891FF1F7CAB000078AB000084AB0000A2
:100E6000B4AB00000BAC00009AAB0000F091FF1F88
:100E70002DE9F74F854F3B6893F8806016F0100F0F
:100E800006F004080AD0B8F1000F04D003B0BDE8A2
:100E9000F04FFFF7DDBE1B2004F014FA16F0020F2E
:100EA0007B4C7C4D0DD022687B4B0AB9236001E05E
:100EB0007A4A13602A7802230AB9764A00E0784A0F
:100EC0001370B8F1000F0DD02268764B0AB9704A42
:100ED00000E0724A13602A7804230AB96D4A00E0E0
:100EE0006F4A137033070DD522686F4B0AB9684AF1
:100EF00000E06A4A13602A7808230AB9654A00E0CC
:100F0000674A1370F0070DD52268684B0AB9604A2A
:100F100000E0624A13602A7801230AB95D4A00E0C2
:100F20005F4A1370624E96F8008008F00108802333
:100F30000093002213463868012102F060F82B78F4
:100F4000012B03D0564B1B78012B3CD13378D907AA
:100F50001FD42368554A934208BF504B4E4A08BFDE
:100F60001B68934202D105F02DFE0AE04D4A9342E0
:100F700002D106F00DF904E04B4A934201D106F08C
:100F8000DDFB3378DA07FCD54FF4FA7005F03EFD4F
:100F900002E0B8F1000F16D13378DB0713D52368D0
:100FA000424A934201D13D4B1B683B4A93424FD189
:100FB000404B1868430803F1376303F5D833B3FB9C
:100FC000F0F005F087FD96F8008008F00108206831
:100FD000DFF8C89003689B689847B0B180230093FE
:100FE00038680121FF22002302F009F8D9F80090A7
:100FF000D9F80030D3F800A0254B18680368DB68E7
:101000009847C1B24846D047E1E7D9F800000368E5
:101010009B689847B0B18023009338680121002273
:10102000FF2301F0ECFFD4F800A0DAF80030D3F889
:1010300000B01A4B18680368DB689847C1B2504685
:10104000D847E2E7386802F029FCFFF70DFB6EE7AE
:10105000144A93420BD1174B1868430803F13763C6
:1010600003F5D833B3FBF0F006F01EF8ABE70E4AF9
:101070009342A8D10F4B1868430803F1B76303F5F7
:101080005843B3FBF0F006F0EDFA9CE7B088FF1F81
:10109000C888FF1FC488FF1F8091FF1FC088FF1FE3
:1010A000C588FF1F9091FF1FA091FF1FC891FF1FD0
:1010B0007C91FF1FF091FF1F38B5044608460D468E
:1010C00008F037FF236802465B68204629469847A8
:1010D00038BDFFFF38B5002504460571457180F81D
:1010E000505004491422063008F042FFA4F84E5034
:1010F000204638BDEDAC00000079704738B5074B8D
:1011000090F8512053F832300124054683F880408E
:10111000962005F07BFC2C71204638BDF0CC0000F9
:1011200038B5084B90F8512053F832300124054669
:1011300083F80041962005F069FC00232B712046BE
:1011400038BD00BFF0CC000090F85130427933B187
:1011500090F85230D3F1010038BF002000E00120A8
:101160001043704706307047B0F94E007047FFFFDC
:1011700038B50446006803681B6A98472046FFF7A5
:10118000CFFF94F852200E4B53F83230012583F8EC
:1011900080500A2005F03AFC2046FFF7AFFF206898
:1011A000084B20221A6003684FF416419B69984748
:1011B00040F2EE2005F02AFC84F8505038BD00BF04
:1011C000F0CC000084F00F4070B50446006803685E
:1011D0001B6A98472046FFF7A3FF94F852200E4B56
:1011E00053F83230012283F800210A2005F00EFC6A
:1011F0002046FFF783FF2568084B20221A602B68E2
:101200009E69074B186801F067FF01462846B04702
:10121000002384F8503070BDF0CC000088F00F40FF
:10122000B088FF1F70B58EB0322201A80E4600258F
:1012300008F09EFE01A83A218DF8355008F05AFEBC
:10124000044608B9307012E04378222B0BD101A874
:10125000294608F04FFE30B110F8012C222A04BFB5
:1012600000F8015C01343046611C08F05AFE0EB0F3
:1012700070BD2DE9F84300250746884691460D705C
:101280002C462E46386803689B68984758B33868E0
:101290000368DB689847C0B20EB945282FD00136E5
:1012A0000D28F6B203D1002308F804300BE00A2819
:1012B000F9D009F1FF339C42F5D008F8040001345D
:1012C000E4B20025DEE7386803689B68984738B1C8
:1012D00038680368DB6898470A2005F097FBF2E757
:1012E0000120BDE8F88301350A20EDB205F08EFB40
:1012F000312DC7D9201C18BF0120BDE8F883304626
:10130000BDE8F88370B5044625460679FFF730FF3F
:10131000002355F81A0B0E496371FFF7CDFE2046E6
:1013200029463222FFF7A5FF38B128460949022293
:1013300008F007FE08B9012300E00023637120468E
:10134000FFF742FF16B92046FFF7EAFE607970BD4D
:1013500010AD00000DAD0000437970B50446F3B147
:1013600090F850600EB9FFF703FF25460C4955F879
:101370001A0BFFF7A1FE322229462046FFF779FF1C
:1013800020462946FFF74EFFA01D2946142208F0EB
:10139000EFFD26B92046BDE87040FFF715BF70BDD0
:1013A00015AD0000437970B50446F3B190F8506074
:1013B0000EB9FFF7DDFE25460C4955F81A0BFFF76D
:1013C0007BFE322229462046FFF753FF204629465E
:1013D000FFF728FF284608F038FCA4F84E0026B98D
:1013E0002046BDE87040FFF7EFBE70BD20AD0000A5
:1013F00070B5244D01602A6892F8713080F8513040
:10140000044692F8720084F8520003B150B91E4BA2
:10141000063403F1140253F8041B44F8041B9342EE
:10142000F9D170BD012105F0BFF994F85220174B96
:1014300053F83230012183F8001194F8510005F07F
:10144000B3F92046FFF75AFE2046FFF75BFF6379AA
:10145000BBB12046FFF78CFE2046FFF7A3FF2046D6
:10146000FFF77AFF2046FFF7AFFE2046FFF746FE64
:101470002468286823689E6901F02EFE01462046F4
:10148000B04770BDB088FF1F2BAD0000F0CC00004E
:10149000F8B5437904460F4643B390F850600EB94F
:1014A000FFF766FE25463A461149206807F076FBAD
:1014B00055F81A0B0F49FFF7FFFD20462946322247
:1014C000FFF7D7FE60B128460B49022208F039FD2C
:1014D00030B9A01D3946142208F04AFD012500E06C
:1014E000002516B92046FFF76FFE2B461846F8BDBB
:1014F0003FAD000028AD00000DAD0000437970B590
:1015000004460D462BB390F850600EB9FFF730FE3D
:101510002A4625461049206807F040FB55F81A0B6B
:101520000E49FFF7C9FD204629463222FFF7A1FEEA
:1015300048B128460A49022208F003FDD0F101050E
:1015400038BF002500E0054616B92046FFF73CFEEF
:101550002B46184670BD00BFFEAC000028AD000051
:101560000DAD0000F8B5437904460F462BB390F853
:1015700050600EB9FFF7FCFD25463A461049206839
:1015800007F00CFB55F81A0B0E49FFF795FD2046A6
:1015900029463222FFF76DFE48B128460A49022249
:1015A00008F0CFFC18B9A4F84E70012500E0002522
:1015B00016B92046FFF708FE2B461846F8BD00BFB7
:1015C0004AAD000028AD00000DAD0000F8B543792C
:1015D00004460F4600F11A050BB9837615E090F822
:1015E00050600EB9FFF7C4FD39462068FFF764FD6F
:1015F00007492068FFF760FD204629463222FFF7A1
:1016000038FE16B92046FFF7DFFD2846F8BD00BFBB
:1016100028AD00000023012110B50A46044683814D
:10162000C381094B4FF4BF7003F084FE0421206096
:101630000122064B4FF4BF7003F07CFE4223606032
:10164000A360204610BD00BF57AD000068AD00008C
:101650000A23034AB1FBF3F1B2FBF1F38360704755
:1016600030D4050010B50446006808F03FFB606800
:1016700008F03CFB204610BDB0F90E20036810B501
:1016800099540A4AC3891468426819B29BB242F855
:1016900021405A1C92B211B2B1F5BF7FA5BF6FF4C1
:1016A000BE729B18C281C38110BD00BFCC89FF1FD1
:1016B000C289838911B218B28842C8BF02F5BF72CD
:1016C000D31A98B200B2704738B50D460446FFF7FA
:1016D000EFFF854204DB062003F0F4FD002038BD57
:1016E000A3891D44ADB2ABB21AB2B2F5BF7FA4BF9D
:1016F000A5F5BF739BB21BB22268D05C38BD82894E
:10170000C089531E9BB2190444BF02F27D139BB2E1
:101710001B1A58425841704700238381C381704788
:1017200038B50D460446FFF7C3FF854204DD0820A7
:10173000BDE8384003F0C6BDA3891D44ADB2ABB2CD
:101740001AB2B2F5BF7FAABFA5F5BF75A381A58167
:1017500038BDFFFF38B50B4B1D6883680446ED1A92
:101760002046FFF7A5FF00280BDDB4F90C206368C5
:1017700053F82230AB4204D820460121FFF7D0FFB6
:10178000EEE738BDCC89FF1F014B0360704700BFF7
:10179000B8AD0000014B0360704700BFB8AD00005A
:1017A00010B5034B0360044607F0BFF9204610BD97
:1017B000B8AD000010B5034B0360044607F0B5F95F
:1017C000204610BDB8AD000030B585B004AC04E9CA
:1017D0000E00089C34B940681A4905B0BDE8304095
:1017E00007F0DCB99DF80430022B07D0032B1ED183
:1017F0001549227C406807F0D1F91CE0B4F90C20AF
:10180000237C012A04D1A2684068104912780BE0B9
:10181000022A07D1A16840680A784D780B4902EB8B
:10182000052201E040680A4907F0B8F903E00948D9
:10183000094907F0B3F9204605B0BDE8304008F08B
:1018400055BA00BFE8AD0000E4B40000F5AD0000FB
:1018500000AE0000C891FF1F1AAE000038B5044664
:1018600008460D4608F065FB236802465B68204683
:101870002946984738BD38B50446FFF7EFFF0546BF
:10188000204607F075F9284438BDFFFFF8B5124F20
:10189000124B03600025FA26044680F8795080F840
:1018A0008D504160426680F8485080F86050A0F842
:1018B0006C602A463B463046012103F03BFDA4F80C
:1018C00080602067012130462A463B4603F032FD06
:1018D000C4F884002046F8BD46AE0000D8AD000034
:1018E0004068014907F05AB956AE00002DE9F041B1
:1018F000244BDFF894801B888AB005A9ADF814301A
:10190000D8F800301A6800910221002400F168071D
:101910000191D5698DF81D40184639460322FE23F2
:10192000A8476D4607AE45F8044B96E8070085E8E2
:1019300007002346D8F800003946224603F08EFC03
:10194000D8F800008DF819401E238DF818308DF856
:101950001A4006AA0368009203220192D3F81CC021
:101960003946FE23E047009496E8070085E8070023
:101970002346D8F800003946224603F06FFC0AB02F
:10198000BDE8F081C8AD0000B888FF1F406801497C
:1019900007F004B9E6AE00000A4B10B5044618681B
:1019A0000023C218013300210A2B82F85410F8D109
:1019B000054B18680268526A904760680349FFF750
:1019C0005AFF10BDB088FF1FB888FF1F5DAF000031
:1019D0002DE9F743854D86490446406807F0DEF857
:1019E0002868666801F08DFB82490246304607F0A0
:1019F000D5F88149606807F0D1F82868666801F079
:101A000074FB7E490246304607F0C8F828686668CD
:101A100001F071FB7A490246304607F0BFF82868AA
:101A2000D4F8048001F076FB0746286801F078FBC3
:101A30000646286801F07AFB3346009071493A4621
:101A4000404607F0ABF860686F4907F0A7F82B68CD
:101A50001B7A13B960686D4908E0022B02D16068F7
:101A60006B4903E0012B03D160686A4907F096F8DF
:101A70006068694907F092F82B6860681B7C0BB1BD
:101A8000664900E06649674E07F088F83068FFF75E
:101A90005BFB374610B16068634901E060686349E9
:101AA00007F07CF82B686249B3F8742060680A2359
:101AB000B2FBF3F207F072F82868666801F042FBA7
:101AC0005C490246304607F069F860685A4907F0F9
:101AD00065F8286801F030FB10B16068574901E0F3
:101AE0006068574907F05AF856496068FFF7B6FE34
:101AF0002868666801F02CFB53490246304607F01F
:101B00004DF82868D4F8048001F0C5FA0646286824
:101B100001F0BEFA324603464C49404607F03EF813
:101B20002868666801F0BDFA49490246304607F068
:101B300035F82868666801F0BCFA464B464A4749C2
:101B4000002818BF1A46304607F028F84449606854
:101B5000264EFFF783FE2868D4F8049001F0B6FA09
:101B60008046286801F0AFFA3E490346424648469F
:101B700007F014F83C4B656818680268526B904790
:101B80003A490246284607F009F83868254DFFF71C
:101B9000DBFA18B33068D4F8048001F0A0FA0746E5
:101BA000306801F099FA3A4603463149404606F05A
:101BB000F5FF28686668FFF7D5FA2E4902463046D9
:101BC00006F0ECFF28686468FFF7CEFA2A4902465F
:101BD000204603B0BDE8F04306F0E0BF6068274947
:101BE00003B0BDE8F04306F0D9BF00BFB088FF1FC7
:101BF000A2AF0000BFAF0000EDAF0000FCAF0000DF
:101C000010B0000026B0000044B0000056B0000044
:101C100065B0000082B00000A2B00000C9B00000B2
:101C2000E6B00000A488FF1FB7B00000D4B00000E9
:101C3000F5B000001AB100003DB1000051B1000044
:101C400088B10000BFB10000E7B1000000B20000A1
:101C500020B200009BAF00009FAF000039B200002F
:101C600052B2000079B20000B888FF1FA7B200008E
:101C7000D1B20000FBB2000017B3000035B3000082
:101C80002DE9F041854D0446286801F0E9FD8449BD
:101C90000646606806F082FF8249606806F07EFFB3
:101CA000286801F022FA03280EDC60680EB97E492C
:101CB00002E0012E03D17D4906F070FF0FE07C4960
:101CC000324606F06BFF0AE00A2396FBF3F203FBB1
:101CD00012636068774912B21BB206F05FFF286892
:101CE0006768C1886D4E09B201F0B0FD0A2290FB11
:101CF000F2F2714912B2384606F050FF286801F03E
:101D0000F4F903280DDD33686C4993F8842060688A
:101D100006F044FF336860686949B3F8822006F032
:101D20003DFF28685D4E01F0E0F903280FDD3368C0
:101D30006449B3F86C20606892B206F02FFF3368F4
:101D40006068B3F86A20604992B206F027FF6068C5
:101D50005E4906F023FF2B681A7A22B960685C4955
:101D600006F01CFF18E0022A03D1DA89606859499D
:101D70000FE0012A10D1DA899B89564960689BB22D
:101D800092B2D21A06F00AFF444B60681B685249AF
:101D90009A8992B206F002FF2B681A7C6AB19A8A7D
:101DA0004E49606812B206F0F9FE3C4B60681B6851
:101DB0004B49DA8A12B206F0F1FE4A49606806F031
:101DC000EDFE2868666801F0C3F9474902463046CF
:101DD00006F0E4FE00262B68334493F854202AB121
:101DE0006068424993F85E3006F0D8FE01360A2E4C
:101DF000F1D13F49606806F0D1FE286801F075F91D
:101E00000328CCBF4FF00A084FF0040800222B68CB
:101E100067689818D1B290F84A00561C30B118463D
:101E200001F0D0FD33490346384605E0184601F07D
:101E3000C9FD314903463846324606F0AFFEF3B2DB
:101E400043453246E3D32D4D2868FFF77DF960B155
:101E500028686668FFF750F9294B2A4A2A49002862
:101E600018BF1A46304606F099FE6068274906F00A
:101E700095FE274B60681A78264906F08FFE264BA0
:101E800060681A78254906F089FE254B6068254967
:101E90001A78BDE8F04106F081BE00BFB088FF1F90
:101EA0005CB3000080B300008FB3000093B3000068
:101EB0009CB30000D7B30000DFB30000F3B3000011
:101EC00005B4000014B4000029B400003DB40000C3
:101ED00056B000000CB0000051B400006DB400001A
:101EE00084B400009BB40000CDB40000DFB4000057
:101EF000EAB4000003B5000021B50000A488FF1F6C
:101F000055B3000058B300002EB5000043B50000E3
:101F1000E491FF1F58B50000D488FF1F7EB5000074
:101F2000E591FF1FA4B5000038B51A490446406882
:101F300006F034FE184B6568186801F0E2F817499E
:101F40000246284606F02AFE6068154906F026FE7D
:101F50006068144906F022FE6068134906F01EFE10
:101F60006068124906F01AFE6068114906F016FE14
:101F70006068104906F012FE60680F4906F00EFE18
:101F800060680E4906F00AFE60680D49BDE83840F9
:101F900006F004BEA2AF0000B088FF1FBFAF000074
:101FA000CAB500009FB60000B2B60000BFB6000080
:101FB000D8B60000FAB6000026B7000044B700000B
:101FC00063B7000070B5294D29490446406806F002
:101FD000E5FD2868666801F094F826490246304617
:101FE00006F0DCFD2449606806F0D8FD23496068EE
:101FF00006F0D4FD2249606806F0D0FD21496068F2
:1020000006F0CCFD2049606806F0C8FD286801F0A4
:102010006CF8032803DD60681C4906F0BFFD2868E2
:10202000666801F08CF81A490246304606F0B6FDA3
:102030006068184906F0B2FD6068174906F0AEFD09
:102040006068164906F0AAFD6068154906F0A6FD0D
:102050006068144906F0A2FD6068134906F09EFD11
:1020600060681249BDE8704006F098BDB088FF1F57
:10207000A2AF0000BFAF0000B1B70000F0B7000092
:1020800004B800002BB8000050B8000089B8000068
:10209000C8B8000011B9000054B90000E5B900004B
:1020A00050BA00008EBA0000CBBA0000FDBA0000A2
:1020B0004068014906F072BD30BB00002DE9F047D1
:1020C000032988B004460D4602D0FFF7F1FF4CE02B
:1020D000006D07F0BAFD8146606D07F0B6FD244B38
:1020E0005FFA89F882464146186801F039F810B95C
:1020F0006068204906E00FFA8AF7B7F5805F04DBD5
:1021000060681D4906F04AFD2FE01E238DF810304F
:102110003B128DF81230194B19491A680097194F64
:1021200019488DF811A0002612B20FFA89F38DF824
:10213000156006F033FD386804AA03688DE82400B2
:1021400068342A46D3F81CC021464346E0476B4614
:1021500008AD43F8046B15E9070083E80700214642
:1021600038683246334603F079F808B0BDE8F087A6
:10217000B088FF1F81BB0000CDBB0000CC89FF1FD2
:1021800035BC0000B888FF1FC891FF1F2DE9F04340
:10219000042989B00446894602D0FFF789FF69E027
:1021A000006D07F052FD0546606D07F04EFD80465C
:1021B000A06D07F04AFD03B2FF2B074603DD606800
:1021C0002E4908224FE02E4EEDB2306829465FFAC4
:1021D00088F800F0C5FF30B38DF81170294F8DF8E5
:1021E0001080386804A900238DF815300368009129
:1021F00002210191032204F16806D3F81CC08DF876
:1022000014202B466D463146E04745F8044B08AB99
:1022100013E9070085E807004B463868314601227C
:1022200003F01CF826E0306800F092FF85421DD1D3
:102230000A2384F86830032384F86A300223A4F860
:102240007430236F84F8695083F80080236F5F70C7
:10225000306804F1680104F17C0201F059FE606805
:10226000064994F88C2006F099FC03E06068064962
:1022700006F094FC09B0BDE8F08300BFE4B40000B0
:10228000B088FF1FB888FF1F51BC00002DE9F04146
:10229000032988B0044602D0FFF70AFF61E0006D11
:1022A000314E07F0D2FCC5B2606D07F0CEFC294676
:1022B000C7B2306800F054FF50B3DFF8B8808DF833
:1022C0001070D8F80000012600238DF811608DF8F9
:1022D000153004A9022302688DF814308DE80A0035
:1022E00004F16807D2F81CC039461A462B46E0476D
:1022F0006B4643F8044B08AC14E9070083E8070079
:102300003946D8F800003246042302F0A7FF28E03F
:10231000306800F01DFF85421FD10A2384F8683021
:10232000022384F86A30A4F87430236F84F869506B
:102330001F70236F01225A70306804F1680104F1A4
:102340007C0201F08DFBD4F8843060681A7807496C
:1023500094F88C3006F022FC03E06068044906F033
:102360001DFC08B0BDE8F081B088FF1FF5AD00008E
:1023700051BC0000B888FF1F2DE9F047042988B040
:102380000446894602D0FFF793FE69E0006D364EA1
:1023900007F05BFCC5B2606D07F057FC5FFA80FA8E
:1023A000A06D07F052FC294607461FFA80F83068F6
:1023B00000F0D6FE48B38DF811702C4F8DF810A0A8
:1023C000386848F3072803228DF8128004A90023F7
:1023D0008DF8153003688DF814208DE8060004F19F
:1023E0006806D3F81CC02B466D463146E04745F8D9
:1023F000044B08AB13E9070085E807004B46386833
:102400003146012202F02AFF2AE0306800F0A0FEE7
:10241000854221D10A2384F86830032384F86A3086
:10242000A4F87430236F84F8695083F800A0236FF8
:102430005F70236F48F3072883F80280306804F147
:10244000680104F17C0201F063FD6068084994F8BA
:102450008C2006F0A3FB03E06068064906F09EFBB3
:1024600008B0BDE8F08700BFB088FF1FB888FF1F25
:10247000E4B4000051BC00002DE9F041032988B00C
:102480000446884602D0FFF713FE5EE0006D304E32
:1024900007F0DBFBC5B2606D07F0D7FB2946C7B27A
:1024A000306800F05DFE28B38DF81070294F0222CD
:1024B00038688DF8112004A900238DF815300368C1
:1024C0008DF814208DE8060004F16806D3F81CC0CE
:1024D00031462B46E0476B4643F8044B08AC14E901
:1024E000070083E80700314638680122042302F020
:1024F000B5FE2AE0306800F02BFE854221D1226F24
:1025000084F869500A2384F86830022384F86A301A
:10251000A4F874801770226F5370306804F168015A
:1025200004F17C0201F09CFAD4F8843060681A78D7
:102530005B78094902EB032294F88C3006F02EFBFD
:1025400003E06068054906F029FB08B0BDE8F081AA
:10255000B088FF1FB888FF1FF5AD000051BC000018
:10256000022938B5044604D02046BDE83840FFF7BC
:102570009FBD056D1049284607F0C9FC60B90F4B97
:10258000186801F025F94FF47A6004F03FFA6068AA
:102590000B49FFF770F938BD28460A4907F0B7FC28
:1025A0000028E1D1054C206801F0DEF82068BDE884
:1025B000384001F02FB900BF5BBC0000B088FF1F9E
:1025C0005FBC000064BC0000022910B5044603D0C3
:1025D000BDE81040FFF76CBD006D07F036FB094BFE
:1025E000C1B2186801F01EF930B96068226D064961
:1025F000BDE8104006F0D2BA60680449FFF73BF925
:1026000010BD00BFB088FF1F68BC0000AEBC00005A
:10261000022938B5044603D0BDE83840FFF748BD6D
:102620000B4D286800F061FD032805DC2046FFF70C
:102630003FFD6068074907E0206D2D6807F005FB46
:1026400085F8840060680449FFF715F938BD00BFBC
:10265000B088FF1FB4BC0000AEBC0000032970B5F9
:1026600004462FD1056D7649284607F050FCA0B9E5
:10267000656D7449284607F04AFC18B9724B012170
:10268000186807E07149284607F041FC0146C8B9BF
:102690006D4B186800F010FD87E028466C4907F084
:1026A00036FCA0B128466B4907F031FC58BB656D7C
:1026B0006949284607F02BFCF8B12846674907F01E
:1026C00026FCD0B12046BDE87040FFF7F1BC656D37
:1026D0005C49284607F01BFC18B95B4B01211868C0
:1026E00008E05A49284607F012FC01460028E9D1C3
:1026F000554B186800F055FD57E0534B0121186801
:1027000001F0A6F951E02846554907F000FC48B908
:102710004D4B606D1D6807F098FAC1B2284600F075
:10272000D8FC42E028464F4907F0F1FB002841D190
:10273000606D07F08EFACF28054602DD60684A49D1
:1027400035E04A4B013093FBF0F007F019F84849A7
:1027500007F01EF90021064607F018FA28B13046A6
:102760004FF07C5106F058FF04E030464FF07C51AA
:1027700006F050FF07F01EFA3E4A03464FF416518A
:1027800010685943FEF7BAFE10B160683A4901E09B
:1027900060683A4906F002FA2B4BE9B2186800F07B
:1027A000A1FC60683649FFF766F860683549FFF7B5
:1027B00062F870BD2846344907F0A9FB70B92D4B6B
:1027C000616D1868FEF764FE10B160682F4901E082
:1027D00060682F49BDE8704006F0E0B928462D49F1
:1027E00007F095FBC0B9606D07F02FFA42F20F7346
:1027F00001B2994202DD60682749EBE71D4D286868
:10280000FEF7B0FE0028E3D028686468FEF7ACFC51
:102810002249024620460FE02846214907F077FB6F
:1028200000287FF44FAF134B616D18686568FEF7A1
:10283000CDFE1C4902462846BDE8704006F0AEB900
:10284000E9BC0000F5BC0000B088FF1FF9BC000027
:10285000FCBC00000CBD000016BD000019BD00004E
:102860001DBD000025BD00002CBD000080841E00A1
:1028700000001646A488FF1F78BD000097BD000029
:10288000B6BD00005FBC0000DABD0000E1BD000085
:10289000E9BD0000EFBD0000F6BD000044BE000031
:1028A0007BBE000085BE0000022970B504460D46BF
:1028B00008D1006D3C4907F02AFB002849D102F0FD
:1028C00061FE6BE0032944D1056D3849284607F0C5
:1028D0001EFB48B9364B606D1D6807F0B6F901B2B2
:1028E000284600F005FC59E02846324907F00FFB66
:1028F00048B92F4B606D1D6807F0A7F901B2284653
:1029000000F0FCFB4AE028462B4907F000FB48B9E1
:10291000274B606D1D6807F098F901B2284600F05A
:1029200014FC3BE02846254907F0F1FAB0B9656D83
:102930002349284607F0EBFA08B9282005E0284685
:10294000204907F0E4FA48B91E20012102F000FEF8
:1029500024E0206D1C4907F0DAFA20B12046BDE8DA
:102960007040FFF7A5BB052DF8D1114D606D2E68A5
:1029700007F06BF9C1B2304600F0CFFBA06D2E68B6
:1029800007F063F9C1B2304600F0CDFBE06D2D6871
:1029900007F05BF9C1B2284600F0CBFB60680B4939
:1029A000FEF769FF70BD00BF90BE000097BE00003B
:1029B000B088FF1FA2BE0000B0BE0000C0BE000075
:1029C000CBBE0000D0BE0000D6BE00005FBC000041
:1029D00070B590F848303F2B84BF3F2380F84830D3
:1029E00090F84830034400221A7204460E460A70DA
:1029F000012394F84800D1B288420DD92144097AC4
:102A0000202904D02BB133780133337001E0012346
:102A100000E000230132ECE73378052BA8BF052343
:102A20003370002304F1080584F860302846202123
:102A300094F8482007F062F994F8603018B904EB74
:102A40008302D5640CE0A84201D101350BE004EB10
:102A50008303DD640546002305F8013B94F86030EC
:102A6000013384F8603094F8602033789A42DDD3E3
:102A7000E46C207808B9307070BD2046474907F0F3
:102A800046FA002867D02046454907F040FA00285A
:102A900063D02046434907F03AFA00285FD0204629
:102AA000414907F034FA00285BD020463F4907F03F
:102AB0002EFA002857D020463D4907F028FA002872
:102AC00053D020463B4907F022FA00284FD0204639
:102AD000394907F01CFA00284BD02046374907F047
:102AE00016FA002847D02046354907F010FA00288A
:102AF00043D02046334907F00AFA00283FD0204649
:102B0000314907F004FA00283BD020462F4907F04E
:102B1000FEF9002837D020462D4907F0F8F90028A3
:102B200033D020462B4907F0F2F900282FD0204659
:102B3000294907F0ECF900282BD02046274907F057
:102B4000E6F940B32046264907F0E1F9002814BF12
:102B50000120112070BD022070BD032070BD042033
:102B600070BD052070BD062070BD072070BD082017
:102B700070BD092070BD0A2070BD0B2070BD0C20F7
:102B800070BD0D2070BD122070BD132070BD0E20D1
:102B900070BD0F2070BD102070BD00BFD9BE0000F9
:102BA000DEBE0000E2BE0000E9BE0000EFBE000095
:102BB00001BF0000F7BE0000FDBE000006BF000020
:102BC0000DBF0000D1C00000A9BE000015BF00006D
:102BD00020BF000027BF00002BBF00002FBF000058
:102BE00033BF000038B50D4C0546206800F07DFA73
:102BF000032811DD206800F078FA20280CD0206826
:102C000000F073FAFE2807D005496868FEF733FE26
:102C100068680449FEF72FFE38BD00BFB088FF1F6B
:102C200037BF0000B0BF000037B5044660680368D6
:102C30009B689847002800F09D8060680368DB6807
:102C40009847C0B20D28F1D00A2804D094F8483033
:102C50003F2B40F0898020460DF10701FFF7B8FEB9
:102C6000A0F11003DBB2012B054606D90E285CD07B
:102C70000F2860D02046FFF7B5FF132D6DD8DFE891
:102C800005F06F0A0E12161A1E22262A30363C4212
:102C9000545A6066484E2046FFF70AFA60E0204624
:102CA000FFF790F95CE02046FFF73EF958E0204638
:102CB000FEF7E6FF54E02046FEF78AFE50E020468D
:102CC000FEF76AFE4CE02046FEF710FE48E0204684
:102CD000FEF75CFE44E020469DF80710FEF700FE7C
:102CE0003EE020469DF80710FFF7E8F938E020465F
:102CF0009DF80710FFF734FC32E020469DF80710DE
:102D0000FFF7D2FD2CE020469DF80710FFF7A6FC48
:102D100026E020469DF80710FFF756FC20E02046ED
:102D20009DF80710FFF774FC1AE020469DF8071085
:102D3000FFF72CFA14E020469DF80710FFF71CFB64
:102D40000EE020469DF80710FFF7A0FA08E02046A5
:102D50009DF80710FFF790FB02E00D2002F0B2FA99
:102D6000002384F8483005E05A1C234484F84820A6
:102D700018725BE703B030BD10B5044600F026F8CA
:102D8000204610BDF0B589B06B4600248DF8154083
:102D900043F8044B08AF06460D4617E9070083E8E1
:102DA0000700304629462246234600F084F809B041
:102DB000F0BD08B500F0D3F8043008BD00F00AB942
:102DC00000F014B900F009B900F012B9F8B50FB26B
:102DD00004460D461646282100222C4B384602F0A8
:102DE000A9FA206106FB05F00022294B00B201215F
:102DF00002F0A0FA002360610246D9B2A94208D2CB
:102E00002169282000FB03110133CA600E8132447E
:102E1000F3E70C2101221F4B384602F08BFA0C26F7
:102E20006FF00B01034600F10C0216FB0511606008
:102E300006FB053682605A1820691860183E5A60F1
:102E40005660282606FB0506283E5E509360012248
:102E5000691E8A4213DA0C2112FB01F601FB023CC7
:102E60009F1911FB021119444CF8087CB96002EB60
:102E7000820100EBC10101329951D2B2E8E7A360AF
:102E8000E360002323702046F8BD00BF04C00000AB
:102E90001DC0000041C0000010B50446406906F0A6
:102EA00025FF206906F022FF606806F01FFF00235F
:102EB0002370204610BD2DE9F843904602789946CC
:102EC0000446836812B91D46E36009E0C568AA6834
:102ED0009A4205D1192002F0F5F90020BDE8F883E7
:102EE000E3682E689B68E360F06833890F46321D03
:102EF00001F1140E57F804CB42F804CB7745F9D111
:102F0000B1F90C7033811BB29F42A8BF1F46F0601D
:102F1000BAB23282896812B206F0FFFE2968089AB6
:102F200081F82590286881F82480034643F81A2BFD
:102F300008AA52F8061FC0F81A10516812891A819F
:102F400059602B689DF824201A762B689DF825205F
:102F50005A762378013323700120BDE8F88310B539
:102F6000047814B18368186810BD152002F0AAF91E
:102F7000204610BD38B503788B4204460D4604DC6C
:102F80001720BDE8384002F09DB919B983689B68E5
:102F900083601BE0013B994203D1C3685B68C36057
:102FA00014E0182002F08EF9A368013D15F0FF052A
:102FB0009B68FAD15A689968916099684A60E2689A
:102FC0009168996091685A604B6093602378013BE7
:102FD000237038BD0021FFF7CDBF10B5044623781C
:102FE0001BB12046FFF7F6FFF9E710BD00787047E8
:102FF000C36880689A68131A58425841704770B580
:1030000004461E469DF8105029B980F8902084F897
:10301000923080F8915094F88F3094F88C008BB1F6
:10302000D243D1B20131F64303F0EEFBF1B294F892
:103030008D000131ED4303F0E7FBE9B294F88E0017
:1030400001310AE0511C03F0DFFB94F88D00711C84
:1030500003F0DAFB94F88E00691CBDE8704003F0C1
:10306000D3BB07B590F89110009190F8902090F89C
:1030700092300121FFF7C3FF03B05DF804FB90F825
:103080009000704790F89200704790F89100704758
:10309000D0F89400704790F8930070470B2002F02E
:1030A0001FBA90F89800704780F898100D2002F031
:1030B00017BA90F89A0070470A461720012102B10A
:1030C0000A4602F0BBB9D0F89C00704790F89B000C
:1030D00070470F2002F004BAD0F8A400704790F8AF
:1030E000A0007047102002F0FBB9B0F9A8007047AB
:1030F000002002F011BAB0F9AA007047022002F0D5
:103100000BBA90F8AF00704780F8AF100A20252165
:1031100002F0E6B990F8B0007047042002F0E0B980
:1031200090F8B1007047052002F0DAB990F8B200CB
:103130007047062002F0D4B990F8AE007047B0F99D
:10314000AC007047B0F9B40070471A2002F0E4B93F
:1031500090F89900704780F899100E2002F0C0B9DD
:1031600059B10023C21892F854208A4203D0013387
:103170000A2BF7D101E0012070470020704710B5FD
:1031800059B10023C418DAB294F854408C4201D1EA
:10319000104604E001330A2BF4D14FF6FF7000B261
:1031A00010BD0A461720002102F048B990F8B3106C
:1031B00010B5044699B990F86F0003F0F5FAB4F928
:1031C000A830032B01DD202B01D14B2000E006208D
:1031D00003F01CFC012384F8B33084F8773010BD71
:1031E000F7B504460A2002F01BF9252884F8AF0041
:1031F00003D020462521FFF787FF002002F016F9B3
:10320000A4F8A800022002F011F9A4F8AA000D20E9
:1032100002F006F984F898000B2002F001F984F816
:10322000930002F02BF80121C4F89400172002F05B
:10323000E5F8003018BF012084F89A000E2002F053
:10324000EFF884F899000F2002F0EAF884F89B0068
:1032500002F014F8C4F89C00102002F0E1F884F8A1
:10326000A00002F00BF8C4F8A400042002F0D8F883
:1032700084F8B000052002F0D3F884F8B1000620ED
:1032800002F0CEF8022184F8B200172002F0B6F85E
:10329000003018BF01200021022384F8850084F843
:1032A000801084F88430172002F0A8F8003018BF8E
:1032B000012084F8AE0010B140F6FF7301E040F247
:1032C000FF33A4F8AC30B4F8AA3013F0010204D1F3
:1032D00003F0200292B202B1022259062272C3F315
:1032E000400222744CBF18220C22C4F888205A07CE
:1032F00001D5322304E01B074CBF50234FF6FF7368
:103300000025A4F8743084F8B3501A2002F08EF827
:10331000B4F8AA30A4F8B400C3F3001384F88F30D3
:103320004FF44873A4F87A304FF49663A4F87C30D5
:10333000012140F2DC53A4F87E300A200A46DE4B1D
:1033400001F0F8FFB4F9A8602060032E5DD12123BD
:1033500084F871301723042084F87230022384F833
:103360006E3084F88C00012103F01EFA052084F8E9
:103370008D00012103F018FA062084F88E00012147
:1033800003F012FA122363722523A37219230B2070
:1033900063740F23A37484F87000012103F004FA0E
:1033A0001D2323711A2323761C2363761523A3760A
:1033B00010231F22E376242384F876202377637773
:1033C000A377E37784F8203084F8213084F86830DC
:1033D00084F8693084F86F202946092003F0E4F965
:1033E0002946202003F0E0F930462946B34D03F08A
:1033F000DBF980260C20012103F0D6F92E60132082
:10340000012103F0D1F92E605AE1202E73D121233E
:1034100084F871301723042084F87230022384F872
:103420006E3084F88C00012103F0BEF9052084F889
:103430008D00012103F0B8F9062084F88E000121E7
:1034400003F0B2F912236372237A012B01D12523F1
:1034500003E0022B0CBF11232423A37219230B209A
:1034600063740F23A37484F87000012103F09CF9A6
:103470001D2323711A2323761C2363761523A37639
:1034800010231F220320E376242384F87620237759
:103490006377A377E37784F8203084F8213084F8C9
:1034A000683084F8693084F86F20014603F07CF9B5
:1034B0000920032103F078F90C20032103F074F9AB
:1034C0000E20032103F070F91320032103F06CF99F
:1034D0001420032103F068F91820032103F064F994
:1034E0001B20032103F060F91E20032103F05CF987
:1034F000202003215AE0042E5BD1032384F871308D
:10350000182384F87230022384F86E30304601218B
:1035100084F88C6003F048F9052084F88D000121BF
:1035200003F042F9062084F88E00012103F03CF9F3
:103530001E206072012103F037F91D23A3721923A5
:10354000202063742123A37484F87000012103F008
:103550002BF91F2384F876300F2323711C23237645
:103560001B2363762423A3762523E3761123237775
:10357000132363771423A3771523E377172384F8A2
:103580002030162384F82130122384F868301A235F
:1035900084F869301020012103F006F91020294633
:1035A00003F0E2F80E2084F86F00294603F0FCF8DF
:1035B00086E0052E7BD1032384F87130182384F82C
:1035C00072301520022384F86E3084F88C000121BB
:1035D00003F0EAF8304684F88D60012103F0E4F846
:1035E000062084F88E00012103F0DEF814206072BA
:1035F000012103F0D9F81023A3721923637420204A
:103600002123A37484F87000012103F0CDF81F2357
:1036100084F876300F2323711C2323761B236376D3
:103620002423A3762523E3761123237713236377BB
:103630002323A3772223E377172384F8203016234C
:1036400084F82130122384F868300E201A2384F87D
:10365000693084F86F00294603F0A6F8092001219B
:1036600003F0A2F82946092003F07EF80B2001217F
:1036700003F09AF829460B2003F076F80C2001217C
:1036800003F092F829460C2003F06EF81D2001216A
:1036900003F08AF829461D2003F066F81E20012158
:1036A00003F082F81E20294603F05EF808E0FE23AE
:1036B000A4F8A83054E000BFC3C0000088F00F4059
:1036C000332301219922009320460023FFF797FC22
:1036D0002046FFF76BFD207902F010FC80B2E080FD
:1036E00094F8760002F00AFCA4F87800A07A02F0C0
:1036F00005FC237C80B2E081A08153B1607C04F0A2
:1037000005FA80B2A082A07C04F000FA80B2E082C8
:1037100001E0A382E382237A5BB1607A012103F0A6
:1037200043F8A07A02F0EAFB80B2A081A3899BB2A1
:1037300000E0A381E38104F10A062546002385F811
:103740005430E386287E85F84A3002F0D7FB2F1BE1
:10375000103704EB4707013580B2B5427880EDD1D0
:10376000204603B0F0BD00BF38B5B0F9A830032B38
:10377000044617DC002580F87750012003F046F955
:10378000114B94F86F001B680121A3F8785003F0E7
:103790000BF894F86F200D4B53F83230012283F868
:1037A000802009E090F86F00012102F0FDFF94F8FD
:1037B0006F00002102F0D8FF002384F8B3300A2004
:1037C000BDE8384003F022B9B088FF1FF0CC0000FC
:1037D00013B5332304460093012100239922FFF7F8
:1037E0000EFC2046FFF7C0FFB4F9A830032B01DD23
:1037F000202B02D14FF47A7001E040F2E24003F056
:1038000005F92046FFF7D2FC204602B0BDE8104083
:10381000FFF727BC014B024A1A6070470CED00E02D
:103820000400FA0511F0E0020ED10B4633B113F09B
:10383000010F1CBF0132D2B25B08F7E7022A03D1A5
:1038400080F8801001207047002070478910EE3901
:1038500021EAE171014B33F911007047D6C0000035
:10386000B0F9A830B0F87800032B08DC40F24C43E4
:10387000984201D980B20EE0B0F5487F03E0202BDA
:1038800005D1B0F5167F94BF0020012003E040F27F
:103890006B135843000B00B27047FFFFB0F9A8301C
:1038A000032B2DE9F041044678DD202B76D03C4AED
:1038B0003C4B15681968691A6429174698466DD9F2
:1038C000FFF7CEFF384B1B68D3F8883090FBF3F03E
:1038D00080B205F0F3FB02460B4605F065FC05F0EF
:1038E00075FE324A13780133DBB213700F22B3FB3B
:1038F000F2F2C2EB02129B1A80B20A2613F0FF0307
:10390000B0FBF6F50CD194F88430002B3DD0B4F820
:1039100082302F2B39D84FF4206393FBF5F532E03A
:10392000012B32D1E188204609B2FFF78FFFB0F5B5
:10393000967FB8BF4FF49670B0F5487FB4BF01468C
:103940004FF44871A1F5967101EB810101EB810102
:1039500089004FF4FA7309B291FBF3F1C1EBC10195
:1039600064224B0193FBF2F394F8842020335343F9
:103970009BB25E434FF4206396FBF5F693FBF5F59F
:10398000AE42B8BF3546A4F8825094F87000B4F83F
:10399000821002F039FF3B68C8F80030BDE8F081C2
:1039A000CC89FF1FD088FF1FB088FF1FCC88FF1F66
:1039B00040F2DE73B0F9B4205943B1FBF2F000B22B
:1039C0007047FFFF084B1B68103103EB410340F2C7
:1039D000DE725B889BB213FB02F3B0F9B420B3FB39
:1039E000F2F000B2704700BFB088FF1F54300021D2
:1039F0000A2206F0B6B95E3000210A2206F0B1B9FB
:103A0000002390F8542012B190F85E2032B90133AF
:103A10000A2B00F10100F4D100207047012070470B
:103A200010B50446FFF71CFF084B1B68B3F9A8301C
:103A3000032B06DD202B04D0B4F8743005339842F4
:103A400000E00028D4BF0020012010BDB088FF1F77
:103A500080F885100A461720022101F0EFBCFFFF15
:103A60002DE9F84F8B68154693F800805A78B5F920
:103A700004309A42B8BF1346DBB208F1FF399944CB
:103A8000AB81002304465FFA89F92B744746C8EBE3
:103A900007064F45F6B200F22E82B82F00F22582BB
:103AA000DFE817F0B9004501BC00C200C8002302DE
:103AB00023022302CE00D400230223022302230286
:103AC00023022302DE00230223022302E400230256
:103AD0002302EA00230223022302230223022302F9
:103AE00023022302230223022302230223022302AE
:103AF0002302230223022302ED00F3002302230208
:103B0000230223022302230223022302230223028D
:103B1000230223022302230223022302FE002302A4
:103B200004010A01100116011C01230222013001C7
:103B300023023701450123023D0123023F014501D4
:103B40002302480123024B015301230251012302A6
:103B50005301720156015D0164016B01230277017B
:103B6000790190012302AA01AD01B401BB01C20198
:103B70002302CC01D401DC01E9012302F90107028F
:103B8000F9010702F9010702F9010702F901070229
:103B9000F9010702F9010702F9010702F901070219
:103BA000F90107022302180218021802180218026B
:103BB0001802180218021802180223022302230214
:103BC00023022302230223022302230223022302CD
:103BD00023022302230223022302230223022302BD
:103BE00023022302230223022302230223022302AD
:103BF000230223022302230223022302230223029D
:103C00001C0223021C0223021C0223021C022302A8
:103C10001C0223021C02AB68952268E12046D5F8FD
:103C200008A0FFF76EFA52E12046D5F808A0FFF78A
:103C30008FFA4CE12046D5F808A0FFF72CFA46E1B0
:103C40002046FFF779FAAB68FF2250E12046D5F80D
:103C500008A0FFF771FA00280CBF03230F2317E118
:103C60002046D5F808A0FFF71CFA30E12046D5F829
:103C700008A0FFF761FA2AE194F8842033E1204696
:103C8000D5F808A0FFF7ECFD21E1E188D5F808A000
:103C9000204609B2FFF7DAFD0A2390FBF3F016E1A4
:103CA0002046D5F808A0FFF720FA10E12046D5F805
:103CB00008A0FFF720FA0AE12046D5F808A0FFF790
:103CC0001AFA03E12046D5F808A0FFF723FAFEE030
:103CD0002046D5F808A0FFF723FAF8E02046D5F8EB
:103CE00008A0FFF723FAF2E02046D5F808A0FFF776
:103CF000C9F983462046FFF7C2F92BF00F0303EB07
:103D00002010E4E02046D5F808A0FFF7BEF9001126
:103D1000DDE02046D5F808A0FFF7CBF9D7E0774BD8
:103D200009E02046D5F808A0FFF7D0F9CFE0AB684E
:103D30000122DCE0724B1A78D5E02046D5F808A0C5
:103D4000FFF7CDF9C3E06F4BF5E7AB680322CEE098
:103D50006D4BD5F808A01868FDF7F6F9B7E06A4B87
:103D6000D5F808A01868FDF7C7F9B0E0664BD5F89C
:103D700008A01868FDF7F8F9A9E0634BD5F808A08A
:103D80001868FDF7F1F9A1E0604B1B6893F88020FB
:103D9000A9E0227AA7E05D4B1B681B7A012B0DD1AD
:103DA0002046FFF7C9F9E289A38992B29BB2D31AE0
:103DB00023EAE37318B9C3F38F0301E0E3899BB2ED
:103DC000AA6817E0514B1B681B7A012B0DD12046C6
:103DD000FFF7B2F9E289A38992B29BB2D31A23EA20
:103DE000E37318B9C3F38F0301E0E3899BB2AA68B8
:103DF00043F3072393557BE0AB68227C77E02046B2
:103E0000D5F808A0FFF798F9A38A2EE02046D5F848
:103E100008A0FFF791F9A38A0CE02046D5F808A086
:103E2000FFF78AF9E38A20E02046D5F808A0FFF7DB
:103E300083F9E38A38BB43F3852317E02046D5F89E
:103E400008A0FFF779F9B4F86C300EE02046D5F8F9
:103E500008A0FFF771F9B4F86C3013E02046D5F8EC
:103E600008A0FFF769F9B4F86A3008B1DBB20FE0D7
:103E7000C3F387030CE02046D5F808A0FFF75CF9F0
:103E8000B4F86A3010B1C3F3072301E0C3F385230C
:103E90000AF806302CE0A7F16C0323F0010320336D
:103EA000234420465988D5F808A009B2FFF780FDC1
:103EB0000DE0A7F16C0323F00103203323442046D7
:103EC0005988D5F808A009B2FFF772FD00120AF868
:103ED00006000DE0E31913F82D2C04E0A7F1AE0263
:103EE000521023689A5CAB6801E0AB6800229A55D7
:103EF0000137FFB2CBE5BDE8F88F00BFE491FF1FAB
:103F0000D488FF1FE591FF1FA488FF1FB088FF1F03
:103F10002DE9F04F8B6891F80CB093F800A0D344D2
:103F20000027ABF1020B85B00546894616465FFABD
:103F30008BFB97811774B846FAB202EB0A03DBB227
:103F400001325B45D2B200F21981D9F80810812BF9
:103F50008C5C00F0E9802DD8432B7ED015D8052B42
:103F600000F00A8109D8032B58D0042B40F00081BF
:103F700028462146FFF792F8FEE0142B62D0172B5B
:103F800068D0102B40F0F48054E0592B00F0A08052
:103F900007D8452B00F0878075D3572B00F0B680EB
:103FA000E6E05B2B00F09F80C0F09B80802B00F050
:103FB000B480DDE0892B00F0C98013D8852B00F098
:103FC000BC8007D8832B00F0B28000F2B38085F864
:103FD0005540D1E0872B00F0B38000F2B48085F823
:103FE0005940C9E0B22B00F0BA800BD8AE2B00F0DC
:103FF000B080B02B00F0B0808A2B40F0B98085F8FB
:104000005D40B9E0B62B00F0AD80B82B00F0AD807C
:10401000B42B40F0AD802B68DC70ADE02846214623
:10402000FFF79EF8002840F0A38028462146FFF7BE
:1040300092F8A1E0022C00F29B8028462146FFF76F
:1040400033F899E028460CB9214600E00021FFF73B
:10405000A8F891E085F884408EE02846FFF7B8FB89
:10406000484B494C1868FFF7B3FB4FF47A6002F0F5
:10407000CDFC206803689B6A9847206803681B6A28
:10408000984720684CE02846FEF7FFFF04F00F0237
:10409000241102EB021204EB0413009000212846C5
:1040A000D2B2DBB211E02846FEF7E9FF024628460D
:1040B000039204F00F04FEF7E5FF04EB0414E4B2EE
:1040C000039A0094034600212846FEF798FF53E028
:1040D0002E4B186814B9FDF723F84DE0FDF70EF8E4
:1040E0004AE0A04648E008EB042421B242F20F73F4
:1040F000994204DC254B1868FDF734FA03E0337C61
:1041000043F0080333744FF0000835E01D4B21469F
:104110001868FFF787FB78B32AE06CB31A4B18686E
:1041200003685B6A984727E085F8544024E085F8E7
:10413000564021E085F857401EE085F858401BE0C6
:1041400085F85A4018E085F85B4015E085F85C403A
:1041500012E02B681C700FE02B685C700CE02B6881
:104160009C7009E02B681C7106E02B685C7103E011
:10417000337C43F0080333740137DDE605B0BDE856
:10418000F08F00BFB088FF1FB888FF1FA488FF1FF3
:1041900038B5456A084B036004462DB12846FEF742
:1041A0007BFE284604F0C1FC201DFDF75BFA034BA3
:1041B0002360204638BD00BFE8C60000B8AD00004F
:1041C00010B50446FFF7E4FF204604F0AEFC20469D
:1041D00010BDFFFF10B5002281800446034B084646
:1041E000012101F0A7F8A06010BD00BF46AE00009D
:1041F0002DE9F04106461B4B46F8043B0446904629
:10420000002530460F46FDF705FA3046414684F852
:10421000285084F83D5084F8515084F86550257634
:10422000FDF716FA04F12C006761FA21FFF7D2FFBF
:1042300004F14000FA21FFF7CDFF04F15400FA2108
:10424000FFF7C8FF182004F06EFC0F21022206467B
:10425000FEF792FD0123666284F8285023762046FB
:10426000BDE8F081E8C6000038B50446406903683F
:104270009B689847E8B1251D2846FDF76BFA6069F1
:1042800003689B68984718B12846FDF738FA38B19B
:1042900094F828301BB1074B1B68236238BD38BD2A
:1042A00060690368DB689847C1B22846FDF7E4F906
:1042B000E5E738BDCC89FF1F82B030B585B00C462C
:1042C00008A981E80C006B4643F8040B07C983E892
:1042D0000700064B9DF82C2018682146042300F0A7
:1042E000BDFF05B0BDE8304002B07047B888FF1F81
:1042F00010B586B000240193059B00938DF80D4006
:104300008DF80C2003AB0CCBFFF7D6FF06B010BD29
:1043100070B588B06B4600208DF8150043F8040B8B
:1043200008AE0D46144616E9070083E80700044B63
:10433000294618682246042300F090FF08B070BD9B
:10434000B888FF1F10B50446406AFEF73BFD002306
:1043500084F8283010BD38B54C780B7B02341C44EF
:104360000B780A2B0D46E4B201D18B7802E0142BB6
:1043700003D10B7C1C44E4B202E00E2000F0A2FF4B
:10438000A889002319B202B2914205DAAA68D25C68
:104390001444E4B20133F5E7E043C0B238BDF8B5E8
:1043A0000B7C03F07F030B740C460546FFF7D3FF2D
:1043B000E08168690368FF211B68984768690368A2
:1043C000FF211B6898476869617803681B689847F4
:1043D0006869217B036802311B68C9B29847686924
:1043E000217C03681B689847277B0026BB1BDBB238
:1043F0006869A1680F2B03680CD83A0901EB021118
:104400005B6807F00F0298476869A17B03681B6827
:104410009847F8BD31445B68102298471036E5E7AD
:1044200070B5142380F840308B780022013B04469D
:104430000D4680F85020052B27D8DFE803F003094C
:104440001426261F6B7880F84130A0F84C201CE021
:104450006B7880F841301F4B2946186804F1400200
:10446000FFF7FEFA11E06B7880F84130194B2946CE
:10447000186804F14002FFF74BFD06E0154E306866
:10448000FFF772F93068FFF7C5F994F84130FE2B59
:104490001FD06B7CEBB90F4E3068FEF702FE02288E
:1044A00009D03068FEF7FDFD0128AB7801D1022B61
:1044B00001D0012B0DD104F1400529462046FFF71C
:1044C0004AFF2946A4F84E002046BDE87040FFF799
:1044D00066BF70BDB088FF1F2DE9F04F8B6885B0B7
:1044E0001A7893F801A0039280460E460224B6F98A
:1044F0000C309C425FDA314FB36838681D5DFEF7BF
:1045000027FE854204D038682946FEF729FE30B3DD
:10451000B368039A1A55DFF8A890B368D9F8000079
:104520000AF1010B23445FFA8BFB02688DE808084F
:1045300008F15407D2F81CC0394603222B46E04745
:104540001E4B18680293FEF703FE8542029B0BD1B7
:10455000012388F8653040463946FFF761FF0AF1CC
:1045600001031C44E4B2C2E718682946FEF7F8FDCF
:10457000E8B1D9F8000003682946DB6A984780B1A2
:10458000B368D9F80000234402688DE8080839466A
:10459000D2F81CC02B463322E04740463946002261
:1045A00002E0404639460122FFF7B2FED7E712206B
:1045B00000F088FED3E705B0BDE8F08FB088FF1F9C
:1045C000B888FF1FF8B50446606AFEF7F9FB0028BB
:1045D00004DC2046BDE8F840FFF7B4BE606A174F20
:1045E000FEF7E7FB457806463868FEF7B1FD8542E1
:1045F0003146204602D1FFF713FF03E002220123D8
:10460000FFF776FE606AFEF7D9FB0D4B38681B6832
:104610002362FEF79DFD85420ED1606AFEF7D0FB56
:10462000002806DD606AFEF7C4FB837CAB42CBD07A
:10463000F8BD637FAB42CCD0F8BD00BFB088FF1F90
:10464000CC89FF1F38B5012380F82830084B057F3F
:104650001B6803620446406AFEF7ABFB4378AB423B
:1046600004D12046BDE83840FFF7ACBF38BD00BFDD
:10467000CC89FF1F2DE9F0438B689B780377B1F954
:104680000C208B68134485B013F8023C4377054631
:104690000C4601264FF0FF08B4F90C309E423ADA7E
:1046A000771CDFF88490A368D9F80000D95DFEF785
:1046B00057FD38B9D9F80000FEF74AFDA368DB5D65
:1046C000834222D1686AFEF77FFB10B11A2000F006
:1046D000F9FDA3689A1905F1540992788DF80C2018
:1046E0009A5D8DF80D200F4ADB5D106803AA016802
:1046F000009202220192D1F81CC04946E04785F899
:104700006680686A4946FEF73DFBA368033613F8E6
:104710000780F6B2C0E72846FFF794FF05B0BDE872
:10472000F08300BFB888FF1FB088FF1F2DE9F84352
:10473000037E0446002B00F0D88090F828302BB17F
:104740006B4B1A68036AD31A642B19D82046FFF7FB
:104750008BFD251D2846FCF7ABFF05280EDD2846FE
:104760000021FCF7B1FFFF2840F0BA802846012164
:10477000FCF7AAFFFF2840F0B38004E0BDE8F8830F
:10478000FFF7E0FDE2E702212846FCF79DFF00234A
:1047900084F82D0084F83D3028460321FCF794FF6F
:1047A00003B2012B074607DD2846FCF781FFFB1CFF
:1047B000834203DBBDE8F883BDE8F88394F8283032
:1047C0004BB1142384F82C3028460421FCF77CFFDD
:1047D00084F83C0008E00A2384F82C3028460421A1
:1047E000FCF772FF84F82E00B4F93030A7F102080C
:1047F0009845A8BF9846A4F8388008F105085FFAE4
:1048000088F80026711DCBB2434509D2284609B26B
:10481000D4F83490FCF758FF09F806000136F1E7A8
:1048200041462846FCF750FF04F12C0660873146CC
:104830002046FFF790FD638F834251D194F82830D2
:1048400083B1606AFEF7BCFA00283DDD606AFEF7BE
:10485000B0FA94F82D30827C9A4235D12046FFF789
:10486000B1FE39E0DFF88C8094F82D90D8F8000084
:10487000FEF76EFC814522D0D8F8000094F82D1088
:10488000FEF76EFC024630B1012220463146134647
:10489000FFF72EFD20E094F82D30FE2B1CD194F86C
:1048A0002E30832B2046314602D1FFF715FE13E050
:1048B000922B02D1FFF7DEFE0EE0FFF729FD204626
:1048C0003146FFF7ADFD07E0627F94F82D309A4244
:1048D00002D12046FFF736FD391D284609B201E016
:1048E00028460121FCF71CFF33E7BDE8F88300BF31
:1048F000CC89FF1FB088FF1F30B585B004AD05E936
:104900000E00089D9DF804300446002D31D0012B87
:1049100005D1294605B0BDE83040FFF740BD022B68
:1049200021D190F82830A3B12946FFF738FD124B6A
:10493000606A1B682362FEF743FA002809DD606A9B
:10494000FEF737FA6B78827C9A4202D12046FFF755
:1049500039FE6A78637F9A420BD1204605B0BDE8E4
:104960003040FFF7EFBC132005B0BDE8304000F049
:10497000A9BC05B030BD00BFCC89FF1F00487047FF
:10498000F8C600000020704738B5056D074B03607E
:1049900004462DB12846FCF765FE284604F0C5F80C
:1049A000204600F02BFC204638BD00BF20C8000088
:1049B00010B50446FFF7E8FF204604F0B6F820469D
:1049C00010BD2DE9F04186B004688DF8142098469A
:1049D000022205AB8E4600F13C07009301920126AE
:1049E000734639468DF81560E4690546A0476C4664
:1049F0000CAB44F8048B93E80700042384E8070019
:104A000028463946324600F029FC06B0BDE8F08160
:104A1000F0B587B000F13C058DF8153005AB8DF889
:104A2000142002680093022301930F46D669294699
:104A30003B4603220446B0476B460C9A43F8042BCE
:104A40000DAA07CA83E80700204629469DF84020A2
:104A50009DF8443000F002FC07B0F0BDF0B587B01F
:104A600004688DF814201F46022205AB8E4600F123
:104A70003C060093019273468DF815203146E46997
:104A80000546A0476C460CAB44F8047B93E807004E
:104A9000042384E8070028463146012200F0DEFBAB
:104AA00007B0F0BDF0B587B006688DF815301B1261
:104AB0008DF814208DF81630032205AB00F13C056B
:104AC000009301920F463B462946F6690446B047DB
:104AD0006B460C9A43F8042B0DAA07CA83E807001B
:104AE000204629469DF840209DF8443000F0B6FB52
:104AF00007B0F0BDF0B589B004AA05238DF81030D9
:104B0000036800920222002400F13C060192DF6952
:104B10008DF8154031468DF811400322FE230546DD
:104B2000B8476B4608AF43F8044B17E9070083E822
:104B30000700284631462246234600F08FFB09B085
:104B4000F0BDFFFFF0B5174C89B005462068FEF7B1
:104B500052FF2068FEF74AFF00232A6800930124D1
:104B6000019305F13C068DF815308DF81630D769A4
:104B70008DF814402846314622462346B8476B46F6
:104B80008DF8174043F8045B08AF17E9070083E886
:104B90000700284631462246032300F05FFB09B098
:104BA000F0BD00BFB088FF1F104B10B50446186859
:104BB000FEF7E5FAC0B200EB4003A26D5B00D1182E
:104BC000D35A23F00202B2F5CA7F03D0A3F5CC7307
:104BD000012B05D88878162894BF0020012010BD2D
:104BE0001F2000F06FFB002010BD00BFB088FF1F2A
:104BF000F8B5044617460E46002500F01DFB164B7F
:104C00002360666584F8255084F8395084F84D5047
:104C1000102003F088FF0646FCF7FCFC30463946BE
:104C20002665FCF715FD01220C4B06210A2000F039
:104C300081FBFA21A06504F11400FFF7CBFA04F11F
:104C40002800FA21FFF7C6FA04F13C00FA21FFF729
:104C5000C1FA25712046F8BD20C800000EC700002B
:104C6000F0B5002189B004463C22806D05F079F84A
:104C7000164B1B6893F8543033B314228DF811206F
:104C800004AA21680092022200250192042604F160
:104C90003C078DF815508DF81050D1F81CC08DF8D8
:104CA000146020463946E0478DF816506D4608AB33
:104CB00045F8044B13E90700334685E80700204612
:104CC0003946012200F0CAFA09B0F0BDB088FF1FD2
:104CD0002DE9F0478AB005AD85E80E009DF8147007
:104CE000129A9DF816609DF81780012F044634D162
:104CF0006AB1092E03D92046FFF7B2FF81E042498D
:104D000052780968731C0E4486F85420DEB2B8F15C
:104D1000FC0FF0D8092EEED82268002308F1010814
:104D2000009301935FFA88F804F13C07D2F81CC0A5
:104D30002046394601224346E0476B468DF816600F
:104D40008DF8178043F8044B95E8070083E80700C7
:104D500020463946012203234DE0042F4ED1002A7C
:104D60004FD09368D0F858C093F801A093F8009002
:104D700006EB4601490009EB0A292CF801900CEBDF
:104D800001089B7888F80230936893F804C0836D1B
:104D90000B44013683F803C0836D194493681B7D6F
:104DA000F6B2003318BF0123092E0B7129D8164B18
:104DB0001B68334493F854301BB300228DF8242031
:104DC00014228DF8252009AA01680092022200F120
:104DD0003C080192D1F81CC04146E0478DF81660AE
:104DE0006E463B4646F8044B95E8070086E8070008
:104DF00020464146012200F031FA02E0042000F092
:104E000061FA0AB0BDE8F087B088FF1F38B54C786A
:104E10000B7B02341C440B780A2B0D46E4B201D103
:104E20008B7802E0142B03D10B7C1C44E4B202E02B
:104E30000B2000F047FAA889002319B202B2914270
:104E400005DAAA68D25C1444E4B20133F5E7E04322
:104E5000C0B238BD2DE9F84FB1F804808D680A9EC4
:104E60000FFA88F70C46924600213A4681462846BA
:104E70009B4604F076FF14222046002104F071FFC7
:104E80009DF82C20A4F804800A23BA42A8BF3A4611
:104E9000A560237084F801B084F802A0A2811EB13D
:104EA0002846314604F039FF48462146FFF7AEFF59
:104EB000E081BDE8F88F2DE9F0410446006DFCF774
:104EC000F7FB012827DD206D0021FCF7FDFBFF2803
:104ED00005D1206D0121FCF7F7FBFF2804D0206DE0
:104EE0000121FCF71DFC16E0206DFCF7E1FB052815
:104EF00011DD0221206DFCF7E7FB03210546206D43
:104F0000FCF7E2FB0128064605D9206DFCF7D0FB33
:104F1000F31C834201DB002533E014236575237500
:104F2000206D0421FCF7D0FBB4F9183084F824007C
:104F3000B71E9F42A8BF1F4627840537FFB2002532
:104F4000691DCBB2BB4209D2206DD4F81C8009B2D6
:104F5000FCF7BAFB08F805000135F1E73946206D8A
:104F6000FCF7B2FB04F1140507466084294620468D
:104F7000FFF74CFF8742B2D1311D206D09B2FCF71B
:104F8000CFFB2846BDE8F08138B50546406D0A23C1
:104F90000B7003680C461B68FF219847686D036817
:104FA000FF211B689847686D617803681B68984704
:104FB000686D217B036802311B68C9B29847686D30
:104FC000A17803681B689847686DA1680368B4F905
:104FD0000C205B689847686DA17B03681B68984745
:104FE00038BD8B6888891B78934207D318440238F0
:104FF000C0B290428CBF0020012070470020704753
:1050000010B58868B1F90C100478C4F10104224489
:10501000D2B28A4204DB2020BDE8104000F052B931
:10502000835410BD2DE9F3470446606D03689B6807
:10503000984758B1606D0368DB689847C1B2206D2E
:10504000FCF71AFB6B4B1B68A360EEE72379002B80
:105050007ED1E068FDF7CAFF002840F3C880E06811
:10506000654EFDF77CFF054630686979FEF787F8E5
:10507000AB79032BB24605F1040601D0332B4AD19C
:10508000B5F91030012B46DD5FFA80F83146204635
:105090000322FFF7A6FF40B3EB681A78134413F816
:1050A000027C6B79FE2B05D1E06802B0BDE8F047C9
:1050B000FDF790BFDAF80000DFF83C913946FEF7C3
:1050C0004FF838B9D9F80000FEF742F8874201D00E
:1050D000002F78D12046314603226B79FFF790FFED
:1050E00020463146FFF792FE688220463146042270
:1050F000FFF777FF78B1A36D08EB480803EB48038F
:10510000204631460422DB78FFF77AFF20463146FD
:10511000FFF77CFE6882206DFCF7FEFA00236B76B9
:1051200020463146FFF730FF6B79FE2B06D1022077
:1051300001F06CFC20463146FFF726FF95F824303D
:10514000237113B9E068FDF745FF2A4B1B681DE08A
:10515000012B32D1E068274FFDF701FF05462046BD
:10516000FFF7A9FE3A68A368064688B995F82510A6
:10517000D31A8B423BD9AB79012B2AD16A7E42BB31
:105180006B762046291DFFF7FFFE3B68A3602EE0EB
:10519000194F71783868FDF7F2FF002806DB3B688D
:1051A0001844337C23F05A0380F85E30AB79922B9D
:1051B0000FD1242000F086F80BE00C2002B0BDE8EF
:1051C000F04700F07FB8D9F80030434483F85470BA
:1051D0008BE7286830B10368009618351E6895E89B
:1051E0000E00B047E068FDF7F5FE0023237102B022
:1051F000BDE8F087CC89FF1FB088FF1F38B5C568B0
:10520000064B036004462DB12846FDF745FE2846AF
:1052100003F08BFC024B2360204638BD60C80000C1
:10522000B8AD000010B50446FFF7E8FF204603F0D4
:105230007CFC204610BDFFFF38B5074B03600446D9
:10524000182003F070FC0F210546FA22FDF7BEFD81
:10525000E560204638BD00BF60C80000F0B505AC71
:105260001646059A44F8042B05460F46E868394669
:105270003246BDE8F040FDF71EBEFFFFFB280CD014
:10528000FC2803D0FA2803D1054870470548704729
:10529000054B0130B3FBF0F070470448704700BF86
:1052A00010552200C0C62D0080841E00A0252600B7
:1052B00038B5044603F0B7FC0546204603F058FC19
:1052C000284438BD37B505462C46002C26DD012D77
:1052D00008DD154B186828B1002300930121FF2237
:1052E000FDF78DFE114B20221A604FF47A7001F009
:1052F0008DFB012D08DD0C4B186828B100220092AF
:1053000001211346FDF77BFE094B20221A604FF462
:105310007A70013C01F07AFB24B2D6E74FF47A6050
:1053200001F074FBD0E700BFB088FF1F84F00F408E
:1053300088F00F4070B51E4600FB01F412B104F076
:105340008DFC02E0204604F0C9FC0C490B6803B94F
:1053500008600B4D0B682A880860C31A13442B8021
:10536000084D2B881C442C8038B907480749324621
:1053700003F014FC1420FFF7A5FF70BDD888FF1FB1
:10538000DC88FF1FD688FF1FC891FF1F98C8000048
:10539000054B1A6840F6B7339A42014602D90348D2
:1053A00003F0C5BB704700BFCC89FF1FC891FF1F2A
:1053B00008B5084B1A6840F6B7339A42014607D938
:1053C000054803F0B4FB0448BDE8084003F0D0BB37
:1053D00008BD00BFCC89FF1FC891FF1F08B5054B52
:1053E0001A6840F6B7339A42014602D90248FFF7DD
:1053F0005FFF08BDCC89FF1FC891FF1F072910B5AB
:105400000C460BD872B600F0D3FE62B60123A3405F
:105410001840C0B240FA04F4E0B210BD002010BD44
:1054200008B572B600F0C4FE62B608BD08B572B623
:1054300000F0D2FE62B600B208BDFFFF2DE9FF41C9
:10544000244DB5F90030642B07460C4690462E4695
:105450000EDD2149684603F04DFC6846FFF798FFD2
:10546000684603F007FCB5F90000FFF7B7FF2DE031
:10547000072921D800F0C4FE0028FBD072B63846B8
:1054800000F096FE62B6012303FA04F418F0010F4F
:105490000CBF20EA04040443E4B200F0B1FE00288B
:1054A000FBD072B63846214600F0B2FE62B63388B1
:1054B0000133338001200AE00849684603F01AFCF2
:1054C0006846FFF775FF684603F0D4FB002004B080
:1054D000BDE8F081DE88FF1FF8CB00004DCC000056
:1054E00070B50C4CB4F90030642B05460E460EDC4A
:1054F00000F086FE0028FBD072B62846314600F048
:1055000087FE62B6238801332380012070BD00200E
:1055100070BD00BFDE88FF1F70B50C4CB4F90030C1
:10552000642B05460E460EDC00F06AFE0028FBD018
:1055300072B62846B1B200F085FE62B62388023307
:105540002380012070BD002070BD00BFDE88FF1FDA
:1055500010B5044659B101210B20FFF7C1FF00210E
:105560000C20FFF7BDFF0D200221FFF7B9FF631EDE
:10557000DBB2FC2B05D821460E20BDE81040FFF71A
:10558000AFBF10BD08B500210220FFF7C5FF002105
:105590001720FFF7C1FF002101221720FFF74EFF60
:1055A00001210A461720FFF749FF01220221172097
:1055B000FFF744FF4FF4AF511A20FFF7ADFF03216F
:1055C0000F20FFF78DFF10200146FFF789FF012113
:1055D0001320FFF785FF01211420FFF781FF03212E
:1055E0001520FFF77DFF03211620FFF779FF01202B
:1055F0000146BDE80840FFF7ABBFFFFF10B572B62C
:10560000094B0A4C01221A702078022101F0CCF8D3
:10561000074A084900231370074A137020780222B2
:1056200000F0BCFF62B610BD1589FF1FFA88FF1F8E
:105630001189FF1FAD560000E488FF1F054B1A7843
:1056400010B51C4612B1044803F05CFA0023237025
:1056500010BD00BFF988FF1FFC88FF1F10B504466E
:1056600003F050FA204610BD0B4B1A7810B51C46BB
:105670000AB1FFF7E3FF094B094A1B68591E914223
:1056800006D830225A4307480749013A03F024FA62
:105690000123237010BD00BFF988FF1FE088FF1FA2
:1056A00057555505FC88FF1F0557000008B50F4BDF
:1056B00019781A46802309B10D4900E00D490B60A5
:1056C000127880230AB90A4A00E00A4A136072B6C7
:1056D000094B187800F0A8FF084B02221A70084BFB
:1056E00003221A70FFF7C0FF62B608BD1489FF1FBE
:1056F00084F00F4088F00F40FA88FF1F1589FF1FC4
:105700001089FF1F3F4B1A78012A70B5194673D0D4
:105710003D4D2B78013BDBB22B70002B70D13B4B06
:105720001878802208B13A4800E03A4802601A78B6
:10573000344C82F001021A700978C9B202292FD1C3
:10574000354B1A78354B53F83230354A93F80062AE
:105750001378072BF6B2334B15D9334A11781878E2
:10576000324BC9B2C0B2585411781423013191FBA5
:10577000F3F003FB1013DBB21370FFF73FFF0423BA
:105780002370012331E01078C0B2441CE4B21470DD
:105790001A7806FA00F01043C0B21870297070BD74
:1057A0002378032B23D11E4B1A78072A04D9FFF73D
:1057B00025FF0423237017E0174A18481478194A64
:1057C000E4B2117850F8340011F0010F4FF00101EC
:1057D00014BF80F8801080F800111178490811700A
:1057E0001A780132D2B21A7002232B7070BD23785E
:1057F000042B05D101232370BDE87040FFF71EBFC5
:1058000070BD00BF1589FF1F1089FF1F1489FF1F7E
:1058100084F00F4088F00F40FA88FF1FF0CC0000A2
:10582000E488FF1F1189FF1F1289FF1FE588FF1FF2
:1058300038B5104B1B7805460C4613B10320FFF713
:1058400041FD0C20012100F0AFFF0B4B80221A60BC
:1058500072B60A4A00231370094A1370094B1D706F
:10586000094BB3FBF4F4094B1C60FFF7C7FE62B6AB
:1058700038BD00BF1589FF1F88F00F401389FF1F37
:105880001289FF1FFA88FF1F20A10700E088FF1F71
:105890000B4B1A7810B58AB11A78012AFCD172B66E
:1058A000084CFFF7CBFE207800F0BEFE20780221E6
:1058B00000F07AFF024B00221A7062B610BD00BFE2
:1058C0001589FF1FFA88FF1F72B6054B1878054B24
:1058D0001B78C0B2DBB262B6C01A18BF0120704795
:1058E0001389FF1F1289FF1F10B5FFF7EDFF80B16D
:1058F00072B6084B08491A78D2B2885C197814221B
:10590000013191FBF2F402FB1412D2B2C0B21A7050
:1059100062B610BD1389FF1FE588FF1FF8B5074663
:10592000104E3578EDB2012DFAD172B60E4C2078BA
:1059300000F07AFE032333700C4B1F700C4B0022D7
:105940001A702078294600F02FFF2278094B53F86F
:10595000323083F80051084B02221A70FFF784FEA0
:1059600062B6F8BD1589FF1FFA88FF1F1189FF1F56
:10597000E488FF1FF0CC00001089FF1F0448054990
:10598000054A002303708023437304F059B900BF14
:10599000FC88FF1F5D5600006087FF1F084B1A68D8
:1059A00042F480721A604FF4A072013A7FF4FDAFA6
:1059B0001A689205FCD42023013B7FF4FDAF7047A9
:1059C000005004402DE9F74F6B4E6C4B3268517C10
:1059D000927C5C5C9D5CFF2C814601D0FF2D02D146
:1059E0001120FFF76FFC3168654A4B7C654F02EB75
:1059F000C303586800230360897C634802EBC1023B
:105A0000624952681360624B620013440B60604B42
:105A10006A0013443B605F4B1A6842F020021A6030
:105A200001235D4A03FA05F503FA04F445EA040389
:105A300013605A4B1A6822F080021A60584A1060AC
:105A4000584818608846B9F1000F7CD0142000F047
:105A5000DDFFFFF7A3FFD8F8003053491B889BB246
:105A6000ADF80030BDF80030BDF800204F4B92B2C9
:105A70000A601A603A684E49128892B2ADF8022064
:105A8000BDF80220BDF8022092B20A6049494FF0E9
:105A90000A0A0A609946FFF781FFD8F80030424DA4
:105AA0001B88D9F800203868414C9BB2ADF804300F
:105AB000BDF80430BDF804103F4B89B219602B6863
:105AC0004FF0060B42F20F7E0BFB02120EFB03138C
:105AD00042F21071B3FBF1F32B6003889BB24FF0DD
:105AE000070CADF80630B2FBFCF2BDF80630BDF88D
:105AF0000600C9F800202268304B80B20BFB02027E
:105B0000DFF8B0B01860DBF800300EFB0303B2FB27
:105B1000FCF2B3FBF1F105200AF1FF3A2260CBF869
:105B2000001000F073FF1AF0FF0AB4D11F4A336867
:105B300011682A688A1A92B29A822168DBF80020DA
:105B40008A1A92B2DA82154B15491A6822F080023D
:105B50001A600A6842F420620A601A6842F0D202AF
:105B60001A60174B80221A70A3F24B334FF40022B5
:105B70001A6003B0BDE8F08FB088FF1FA4CC00000E
:105B8000F0CC00003489FF1F000003033089FF1FA1
:105B90000051044038800440085004400050044044
:105BA0000450044080004D003889FF1F2C89FF1FDE
:105BB0002489FF1F1889FF1F2889FF1F2089FF1FC5
:105BC00053E400E02D4BF7B51A6812F4805F1A68B1
:105BD0000AD042F480521A60294B1A880020013200
:105BE0001A80FFF7EFFE47E042F400421A60254BAF
:105BF0001B681B889BB2ADF80430BDF80430BDF8BB
:105C00000420214B92B21A60204B1C684FF0060C06
:105C100007270CFB0424B4FBF7F41C601C4B196829
:105C200042F20F7606FB012242F21075B2FBF5F24A
:105C30001A60184B18491B681B889BB2ADF80630D8
:105C4000BDF80630BDF806309BB20B6013490868FA
:105C50000CFB0030B0FBF7F0086011490F6806FB41
:105C60000733B3FBF5F30B600E49A21A0968C31A98
:105C700092B29BB28A82CB8203B0F0BD0050044046
:105C80001C89FF1F3089FF1F2889FF1F2C89FF1FD8
:105C90003889FF1F3489FF1F2089FF1F2489FF1FB8
:105CA0001889FF1FB088FF1F024B4FF400221A60B3
:105CB000704700BF88E100E0F0B5304B1B681B0661
:105CC000FBD42F4B1B6813F08002F6D172B62D4B1C
:105CD0001978002950D02C4908684F688E68CD6823
:105CE0000C6938441431304409682844204408447D
:105CF000C0F34E00254940F400400860C86A0F6BAD
:105D00004E6B8D6BCC6B384440313044096828446D
:105D100020440844C0F34E001D4940F40040086090
:105D200001F10811143151F8140C51F8107C51F89C
:105D30000C6C51F8085C51F8044C09683844304444
:105D4000284420440844C0F34E00124940F4004067
:105D50000860C86A0F6B4E6B8D6BCC6B384440315A
:105D600030440968284420440844C0F34E000A49DE
:105D700040F4004008601A7062B6F0BD24B00340E1
:105D800024B00B403D89FF1F38B003402CB00340C6
:105D900030B003402CB00B4030B00B4010B5204B5E
:105DA0002048214960221A70E1225A701F4B204A74
:105DB0001C78204B082C01D1012402E00A2C03D1CD
:105DC00039240460132005E00C2C0CBF35243D243D
:105DD00004601220086014601860174B17491B7884
:105DE000174A03B101230B601360164B164A19784A
:105DF000164B012901D880210BE0042901D8842108
:105E000007E0082901D8852103E0102994BF8621E5
:105E10008721116019600E4B01221A7010BD00BF5E
:105E20000040074008B003400CB003406587FF1FE7
:105E300008B00B400CB00B404089FF1F20B003405E
:105E400020B00B406687FF1F24B0034024B00B40F6
:105E50003D89FF1F0C2804D9102828BF10201023CB
:105E600007E00A2804D8092834BF08230A2300E0E1
:105E70000C23094AD9B2081A1070084A10788342D4
:105E800008D0074B11701B7813B1064B00221A6023
:105E9000FFF784BF704700BF3C89FF1F6587FF1F66
:105EA0003D89FF1F24B0034010B5114B1B780446F9
:105EB0000BB1FFF701FF012C0E4A01D8002302E0CD
:105EC000042C02D8042313600EE0082C03D8052309
:105ED0001360082308E0102C03D806231360102356
:105EE00002E0072313602023034A137010BD00BF94
:105EF0003D89FF1F24B003406687FF1F0D2838B57A
:105F00000FD9172801D80E380AE0A0F11A03052B83
:105F100001D8093804E0A0F12203062B47D818382D
:105F2000C0B2244B1C5C244B1B780BB1FFF7C4FEA2
:105F3000210614D472B6214B214D1C6001232B7015
:105F400062B672B61D4B1B681A0601D51D4B1FE0C9
:105F50002B78002BEFD062B602F0F8FEF1E772B6B4
:105F6000194B1A4D1A6814F0400F14BF22F010029A
:105F700042F010021A60164B04F03F021A6001232F
:105F80002B7062B672B6124B1B681B0608D5114BFC
:105F9000186800232B7062B60F4B1B78184138BD70
:105FA0002B78002BDCD062B602F0D0FEEAE70020AE
:105FB00038BD00BFC6CC00003D89FF1F00B00340C4
:105FC0003F89FF1F10B003400CB00B403E89FF1FFC
:105FD00000B00B4010B00B403C89FF1F0D2810B5DE
:105FE0000FD9172801D80E380AE0A0F11A03052BA3
:105FF00001D8093804E0A0F12203062B27D818386D
:10600000C0B2134B1C5C134B1B780BB1FFF754FE53
:10601000230607D472B6104B44F040041C600122E2
:106020000E4B12E072B60E4B1A6814F0400F14BFFC
:1060300022F0100242F010021A6004F03F04094BF3
:1060400044F040041C60084B01221A7062B610BD77
:10605000C6CC00003D89FF1F00B003403F89FF1FF1
:106060000CB00B4000B00B403E89FF1F0D280FD92C
:10607000172801D80E380AE0A0F11A03052B01D821
:10608000093804E0A0F12203062B26D81838C0B244
:10609000134B1B56002B08DB124B1B6813F0800FB1
:1060A000114B12D072B6114A07E0114B1B6813F066
:1060B000800F104B09D072B60F4A106800221A7078
:1060C00062B60E4B1B78184170471B78002B14BF2B
:1060D0004FF0FF306FF0010070470020704700BFA5
:1060E000C6CC000000B003403F89FF1F10B0034042
:1060F00000B00B403E89FF1F10B00B403C89FF1FD2
:10610000084B1A6842F480521A60074B1A78074B02
:106110000AB1802200E0C0221A70054B80F30C0007
:10612000188070472C8004404089FF1F21C00C401C
:1061300000C00C40024B1B78DB07FBD5704700BF4B
:10614000010002407FB5174B6A4603F110056E4609
:1061500018685968144603C40833AB422246F7D185
:10616000114B1A7812F0020F1D4612D080229A713C
:1061700033229A7203225A7272B60C4C46F0010610
:106180002046B04762B6237813F0700301D0237025
:1061900006E044F621632A78D20701D4013BFAD104
:1061A00004B070BDDECC00000100024000000240DF
:1061B000B0F5006F10B5044609D2064B1B78DB071B
:1061C00001D4FFF7BFFF04F1A054207810BD0020D8
:1061D00010BD00BF0100024040F2FE73984210B5AE
:1061E000044609D8054B1B78DB0701D4FFF7AAFF4B
:1061F00004F1A054208810BD002010BD0100024011
:10620000024B187800F00100704700BF0100024007
:10621000B0F5006F38B504460D460FD2084B1B7819
:10622000DB0701D4FFF78EFF04F1A0542378AB42C3
:1062300004D02570BDE83840FFF77CBF38BD00BFF3
:106240000100024038B540F2FE73984204460D4604
:106250001ED8104B1B78DB0701D4FFF773FF14F037
:10626000010F04F1A05404D12388AB4210D0258043
:106270000AE02378AB4202D02570FFF75BFF63781A
:106280002D0AAB4204D06570BDE83840FFF752BF1D
:1062900038BD00BF01000240024B1A6801321A608B
:1062A000704700BFCC89FF1F08B50B4C236858030B
:1062B00001D501F035FD2368590501D500F060FED8
:1062C00023681A0501D501F039F92368DB04ECD500
:1062D00001F0A2FBE9E700BF3480044008B5FFF7F6
:1062E000E3FFFFFF014B10221A807047002005409A
:1062F0007047FFFF024A1368184410601846704741
:106300006887FF1F002070474FF0FF3070474FF045
:10631000FF307047FEE7FFFFEFF313839BB9EFF306
:10632000108098B9EFF3058323B10F2B04D9084AE5
:10633000985C01E04FF48070EFF311833BB183422E
:1063400038BF184670474FF0FF3070471846704707
:10635000F0E300E01F4B10B51C681C60E00304D59F
:106360001D4B1A680AB11B689847A10304D51A4B44
:106370005A680AB15B689847E20704D5164B1A6C55
:106380000AB11B6C9847A30704D5134B5A6C0AB18A
:106390005B6C9847200704D50F4B9A6C0AB19B6C35
:1063A0009847610704D50C4BDA6C0AB1DB6C98474F
:1063B000220304D5084B5A6E0AB15B6E98476303FB
:1063C00006D5054BD3F8802012B1D3F8803098471A
:1063D00010BD00BFA0A004404489FF1F2C4B10B586
:1063E0001C681C60200704D52A4B5A6A0AB15B6AF4
:1063F0009847E10604D5274B9A6A0AB19B6A9847E9
:10640000620604D5234BDA6A0AB1DB6A9847230691
:1064100004D5204B1A6B0AB11B6B9847A00604D514
:106420001C4B5A6B0AB15B6B9847E10704D5194BBB
:10643000DA6B0AB1DB6B9847A20704D5154B9A6D4E
:106440000AB19B6D9847630704D5124BDA6D0AB108
:10645000DB6D9847A00504D50E4BDA6E0AB1DB6EF2
:106460009847E10504D50B4B1A6F0AB11B6F98478B
:10647000620504D5074B5A6F0AB15B6F9847230535
:1064800004D5044B9A6F0AB19B6F984710BD00BFAB
:10649000A0B004404489FF1F1E4B10B51C681C604F
:1064A000E00704D51C4B9A680AB19B6898472106FF
:1064B00004D5194B5A690AB15B699847E20604D5BD
:1064C000154B9A690AB19B699847630704D5124B2B
:1064D000DA690AB1DB699847200704D50E4B1A6ABE
:1064E0000AB11B6A9847A10704D50B4B9A6B0AB1F6
:1064F0009B6B9847A20604D5074B1A6D0AB11B6D1A
:106500009847630604D5044B5A6D0AB15B6D9847F2
:1065100010BD00BFA0C004404489FF1F114B10B53F
:106520001C681C60E00404D50F4BDA680AB1DB6814
:106530009847A10404D50C4B1A690AB11B69984706
:10654000A20604D5084B1A6E0AB11B6E9847E306E3
:1065500006D5054BD3F8842012B1D3F88430984780
:1065600010BD00BFA09004404489FF1F094B10B527
:106570001C681C60A20704D5074B9A6E0AB19B6E7B
:106580009847E30704D5044BDA6F0AB1DB6F9847ED
:1065900010BD00BFA0D004404489FF1F212830B5A2
:1065A00031D8042A2FD8DFE802F00709050B0300D1
:1065B0000B2306E00A2304E0082302E00C2300E09A
:1065C0000923114A114D02EBC0025468104AC2F867
:1065D0009C51104DC2F8A0510F4DC2F8A4510F4D5F
:1065E000C2F8A8510E4DC2F8AC5172B622680D4DDA
:1065F00022F47022226042F0807242EA034345F89E
:106600002010236062B630BDF0CC00001D65000094
:106610000082FF1F55630000DD63000099640000E5
:106620006D6500004489FF1F094B03EBC0035A68E6
:1066300072B6136823F0877323F4803343F08073BA
:106640001360044B002243F8202062B6704700BF5D
:10665000F0CC00004489FF1F044B054900221A605A
:106660000A60044A106010221A60704714D0034078
:1066700004D0034000D003402DE9F04105460E460A
:1066800008462E4903F06EFA2D4B002847F61228D3
:1066900014BF0227012708BF9846002428FA04F0F7
:1066A00003F06AF84FF05E5103F0BEF80146304641
:1066B00003F06CFA10B90134072CEFD128FA04F07A
:1066C00003F05AF8314603F063F94FF07C5102F0C1
:1066D000A1FF03F095FA4FF6FF73984228BF1846C2
:1066E000EB1E012B06D8174B174900221A600A60CF
:1066F000164A1BE0A5F10903012B06D9A5F11403E5
:10670000032B02D96B1F012B06D8114B1149002214
:106710001A600A60104A09E0202D01D0192D0BD112
:106720000E4B0F4900221A600A600E4A04F007045B
:1067300044EAC70710601F60BDE8F081001BB74046
:10674000006CDC020090034004900340089003407A
:1067500000800340048003400880034000800B4019
:1067600004800B4008800B40212810B518D80D4A32
:1067700052F8303093F880423CB1012211B183F8D5
:10678000802010BD83F8002110BD02EBC0004368DB
:106790001A6811B142F0030201E022F002021A600D
:1067A00010BD00BFF0CC0000212829D8154A02EB0B
:1067B000C00301295B6852F8302004D182F88012AE
:1067C0004FF4A2721BE0002082F8800211B18A1EF1
:1067D000012A12D84FF4807202291A6003D11A6874
:1067E00042F003020BE003290AD11A6842F00202C8
:1067F0001A601A6822F0010201E040F203121A60E6
:10680000704700BFF0CC0000282838B5604A044625
:106810000B4611D112780B2A04D8C2F10C0201FAEE
:1068200002F304E00C2A1CBF0C3A41FA02F31846AA
:10683000BDE83840FFF764BC11780125002B05FA4C
:1068400001F2D8BF002102DD934205D32946FFF7AC
:106850008BFF2046294697E00338C2B2012A01D8AF
:106860004C4A06E0202C01D0192C01D14A4A00E004
:106870004A4A126802FB0332CA401D287BD8DFE86F
:1068800000F0575F4E337A7A212A7A7A7A7A7A7AC6
:106890007A7A7A3C450F187A707A7A7A7A7A7A67B5
:1068A0003F4B1A6003F5973340F2444203F5FA7305
:1068B0005FE03C4B1A6003F5973340F2444203F526
:1068C000F87356E0384B1A6003F5973340F24442B0
:1068D00003F5F6734DE0354B1A6003F5973340F23C
:1068E000444203F5F47344E0314B1A6003F59F33DF
:1068F00040F2444203F5F0733BE02E4B1A6003F57F
:106900009F3340F2444203F5EE7332E02A4B1A60A3
:1069100003F59F3340F2444203F5EC7329E0274B23
:106920001A6003F59F3340F2444203F5EA7320E016
:10693000234B1A6003F580334FF45172203318E073
:10694000204B1A6003F580334FF451721C3310E072
:106950001D4B1A60A3F5DB234FF45172A3F5F963C5
:1069600007E01A4B1A60A3F5DB234FF45172A3F230
:10697000CC731A6038BD7F2B2046D4BF0021012183
:10698000FFF7F2FE20460121BDE83840FFF70CBFBB
:106990006C87FF1F0890034008800B40088003406D
:1069A000108003401880034020800340288003406B
:1069B00030800340388003404080034048800340DB
:1069C000109003401890034010800B4018800B403B
:1069D00072B60B4B0B491A680B4B1B68096862B601
:1069E000490102D5322A88BF0133C2F5BB3260218A
:1069F000FF32B2FBF1F24FF47A7000FB03207047D4
:106A000018E000E004ED00E0CC89FF1F38B5044633
:106A1000FFF7DEFF054624B938BD013C0AD005F575
:106A20007A75FFF7D5FF401BB0F57A7FF5D202F0FB
:106A30008DF9F6E738BDFFFF1F4B4FF4000210B58C
:106A40001A604FF080721A604FF000721A604FF0B7
:106A500080621A604FF000621A60184B184A194C95
:106A600000204BF6FF711860596028231360936073
:106A7000136193611362936213639363092222602B
:106A800004F58054043420606160A360236144F8FD
:106A9000042C04F5FE2420600B4801600B490B60B8
:106AA0008B600B4B1A60FFF779F9FA20FFF7AEFF06
:106AB000BDE8104001F032BC08E100E00480034072
:106AC0000C8003400080034008800B400C800B408A
:106AD00000800B401D4B1A6842F480621A601C4A09
:106AE000002313801B4A13801B4A13701B4A137028
:106AF0001B4A13701B4B40F213321A604FF4517251
:106B00005A60194BC0F344321A70C0F347125A70DE
:106B10000221042200F01F0098729A70D9745A75ED
:106B200088221A743C22DA709A7842F0A0029A7095
:106B30009A7902F0DF029A710C4B40226FF44A718D
:106B40001A700B444FF400521A60704734800440AE
:106B5000588BFF1FD689FF1F608BFF1F5A8BFF1FAB
:106B6000D489FF1F40A0044000A006402DE400E0AF
:106B7000134A937800F0030103F0EC030B43410741
:106B800048BF43F01003937000F00F03042B0C492F
:106B900003D18B7943F040038B715379C20603F024
:106BA000EF03074A48BF43F01003537193798106FE
:106BB00003F0EF0348BF43F010039371704700BF29
:106BC00000A0064008B5114B1B685B0500D408BD4A
:106BD0000F4B1A7802F0FF0312B102F0B7F8F7E793
:106BE0000C4A4FF4005111600B4A0C49D37040F22B
:106BF00003120A604A600A4A13800A4A13800A4B49
:106C00001B680BB101221A7008BD00BF348004401C
:106C1000D489FF1F84E100E000A0064040A00440AA
:106C2000588BFF1FD689FF1FD089FF1F38B5044638
:106C3000094B1B7803F0FF05002BF9D120460121F9
:106C4000FFF7B2FD20462946FFF78EFD034B53F8B0
:106C50003420034B1A6038BDD489FF1FF0CC0000EC
:106C60005C8BFF1F0D4A38B5146814F480624FF036
:106C7000000410D021280A4D0AD80A4A012152F8EE
:106C800030302B60FFF790FD2B681C70012038BD61
:106C90002C60204638BD104638BD00BF348004400B
:106CA000D089FF1FF0CC00000E4B1B6813F48063EB
:106CB00016D012280C4B03D140F202310B4A04E0EB
:106CC000142809D10A4A40F2023111605A7B42F07D
:106CD00001025A73012070475A7B02F0FE025A7378
:106CE000002070473480044000A006400CA00440FF
:106CF00014C00440F8B51F4B1B685A05064638D52A
:106D00001D4B1B680BB101221A701C4B9A7942F083
:106D100020029A711A4B1C780134802C1F4628BF20
:106D20000024184D2B78A34218D1FFF7F5FA40281C
:106D30000FDC124A13791B06F3D52B781249013365
:106D4000802B28BF0023C95CDBB2C9B2D1712B7084
:106D5000E7E7FF28E5DD01F0F9FFE2E70A4BF6B2CD
:106D60001E550A4B01221A70044BE4B2BC223C703F
:106D7000DA70F8BD348004405C8BFF1F00A0064031
:106D8000608BFF1F5A8BFF1FD889FF1FD489FF1FFD
:106D9000294B1B685A052DE9F04707468A4649D515
:106DA000264B1B680BB101221A70254B9A7942F0D1
:106DB00020029A713D4607EB0A039D4237D2DFF865
:106DC0009080204E98F8004096F800900134802C76
:106DD00028BF00245FFA89F9A1451DD1184BBC22B8
:106DE000DA70FFF799FA40280FDC154A13791B0671
:106DF0000FD5337814490133802B28BF0023C95C99
:106E0000DBB2C9B2D171337003E0FF2801DD01F0BC
:106E10009DFF33784B45E4D00B4B15F8012B1A55E9
:106E20000A4B0122E4B21A7088F80040C3E7044B11
:106E3000BC22DA70BDE8F087348004405C8BFF1F11
:106E400000A006405A8BFF1FD889FF1FD489FF1F5F
:106E5000608BFF1F08B5034B1B7813B101F076FF61
:106E6000F9E708BDD489FF1F064A074B1B78107845
:106E7000DBB2C0B283422CBF7F3000F1FF30C01ABA
:106E8000704700BF5A8BFF1F608BFF1F054B188890
:106E9000054B1B8880B29BB2984238BF00F58070CA
:106EA000C01A7047588BFF1FD689FF1F114B12491C
:106EB0001A880B8892B29BB29A4210B516D0013351
:106EC000B3F5807F28BF00230C489CB2C05C0C80C7
:106ED0000B490968C0B259B19A4238BF02F58072B5
:106EE000D31A1A2B04DC00230B7010BD4FF0FF30B7
:106EF00010BD00BF588BFF1FD689FF1F588AFF1F88
:106F0000D089FF1F094B1A88094B1B8892B29BB28C
:106F10009A4208D00133B3F5807F28BF0023054A89
:106F2000D05CC0B270474FF0FF307047588BFF1FE6
:106F3000D689FF1F588AFF1F0C4B1B685B0514D5B1
:106F40000B4BDA7802F0CB02DA7040225A74DA780E
:106F500042F03402DA70074B1A88074B92B21A805B
:106F6000064B1B680BB100221A7070473480044036
:106F700000A00640D689FF1F588BFF1FD089FF1F36
:106F800030B53E4B1A7912F0300F32D072B69A7D7E
:106F900002F0FF0022B9DA7940225A7462B628E082
:106FA00062B6374A3749138809889BB289B21446BA
:106FB000324AD5795A1CB2F5807F28BF00228A4216
:106FC000EDB202D0304B9D541346421E12F0FF002A
:106FD000EED19AB222802D4A126852B18B4236BF4E
:106FE000C1F58071C1EB03035B18272BC4BF0123DC
:106FF0001370224BD978C9B20A0620D51B791D0619
:107000001DD5234B234A1D781378EDB2DBB2104611
:10701000AB420CD0194A0133802B14791E4C28BF87
:107020000023E45CE4B2D471127D072AF0D9DBB20C
:107030000370124B1A79140644BF7C22DA700F4B8E
:107040009A7C500706D5154A10780130C0B21070EE
:1070500004229A74490610D5084B1A7952060CD5A9
:107060000F4A002111700F4A126802B111709A790B
:1070700002F0DF029A713C22DA7030BD00A00640B7
:10708000588BFF1FD689FF1F588AFF1FD089FF1F0B
:10709000608BFF1F5A8BFF1FD889FF1FE491FF1FD2
:1070A000D489FF1F5C8BFF1F1B4B1A6842F40062E0
:1070B0001A601A4A00231380194A1380194A137060
:1070C000194A1370194A1370194B40F247321A606B
:1070D000184BC0F344321A70C0F347125A7000F0D4
:1070E0001F000422022198729A70D9745A7588225E
:1070F0001A743C22DA709A7842F0A0029A709A7957
:1071000002F0DF029A710C4B40221A70A3F22B336B
:107110004FF400421A607047348004406C8DFF1FAA
:107120006A8BFF1F748DFF1F6E8DFF1F688BFF1F03
:1071300010B0044000B006402FE400E0134A9378FA
:1071400000F0030103F0EC030B43410748BF43F099
:107150001003937000F00F03042B0C4903D18B79BB
:1071600043F040038B715379C20603F0EF03074AE3
:1071700048BF43F0100353719379810603F0EF0386
:1071800048BF43F010039371704700BF00B0064042
:1071900008B5114B1B681B0500D408BD0F4B1A78AE
:1071A00002F0FF0312B101F0D1FDF7E70C4A4FF4F2
:1071B000004111600B4A0C49D37040F203120A607F
:1071C0004A600A4A13800A4A13800A4B1B680BB1B3
:1071D00001221A7008BD00BF34800440688BFF1F75
:1071E00084E100E000B006400CB004406C8DFF1F4D
:1071F0006A8BFF1F648BFF1F38B50446094B1B7851
:1072000003F0FF05002BF9D120460121FFF7CCFA4E
:1072100020462946FFF7A8FA034B53F83420034BC6
:107220001A6038BD688BFF1FF0CC0000708DFF1F07
:107230000D4A38B5146814F400624FF0000410D001
:1072400021280A4D0AD80A4A012152F830302B6011
:10725000FFF7AAFA2B681C70012038BD2C6020466D
:1072600038BD104638BD00BF34800440648BFF1F1A
:10727000F0CC00000B4B1B6813F4006310D01728F0
:10728000094B09D1094A40F2023111605A7B42F0A0
:1072900001025A73012070475A7B02F0FE025A73B2
:1072A000002070473480044000B0064008B004401D
:1072B000F8B51F4B1B681A05064638D51D4B9A7941
:1072C00042F020029A711C4B1B680BB101221A700C
:1072D0001A4B1C780134802C1F4628BF0024184DFF
:1072E0002B78A34218D1FFF717F840280FDC114A7A
:1072F00013791B06F3D52B7812490133802B28BF55
:107300000023C95CDBB2C9B2D1712B70E7E7FF285B
:10731000E5DD01F01BFDE2E70A4BF6B21E550A4B14
:1073200001221A70034BE4B2BC223C70DA70F8BD43
:107330003480044000B00640708DFF1F748DFF1F25
:107340006E8DFF1F6C8BFF1F688BFF1F294B1B6807
:107350001A052DE9F04707468A4649D5264B9A7902
:1073600042F020029A71254B1B680BB101221A7062
:107370003D4607EB0A039D4237D2DFF89080204E4E
:1073800098F8004096F800900134802C28BF002423
:107390005FFA89F9A1451DD1174BBC22DA70FEF7BF
:1073A000BBFF40280FDC144A13791B060FD5337836
:1073B00014490133802B28BF0023C95CDBB2C9B25A
:1073C000D171337003E0FF2801DD01F0BFFC337899
:1073D0004B45E4D00B4B15F8012B1A550A4B0122F3
:1073E000E4B21A7088F80040C3E7034BBC22DA709D
:1073F000BDE8F0873480044000B00640708DFF1F68
:107400006E8DFF1F6C8BFF1F688BFF1F748DFF1F1E
:1074100008B5034B1B7813B101F098FCF9E708BDE0
:10742000688BFF1F064A074B1B781078DBB2C0B28F
:1074300083422CBF7F3000F1FF30C01A704700BF7D
:107440006E8DFF1F748DFF1F054B1888054B1B8821
:1074500080B29BB2984238BF00F5C070C01A704726
:107460006C8DFF1F6A8BFF1F114B12491A880B8806
:1074700092B29BB29A4210B516D00133B3F5C07FD9
:1074800028BF00230C489CB2C05C0C800B490968E3
:10749000C0B259B19A4238BF02F5C072D31A1A2B42
:1074A00004DC00230B7010BD4FF0FF3010BD00BF97
:1074B0006C8DFF1F6A8BFF1FEC8BFF1F648BFF1F00
:1074C000094B1A88094B1B8892B29BB29A4208D08A
:1074D0000133B3F5C07F28BF0023054AD05CC0B29A
:1074E00070474FF0FF3070476C8DFF1F6A8BFF1F96
:1074F000EC8BFF1F0C4B1B681B0514D50B4BDA786C
:1075000002F0CB02DA7040225A74DA7842F0340288
:10751000DA70074B1A88074B92B21A80064B1B6829
:107520000BB100221A7070473480044000B006404E
:107530006A8BFF1F6C8DFF1F648BFF1F30B53E4BA6
:107540001A7912F0300F32D072B69A7D02F0FF0035
:1075500022B9DA7940225A7462B628E062B6374A14
:107560003749138809889BB289B21446324AD579C3
:107570005A1CB2F5C07F28BF00228A42EDB202D069
:10758000304B9D541346421E12F0FF00EED19AB2CA
:1075900022802D4A126852B18B4236BFC1F5C071AC
:1075A000C1EB03035B18272BC4BF01231370224BCD
:1075B000D978C9B20A0620D51B791D061DD5234BE3
:1075C000234A1D781378EDB2DBB21046AB420CD0E3
:1075D000194A0133802B14791E4C28BF0023E45C28
:1075E000E4B2D471127D072AF0D9DBB20370124BDA
:1075F0001A79140644BF7C22DA700F4B9A7C50072C
:1076000006D5154A10780130C0B2107004229A7461
:10761000490610D5084B1A7952060CD50F4A00219D
:1076200011700F4A126802B111709A7902F0DF02EC
:107630009A713C22DA7030BD00B006406C8DFF1F9D
:107640006A8BFF1FEC8BFF1F648BFF1F748DFF1F66
:107650006E8DFF1F6C8BFF1FD488FF1F688BFF1F71
:10766000708DFF1F174B1A6842F480521A60164A39
:1076700000231380154A1380154A1380154A13807E
:10768000154A1370154A40F2133111604FF45171CD
:107690005160134AC0F344311170C0F3471100F038
:1076A0001F0051709072937013742C23D3700D4B84
:1076B00040226FF44B711A700B444FF400321A6081
:1076C000704700BF348004408090FF1F7E8DFF1FF5
:1076D0008890FF1F8290FF1F7C8DFF1F08C0044011
:1076E00000C0064031E400E0134A937800F0030143
:1076F00003F0EC030B43410748BF43F010039370C2
:1077000000F00F03042B0C4903D18B7943F04003A5
:107710008B715379C20603F0EF03074A48BF43F069
:10772000100353719379810603F0EF0348BF43F0D0
:1077300010039371704700BF00C0064008B5114B9D
:107740001B68DB0400D408BD0F4B1A7802F0FF035E
:1077500012B101F0FBFAF7E70C4A4FF40031116067
:107760000B4A0C49D37040F203120A604A600A4A7D
:1077700013800A4A13800A4B1B680BB101221A704E
:1077800008BD00BF348004407C8DFF1F84E100E011
:1077900000C0064008C004408090FF1F7E8DFF1F80
:1077A000788DFF1F38B50446094B1B7803F0FF05A1
:1077B000002BF9D120460121FEF7F6FF204629468D
:1077C000FEF7D2FF034B53F83420034B1A6038BD49
:1077D0007C8DFF1FF0CC00008490FF1F0D4A38B550
:1077E000146814F480524FF0000410D021280A4D80
:1077F0000AD80A4A012152F830302B60FEF7D4FF34
:107800002B681C70012038BD2C60204638BD104606
:1078100038BD00BF34800440788DFF1FF0CC0000DD
:107820000B4B1B6813F4805310D00E28094B09D161
:10783000094A40F2023111605A7B42F001025A7348
:10784000012070475A7B02F0FE025A7300207047F5
:107850003480044000C0064004C00440F8B51F4B0B
:107860001B68DA04064638D51D4B1B680BB1012294
:107870001A701C4B1C88A4B20134B4F5C07F1F469B
:1078800028BF0024184D2B889BB2A3421AD1FEF7C3
:1078900043FD402811DC154A13791B06F2D52B88CD
:1078A00013499BB20133B3F5C07F28BF0023C95CE5
:1078B0009BB2C9B2D1712B80E4E7FF28E2DD01F071
:1078C00045FADFE70A4BF6B21E550A4B01221A7041
:1078D000064BA4B2AC223C80DA70F8BD3480044080
:1078E0008490FF1F8890FF1F8290FF1F00C00640FA
:1078F000808DFF1F7C8DFF1F38B504464518AC42B4
:1079000004D014F8010BFFF7A9FFF8E738BDFFFF1B
:1079100008B5034B1B7813B101F018FAF9E708BD5D
:107920007C8DFF1F064A074B1B8810889BB280B2D4
:1079300083422CBF00F27F1000F1FF30C01A704765
:107940008290FF1F8890FF1F054B1888054B1B88EE
:1079500080B29BB2984238BF00F5C070C01A704721
:107960008090FF1F7E8DFF1F114B12491A880B88D4
:1079700092B29BB29A4210B516D00133B3F5C07FD4
:1079800028BF00230C489CB2C05C0C800B490968DE
:10799000C0B259B19A4238BF02F5C072D31A1A2B3D
:1079A00004DC00230B7010BD4FF0FF3010BD00BF92
:1079B0008090FF1F7E8DFF1F008FFF1F788DFF1FA0
:1079C000094B1A88094B1B8892B29BB29A4208D085
:1079D0000133B3F5C07F28BF0023054AD05CC0B295
:1079E00070474FF0FF3070478090FF1F7E8DFF1F64
:1079F000008FFF1F054B1A88054B92B21A80054B6A
:107A00001B680BB100221A70704700BF7E8DFF1FEC
:107A10008090FF1F788DFF1F10B5314B1A799206A9
:107A200023D5304AD87913882F499BB2013309886E
:107A3000B3F5C07F28BF002389B28B42C0B203D008
:107A40002A49C85499B21180294A116869B1294A52
:107A5000128892B2934236BFC2F5C072C2EB0303E2
:107A60009B18272BC4BF01230B701D4AD178C9B2C4
:107A70000C0618D51379180615D51F4B1D481C8800
:107A80000388A4B29BB29C4202D16C23D3700AE05B
:107A90000133B3F5C07F28BF0023184CE45C9BB2D0
:107AA000E4B2D47103800E4B9A7C520706D5144A77
:107AB00010780130C0B2107004229A744B060ED5B3
:107AC000074B1A7912F0400F194608D00D4B0022CF
:107AD0001A700D4B1B6803B11A702C23CB7010BDAC
:107AE00000C006408090FF1F7E8DFF1F008FFF1F8C
:107AF000788DFF1F8290FF1F8890FF1F808DFF1FD2
:107B0000E591FF1F7C8DFF1F8490FF1F21282BD83C
:107B1000164B1B5CFF2B27D0154A02EBC00000213F
:107B200042681160134A106840F020001060124A49
:107B300001201160114998400860114841F8040C77
:107B4000104911604FF4A07101397FF4FDAF116845
:107B50008905FCD42022013A7FF4FDAF0A4A1BB20A
:107B600032F8130080B270470020704700CE00004A
:107B7000F0CC00003880044000500440085004401D
:107B80000000020380014A0000510440F0B50C4B94
:107B90000C4C1A7842F0020504EBC50682F0010293
:107BA000706009481A700678002E0CBF8827C82715
:107BB00086F0010647EA0141067044F83510F0BD31
:107BC000F490FF1F0080FF1F6C91FF1F431E032BCB
:107BD00010B510D872B6094A52F8230048B141686E
:107BE00042F82310064A018832F81340611A22F83D
:107BF000131062B610BD002010BD00BFE490FF1F3F
:107C0000E691FF1F013803280AD872B6054B53F8D6
:107C10002030002013B101305B68FBE762B670478B
:107C2000002070473891FF1F10B572B60123174A24
:107C30001A4412F8012C12071CD59900144A52F864
:107C400031402CB902EB431308305860114B09E066
:107C500041F0010152F8314064B902EBC103083030
:107C600058600D4B42F831300C4B1A78013A1A70BB
:107C700062B610BD0133052BD9D162B6074B002285
:107C80001A70BDE8104000F0A7BB00BF58CF00003D
:107C90000080FF1F88004000C80040006291FF1F65
:107CA000431E032B30B532D8194A400140F0100072
:107CB000104472B6174CE25C032A09D8DFE802F0E0
:107CC000160218050830022213E00830042210E0E2
:107CD0001148124A50F8234014B940F8231002E02A
:107CE00052F82300416042F823100FE0032200E025
:107CF0000522E25410F0080F01F108030A884360DE
:107D00000CBF8823C82343EA0243036062B630BD38
:107D10000080FF1FA090FF1F3891FF1F4891FF1F99
:107D20002DE9F84FAB4F3C78E4B214F0040F3D4618
:107D300019D0A94B1B78A3B1A84A117801F0FF0311
:107D400021B1013BDBB2137003B900BEA44A117824
:107D500001F0FF0329B1013BDBB213700BB900F056
:107D60004FFC04233B7004F0080303F0FF02002BD8
:107D700000F067829B4B9C4C1A78D2B215094FEAEF
:107D8000920840F0E48104EBC803596854F8383095
:107D9000C3F38303013B0C2B00F2D681DFE813F021
:107DA00095019501D401D401D401D401D401D401A9
:107DB000B001D401D401D4010D008C4D0A684B6888
:107DC0008B486B6001218B4B44F838302A60DFF818
:107DD0005082017092B240F2816000238242C8F862
:107DE00000302361A36117D8B2F5D06F80F01E81F7
:107DF000B2F5817F00F0CF8006D8802A00F0BA80EB
:107E0000822A00F0BB8031E140F202339A4200F056
:107E1000D180B2F5A06F1CE042F22100824200F056
:107E200051810ED8B2F5086F00F09E80B2F5106F48
:107E300040F01C81684B6C4EAA781A7006F18009DC
:107E40000AE042F221218A4200F0088142F2213305
:107E50009A4200F00F8109E1336A1B0603D5706A6C
:107E6000083800F0B9FA08364E45F5D10026B1467B
:107E7000DFF8B0A156F80A0028B1D0F804B000F03D
:107E8000ABFA5846F8E74AF806005B4BDFF898A1D2
:107E9000F05056F80A0028B1D0F804B000F09CFA6F
:107EA0005846F8E7554B4AF80600F050544B23F873
:107EB0001900544B19F80320023A032A08D8DFE8C6
:107EC00002F002040204002200E0012203F809206B
:107ED00009F10109B9F1040F06F10406C8D14A4BB2
:107EE00000221A7001269A46484A494B32443344CC
:107EF00012F8012C9B0012F0080F1A704FEA860945
:107F000025D000F04BFA38B104EB46130830586026
:107F1000404B44F8393006E09AF8003044F8390014
:107F200001338AF8003000F039FA49F0010338B122
:107F300004EBC302083050602E4A44F8332006E0B8
:107F400044F833009AF8003001338AF8003049F0E1
:107F50000202013649F003090023052E44F83230AD
:107F600044F83930C0D186E01B4B2B4C1B78237072
:107F70000B4683E0284C237063707EE0AA88042AB5
:107F800074D8254C920023706370244B9B5C9E0731
:107F900073D5217071E0AA8802F07F02042A65DCA3
:107FA0006B88002B62D191001C4A0A44117821F0A1
:107FB000020159E0AA8802F07F02042A56DC6B888D
:107FC000002B53D19100154A0A44117841F0020167
:107FD0004AE000BF802007406B91FF1FF590FF1F14
:107FE0006D91FF1F902007400080FF1F5891FF1FD9
:107FF0006C91FF1FC80040009090FF1F4891FF1F29
:10800000E691FF1FA090FF1F6291FF1F58CF000055
:1080100030C80110880040006391FF1FC020074056
:108020008C90FF1FE490FF1F3891FF1F6A88A9887A
:108030009F4B53F8084CA3F10C00BCB133F80C6C07
:10804000964209D133F80A6C8E4205D1120A032AEE
:108050000CBF2378038911E00C33EAE7954A1168D5
:10806000954A1160A978954A117004E0944B0F224B
:108070001A7027E000231C4600E00223EE88B3427A
:1080800038BF1E46402E34BF35464025204629467F
:10809000FFF77CFD761B2C4403D1402D12D13546D1
:1080A00003E0402E34BF3546402520462946FFF7E1
:1080B0006DFD761B2C4401D1402D03D1814AC8F8B7
:1080C000004016800122804B3DE0804B1A8842F22E
:1080D00021039A4210D100237D4AC85C9854013391
:1080E000072BF9D11368862B02D17A4B0F221A7015
:1080F00000200146FFF74AFD774B44F8383023E073
:10810000764E3568B5B1DFF8BC81B8F80090B9F1AA
:10811000400F34BF4C46402428462146FFF736FD29
:10812000C4EB09039BB2A8F800300BB9402C00D176
:108130002B193360654B1A88B2F5A06F04D1002269
:108140005A709A78664B1A7001225F4B6CE004EB10
:10815000C806013D736802F00802A3F10800EDB201
:1081600002F0FF01002A36D000F036F95D485E4B80
:1081700050F82520EAB1516840F8251002F10801B5
:108180007160595D03290BD8DFE801F0020406088D
:10819000032104E0022102E0052100E004215955F9
:1081A00016F0080F12880CBF8823C82343EA024345
:1081B00042E05A5D032A07D8DFE802F0404002049B
:1081C000002206E0012204E016F0080F0CBF022294
:1081D00003225A5532E054F83820120C23F8082CA8
:1081E00022B3DFF834E123F8061C43F8041C5EF8E0
:1081F00025303E4913B94EF8250002E051F82530EC
:1082000058603B4B41F8250033F815100A4423F819
:10821000152000F0C3F810B10830706006E0354B4F
:1082200044F838001A7801321A7007E02A4B324AB3
:1082300016F0080F08BF134644F8383008233B7087
:1082400070E5E0071FD520492B482C4C02230B700A
:108250002B4B1A702B4B186098602B48D8601A6112
:108260009A615C60164B0D2018702848FF2303703C
:108270002B700274264A1370264B9F221A7001231A
:108280000B70BDE8F88F210604D50D4B0D221A7036
:1082900080232B70A20705D51C4B1A78D2B21A7016
:1082A00002232B70E30644BF10232B70BDE8F88F28
:1082B00068CF0000CC89FF1FF891FF1F7C91FF1F42
:1082C000C02007406091FF1F942007405891FF1F76
:1082D000F091FF1FF590FF1FC80040008C90FF1F1A
:1082E000982007403891FF1FA090FF1F9090FF1F1C
:1082F000E691FF1F6291FF1F88004000A490FF1FBE
:10830000F490FF1F0080FF1FF890FF1F8820074098
:108310008C20074084200740E490FF1F08B500F040
:1083200053FD00221A4B0021D15098180832882A98
:108330004160F7D1174A106840F48020106002F5C0
:1083400028326832C3F307201070C3F307401B0EB6
:1083500010751376FF2302F81C3C02F8143C02F857
:108360008C3C012302F8083C82F8641002F8183CA7
:10837000094B70226FF450711A700B444FF4007265
:108380001A6003F1C04303F5C82310221A7008BD18
:108390000080FF1F3480044049E400E072B60C4ABC
:1083A0001168B1FA81F30B2B02D962B60020704735
:1083B0004FF00040D84021EA0001116062B6054943
:1083C00048225343C8180022CA504260704700BF79
:1083D0007087FF1F0084FF1F0C4B4822C31AB3FB9A
:1083E000F2F30B2B11D80A4A127822B1094A1278FB
:1083F0000AB1FFF719BC72B6074A4FF0004121FAE3
:1084000003F311681943116062B670470084FF1FBF
:108410006291FF1F6B91FF1F7087FF1F10B5104CFB
:1084200023686BB120684288531C0244147A028886
:10843000934212D3FFF7D0FF094B00221A600DE0E0
:10844000084B1B7813B94FF0FF3010BD0320FFF726
:10845000BDFB20600028E5D1F5E74380204610BD34
:108460007891FF1F6B91FF1F10B50B4C236813B160
:1084700023686BB902E0094B1B7813B94FF0FF304A
:1084800010BD0320FFF7A2FB20600028F0D1F5E724
:108490005A881344187A10BD7891FF1F6B91FF1F03
:1084A000044B9888044B1B681BB11A885B88D31A4D
:1084B00018447047E691FF1F7891FF1F2DE9F8439C
:1084C0002D4E012307460C463370002C4FD02B4D08
:1084D0002B68A9462BBB4AF2F928294B1B7803F0DD
:1084E000FF020BB9327015E00420FFF78BFB072861
:1084F00008D801233370FFF751FFC9F8000080B995
:108500001D4B1870B8F101081E4B01D01A782AB122
:1085100001221A704FF0FF30BDE8F88300F016FC1E
:10852000DBE72968174A488800231370C0F140022E
:10853000944238BF224600F1080C10448C44488015
:10854000A41A934204D0F85C0CF803000133F8E756
:108550001F444B883F2B06D940230B800420FFF794
:108560009FFB00232B60084B05221A70ADE7347087
:108570002046BDE8F88300BF6E91FF1F7091FF1F7A
:108580006B91FF1F7491FF1F6D91FF1F07B502AB29
:10859000012103F8010D1846FFF790FF03B05DF8C5
:1085A00004FBFFFF2DE9F041114B1B78F3B1114E95
:1085B000114B3468114D01271F7098464CB10027AC
:1085C00063882F70042023802146FFF769FB376002
:1085D00009E0FFF7E3FE014620B104202C70FFF70D
:1085E0005FFB00E02F70002388F80030BDE8F081C9
:1085F0006B91FF1F7091FF1F6E91FF1F6D91FF1F09
:1086000038B50E4B1B7803F0FF05ABB90C4C216855
:1086100031B14B880B800420FFF742FB256038BD49
:10862000FFF7BCFE014620B10420BDE83840FFF74B
:1086300037BB044B01221A7038BD00BF6E91FF1F7B
:108640007091FF1F6D91FF1F08B50368C9B21B68C9
:10865000984708BD08B50368C9B21B68984708BDAC
:1086600008B50368C9B21B68984708BD08B5036818
:10867000C9B21B68984708BD4B0803F1376000F585
:10868000D830B0FBF1F0FEF725BA10B54B0803F176
:10869000376000F5D8301446B0FBF1F0FEF71AFA57
:1086A0002046BDE81040FEF763BAFEF78BBA0846D5
:1086B000FEF7BCBA08B50846FEF7D4FA003018BF7A
:1086C000012008BD08B50846FEF7EEFA003018BFD5
:1086D000012008BDFEF7DABBFEF714BCFEF7E6BBCF
:1086E000FEF7B8BBFEF728BCFEF7BEBB08B50846D0
:1086F000FEF700FB012008BD08B50846FEF7FAFAB0
:10870000012008BD10B5084614461146FEF740FB8F
:10871000204610BD38B508460D4601F00AFC044657
:1087200021462846FEF734FB204638BD7047FFFF40
:10873000044B00221A714FF47A711A73024A99603D
:108740001A6070478091FF1F30CE000008B50368A3
:10875000C9B21B68984708BD08B50368C9B21B6851
:10876000984708BD08B50368C9B21B68984708BD9B
:1087700008B50368C9B21B68984708BD4B0803F1E8
:10878000376000F5D830B0FBF1F0FEF78DBC10B5C6
:108790004B0803F1376000F5D8301446B0FBF1F018
:1087A000FEF782FC2046BDE81040FEF7C7BCFEF78E
:1087B000EFBC0846FEF720BD08B50846FEF738FDB9
:1087C000003018BF012008BD08B50846FEF752FD6D
:1087D000003018BF012008BDFEF736BEFEF770BEA0
:1087E000FEF742BEFEF714BEFEF784BEFEF71ABEC9
:1087F00008B50846FEF75CFD012008BD08B508462F
:10880000FEF756FD012008BD10B508461446114676
:10881000FEF79CFD204610BD38B508460D4601F018
:1088200088FB044621462846FEF790FD204638BDC9
:108830007047FFFF044B00221A714FF47A711A73CC
:10884000024A99601A6070479091FF1F88CE00001D
:1088500008B50368C9B21B68984708BD08B5036826
:10886000C9B21B68984708BD08B50368C9B21B6840
:10887000984708BD08B50368C9B21B68984708BD8A
:108880004B0803F1B76000F55840B0FBF1F0FEF77C
:10889000E9BE10B54B0803F1B76000F55840144627
:1088A000B0FBF1F0FEF7DEFE2046BDE81040FEF71B
:1088B0001BBFFEF743BF0846FEF774BF08B5084666
:1088C000FEF78CFF003018BF012008BD08B5084630
:1088D000FEF7A6FF003018BF012008BDFFF734B82F
:1088E000FFF76EB8FFF740B8FFF712B8FFF782B88E
:1088F000FFF718B808B50846FEF7B0FF012008BD1D
:1089000008B50846FEF7AAFF012008BD10B50846C5
:1089100014461146FEF7F0FF204610BD38B5084654
:108920000D4601F006FB044621462846FEF7E4FF0B
:10893000204638BD7047FFFF044B00221A714FF4E8
:108940007A711A73024A99601A607047A091FF1FEA
:10895000E0CE000008B5034B01221A60024B1B68F1
:10896000984708BD0C710340B891FF1F08B5034B31
:1089700001221A60024B5B68984708BD1C710340D6
:10898000B891FF1F08B5034B01221A60024B9B6888
:10899000984708BD2C710340B891FF1F08B5034BE1
:1089A00001221A60024BDB68984708BD3C71034006
:1089B000B891FF1F054B1A6842F400021A60044B7D
:1089C00000221A60034B01221A7070473C80044059
:1089D00000700340B491FF1F064B01221A6003F59B
:1089E00088333C331A6822F400021A60024B0022DA
:1089F0001A70704700700340B491FF1FF0B54578BE
:108A0000134C144F2B011A194260134A9E188660AA
:108A1000066947F8256000259D501951032199509A
:108A20004378427B4433DBB2037303F1604303F5C5
:108A3000644301211A70027B53119B0003F16043D0
:108A400003F5614302F01F0201FA02F21A60F0BD61
:108A500000710340B891FF1F08710340F8B50C4B3B
:108A60001B7806460F460BB9FFF7A4FF0024094DFB
:108A7000625DE3B23AB9304673703946FFF7BEFF24
:108A800001202855F8BD0134042CF0D10020F8BD98
:108A9000B491FF1FB091FF1F8268002310B51360CF
:108AA000027B0121541102F01F0201FA02F208496F
:108AB00041F82420074A41785354D15C31B901333D
:108AC000042BFAD1BDE81040FFF786BF10BD00BFF0
:108AD00080E100E0B091FF1F037870B504460D46B9
:108AE00016461BB1FFF7D8FF0023237025612046EF
:108AF0003146FFF7B3FF10B10123237000E020706F
:108B0000207870BD037810B504460BB1FFF7C4FFA1
:108B10000023237010BD08B5F7F7A4FCF7F7D2FDCA
:108B200000F014F9FAE701F0D9B801F0DFB82DE947
:108B3000F04100258C688AB0074688462E4694B1DD
:108B40002B46404601A9212200F0E7F83B68202C83
:108B500034BF224620225B68384601A91544A41A76
:108B600098470644EBE730460AB0BDE8F081FFFFC6
:108B700007B5064B1B88ADF80430036801A95B6894
:108B80000222984703B05DF804FB00BF30CF00001D
:108B900008B503685B689847002008BD0EB403B5AC
:108BA00003AA52F8041B019201F0B4FA02B05DF876
:108BB00004EB03B0704770B505468AB022B903686C
:108BC000C9B21B6898472CE0012A08BF0A2221B9C4
:108BD00030228DF82520212413E02124B1FBF2F06E
:108BE00002FB1011C9B209290AAE94BF30313731E6
:108BF0002644C9B206F8241C014610B1013CE4B277
:108C0000ECE733B1013CE4B20AAB23442D2203F874
:108C1000242C2B6801A95B6828462144C4F1220258
:108C200098470AB070BD0029BABF49422D230023DE
:108C30000A22FFF7C0BFFFF733BCFFF7EFBBFFF718
:108C400013BCFFF7AFBC0846FFF7A0BC08461146AF
:108C5000FFF734BC7047FFFF044B00221A714FF43A
:108C60007A711A73024A99601A607047C891FF1F9F
:108C700040CF000010B50446006801F037F82046E8
:108C800010BD38B504460D460068013101F018F9F1
:108C900010B184E82100012038BD43688B4210B533
:108CA000044606D2FFF7EDFF20B1A3680BB9226896
:108CB0001370012010BDF8B504460F46154622B9C1
:108CC000036803B11A7000230BE01146FFF7E5FFBC
:108CD000064640B9206810B101F008F8266000236C
:108CE0006360A36004E0A5602068394601F019F9CB
:108CF0002046F8BD38B50023044603604360836016
:108D000003730D4639B1084601F013F929460246AE
:108D10002046FFF7D0FF204638BD38B50C469AB143
:108D200091B181688B4202D30023237038BDC91AE8
:108D3000551E8D4228BF0D4601682A46194420461B
:108D400001F016F90023635538BDFFFF10B50E4C36
:108D50002378BBB901232370FFF7A2FB08B1FFF70B
:108D600079FFFEF793F808B1FFF7E0FCFEF76CFB24
:108D700008B1FFF75DFDFEF7E7FD08B1FFF7DAFD8B
:108D80000023237010BD00BFD891FF1F10B5002332
:108D9000B0FBF2F402FB1400092894BF30303730E6
:108DA000C0B2C85420460CB10133F1E7CA18547060
:108DB00022469A4206DA885CCC5C8C54C854013254
:108DC000013BF6E7084610BD1FB572B6154B702281
:108DD0001A70154A412111700F2102F8011C8022DE
:108DE0001A701A781206FCD5104B186862B6104B30
:108DF000984298BF0A2301AC98BF584321460A22E3
:108E0000FFF7C4FF0023E15C0A4A29B102EB4300EB
:108E100001330A2B4180F6D101335B00137004B09B
:108E200010BD00BF000002400700024008000240E1
:108E30007F969800FC87FF1F81F0004102E000BF91
:108E400083F0004330B54FEA41044FEA430594EA0A
:108E5000050F08BF90EA020F1FBF54EA000C55EA45
:108E6000020C7FEA645C7FEA655C00F0E2804FEA16
:108E70005454D4EB5555B8BF6D420CDD2C4480EAF8
:108E8000020281EA030382EA000083EA010180EA28
:108E9000020281EA0303362D88BF30BD11F0004F76
:108EA0004FEA01314FF4801C4CEA113102D04042AC
:108EB00061EB410113F0004F4FEA03334CEA1333E7
:108EC00002D0524263EB430394EA050F00F0A780FF
:108ED000A4F10104D5F1200E0DDB02FA0EFC22FAFA
:108EE00005F2801841F1000103FA0EF2801843FAEE
:108EF00005F359410EE0A5F120050EF1200E012ADF
:108F000003FA0EFC28BF4CF0020C43FA05F3C0181C
:108F100051EBE37101F0004507D54FF0000EDCF195
:108F2000000C7EEB00006EEB0101B1F5801F1BD33E
:108F3000B1F5001F0CD349085FEA30004FEA3C0C42
:108F400004F101044FEA445212F5800F80F09A8038
:108F5000BCF1004F08BF5FEA500C50F1000041EB3C
:108F6000045141EA050130BD5FEA4C0C404141EB40
:108F7000010111F4801FA4F10104E9D191F0000F67
:108F800004BF01460020B1FA81F308BF2033A3F1EA
:108F90000B03B3F120020CDA0C3208DD02F1140CE1
:108FA000C2F10C0201FA0CF021FA02F10CE002F11C
:108FB0001402D8BFC2F1200C01FA02F120FA0CFC15
:108FC000DCBF41EA0C019040E41AA2BF01EB04515E
:108FD000294330BD6FEA04041F3C1CDA0C340EDC5C
:108FE00004F11404C4F1200220FA04F001FA02F39F
:108FF00040EA030021FA04F345EA030130BDC4F15D
:109000000C04C4F1200220FA02F001FA04F340EA51
:109010000300294630BD21FA04F0294630BD94F002
:10902000000F83F4801306BF81F480110134013DE9
:109030004EE77FEA645C18BF7FEA655C29D094EA5A
:10904000050F08BF90EA020F05D054EA000C04BFD8
:109050001946104630BD91EA030F1EBF00210020C3
:1090600030BD5FEA545C05D14000494128BF41F062
:10907000004130BD14F580043CBF01F5801130BDC6
:1090800001F0004545F0FE4141F470014FF0000051
:1090900030BD7FEA645C1ABF194610467FEA655C02
:1090A0001CBF0B46024650EA013406BF52EA0335A4
:1090B00091EA030F41F4002130BD00BF90F0000F92
:1090C00004BF0021704730B54FF4806404F13204CE
:1090D0004FF000054FF0000150E700BF90F0000F87
:1090E00004BF0021704730B54FF4806404F13204AE
:1090F00010F0004548BF40424FF000013EE700BF7E
:1091000042004FEAE2014FEA31014FEA02701FBF0D
:1091100012F07F4393F07F4F81F06051704792F0DF
:10912000000F14BF93F07F4F704730B54FF4607459
:1091300001F0004521F0004120E700BF50EA0102A4
:1091400008BF704730B54FF000050AE050EA010251
:1091500008BF704730B511F0004502D5404261EBC1
:1091600041014FF4806404F132045FEA915C3FF402
:10917000DCAE4FF003025FEADC0C18BF03325FEA9B
:10918000DC0C18BF033202EBDC02C2F1200300FA50
:1091900003FC20FA02F001FA03FE40EA0E0021FA75
:1091A00002F11444C1E600BF70B54FF0FF0C4CF45F
:1091B000E06C1CEA11541DBF1CEA135594EA0C0F15
:1091C00095EA0C0F00F0DEF82C4481EA030621EA50
:1091D0004C5123EA4C5350EA013518BF52EA03358B
:1091E00041F4801143F4801338D0A0FB02CE4FF03D
:1091F0000005E1FB02E506F00042E0FB03E54FF06D
:109200000006E1FB03569CF0000F18BF4EF0010E64
:10921000A4F1FF04B6F5007F64F5407404D25FEA60
:109220004E0E6D4146EB060642EAC62141EA555113
:109230004FEAC52040EA5E504FEACE2EB4F1FD0C55
:1092400088BFBCF5E06F1ED8BEF1004F08BF5FEAD3
:10925000500E50F1000041EB045170BD06F0004685
:1092600046EA010140EA020081EA0301B4EB5C0432
:10927000C2BFD4EB0C0541EA045170BD41F480112A
:109280004FF0000E013C00F3AB8014F1360FDEBF4F
:10929000002001F0004170BDC4F10004203C35DA2B
:1092A0000C341BDC04F11404C4F1200500FA05F3AE
:1092B00020FA04F001FA05F240EA020001F000424F
:1092C00021F0004110EBD37021FA04F642EB0601C5
:1092D0005EEA430E08BF20EAD37070BDC4F10C04EF
:1092E000C4F1200500FA04F320FA05F001FA04F2B3
:1092F00040EA020001F0004110EBD37041F100019F
:109300005EEA430E08BF20EAD37070BDC4F12005A9
:1093100000FA05F24EEA020E20FA04F301FA05F211
:1093200043EA020321FA04F001F0004121FA04F2B9
:1093300020EA020000EBD3705EEA430E08BF20EA89
:10934000D37070BD94F0000F0FD101F000464000C3
:1093500041EB010111F4801F08BF013CF7D041EA45
:10936000060195F0000F18BF704703F00046520049
:1093700043EB030313F4801F08BF013DF7D043EA1A
:109380000603704794EA0C0F0CEA135518BF95EAD0
:109390000C0F0CD050EA410618BF52EA4306D1D157
:1093A00081EA030101F000414FF0000070BD50EA76
:1093B000410606BF1046194652EA430619D094EA00
:1093C0000C0F02D150EA013613D195EA0C0F05D1EA
:1093D00052EA03361CBF104619460AD181EA03013E
:1093E00001F0004141F0FE4141F470014FF00000F6
:1093F00070BD41F0FE4141F4780170BD70B54FF091
:10940000FF0C4CF4E06C1CEA11541DBF1CEA135510
:1094100094EA0C0F95EA0C0F00F0A7F8A4EB0504F2
:1094200081EA030E52EA03354FEA013100F08880E9
:109430004FEA03334FF0805545EA131343EA1263B2
:109440004FEA022245EA111545EA10654FEA002667
:109450000EF000419D4208BF964244F1FD0404F520
:10946000407402D25B084FEA3202B61A65EB03057C
:109470005B084FEA32024FF480104FF4002CB6EB39
:10948000020E75EB030E22BFB61A754640EA0C00B9
:109490005B084FEA3202B6EB020E75EB030E22BFF9
:1094A000B61A754640EA5C005B084FEA3202B6EB3A
:1094B000020E75EB030E22BFB61A754640EA9C00F9
:1094C0005B084FEA3202B6EB020E75EB030E22BFC9
:1094D000B61A754640EADC0055EA060E18D04FEA87
:1094E000051545EA16754FEA06164FEAC30343EA27
:1094F00052734FEAC2025FEA1C1CC0D111F4801FF4
:109500000BD141EA00014FF000004FF0004CB6E7EC
:1095100011F4801F04BF01430020B4F1FD0C88BF8B
:10952000BCF5E06F3FF6AFAEB5EB030C04BFB6EB96
:10953000020C5FEA500C50F1000041EB045170BD89
:109540000EF0004E4EEA113114EB5C04C2BFD4EBB6
:109550000C0541EA045170BD41F480114FF0000E3A
:10956000013C90E645EA060E8DE60CEA135594EAB6
:109570000C0F08BF95EA0C0F3FF43BAF94EA0C0FB9
:109580000AD150EA01347FF434AF95EA0C0F7FF42E
:1095900025AF104619462CE795EA0C0F06D152EA82
:1095A00003353FF4FDAE1046194622E750EA410666
:1095B00018BF52EA43067FF4C5AE50EA41047FF477
:1095C0000DAF52EA43057FF4EBAE12E74A0011D229
:1095D00012F5001211D20DD56FF47873B3EB62520D
:1095E0000ED44FEAC12343F0004343EA505323FA19
:1095F00002F070474FF00000704750EA013002D18E
:109600004FF0FF3070474FF00000704780F000408F
:1096100002E000BF81F0004142001FBF5FEA41034A
:1096200092EA030F7FEA226C7FEA236C6AD04FEA4A
:109630001262D2EB1363C1BFD2184140484041408F
:10964000B8BF5B42192B88BF704710F0004F40F441
:10965000000020F07F4018BF404211F0004F41F45D
:10966000000121F07F4118BF494292EA030F3FD029
:10967000A2F1010241FA03FC10EB0C00C3F120033C
:1096800001FA03F100F0004302D5494260EB4000CB
:10969000B0F5000F13D3B0F1807F06D340084FEA36
:1096A000310102F10102FE2A51D2B1F1004F40EB2B
:1096B000C25008BF20F0010040EA03007047490093
:1096C00040EB000010F4000FA2F10102EDD1B0FA5E
:1096D00080FCACF1080CB2EB0C0200FA0CF0AABF53
:1096E00000EBC25052421843BCBFD04018437047F1
:1096F00092F0000F81F4000106BF80F400000132F7
:10970000013BB5E74FEA41037FEA226C18BF7FEACD
:10971000236C21D092EA030F04D092F0000F08BF0F
:109720000846704790EA010F1CBF0020704712F0F6
:109730007F4F04D1400028BF40F00040704712F135
:1097400000723CBF00F50000704700F0004343F09A
:10975000FE4040F4000070477FEA226216BF0846D0
:109760007FEA23630146420206BF5FEA412390EA93
:10977000010F40F4800070474FF0000304E000BF89
:1097800010F0004348BF40425FEA000C08BF70473A
:1097900043F0964301464FF000001CE050EA0102FE
:1097A00008BF70474FF000030AE000BF50EA010213
:1097B00008BF704711F0004302D5404261EB410100
:1097C0005FEA010C02BF84460146002043F0B64325
:1097D00008BFA3F18053A3F50003BCFA8CF2083A4A
:1097E000A3EBC25310DB01FA02FC634400FA02FC53
:1097F000C2F12002BCF1004F20FA02F243EB02005A
:1098000008BF20F00100704702F1200201FA02FCBB
:10981000C2F1200250EA4C0021FA02F243EB0200AE
:1098200008BF20EADC7070474FF0FF0C1CEAD052F2
:109830001EBF1CEAD15392EA0C0F93EA0C0F6FD0B3
:109840001A4480EA010C400218BF5FEA41211ED091
:109850004FF0006343EA501043EA5111A0FB01317D
:109860000CF00040B1F5000F3EBF490041EAD37152
:109870005B0040EA010062F17F02FD2A1DD8B3F1CE
:10988000004F40EBC25008BF20F00100704790F03D
:10989000000F0CF0004C08BF49024CEA502040EA8F
:1098A00051207F3AC2BFD2F1FF0340EAC250704755
:1098B00040F400004FF00003013A5DDC12F1190F93
:1098C000DCBF00F000407047C2F10002410021FA05
:1098D00002F1C2F1200200FA02FC5FEA310040F11D
:1098E000000053EA4C0308BF20EADC70704792F096
:1098F000000F00F0004C02BF400010F4000F013ACE
:10990000F9D040EA0C0093F0000F01F0004C02BFC8
:10991000490011F4000F013BF9D041EA0C018FE737
:109920000CEAD15392EA0C0F18BF93EA0C0F0AD03D
:1099300030F0004C18BF31F0004CD8D180EA010063
:1099400000F00040704790F0000F17BF90F0004FFC
:10995000084691F0000F91F0004F14D092EA0C0FDE
:1099600001D142020FD193EA0C0F03D14B0218BF71
:10997000084608D180EA010000F0004040F0FE40B7
:1099800040F40000704740F0FE4040F44000704753
:109990004FF0FF0C1CEAD0521EBF1CEAD15392EAD2
:1099A0000C0F93EA0C0F69D0A2EB030280EA010CC2
:1099B00049024FEA402037D04FF0805343EA11115B
:1099C00043EA10130CF000408B4238BF5B0042F1B9
:1099D0007D024FF4000C8B4224BF5B1A40EA0C005E
:1099E000B3EB510F24BFA3EB510340EA5C00B3EB90
:1099F000910F24BFA3EB910340EA9C00B3EBD10F7E
:109A000024BFA3EBD10340EADC001B0118BF5FEACF
:109A10001C1CE0D1FD2A3FF650AF8B4240EBC250F8
:109A200008BF20F0010070470CF0004C4CEA5020B9
:109A30007F32C2BFD2F1FF0340EAC250704740F408
:109A400000004FF00003013A37E792F0000F00F0FA
:109A5000004C02BF400010F4000F013AF9D040EA78
:109A60000C0093F0000F01F0004C02BF490011F40C
:109A7000000F013BF9D041EA0C0195E70CEAD15304
:109A800092EA0C0F08D142027FF47DAF93EA0C0FEB
:109A90007FF470AF084676E793EA0C0F04D14B02CF
:109AA0003FF44CAF08466EE730F0004C18BF31F081
:109AB000004CCAD130F000427FF45CAF31F000437B
:109AC0007FF43CAF5FE700BF4FF0FF3C06E000BF14
:109AD0004FF0010C02E000BF4FF0010C4DF804CD37
:109AE0004FEA40024FEA41037FEA226C18BF7FEA47
:109AF000236C11D001B052EA530C18BF90EA010F49
:109B000058BFB2EB030088BFC81738BF6FEAE170D7
:109B100018BF40F0010070477FEA226C02D15FEA73
:109B2000402C05D17FEA236CE4D15FEA412CE1D0DF
:109B30005DF8040B704700BF844608466146FFE7A6
:109B40000FB5FFF7C9FF002848BF10F1000F0FBD88
:109B50004DF808EDFFF7F4FF0CBF012000205DF881
:109B600008FB00BF4DF808EDFFF7EAFF34BF012006
:109B700000205DF808FB00BF4DF808EDFFF7E0FF9F
:109B800094BF012000205DF808FB00BF4DF808EDF0
:109B9000FFF7D2FF94BF012000205DF808FB00BF53
:109BA0004DF808EDFFF7C8FF34BF012000205DF835
:109BB00008FB00BF4FEA4002B2F1FE4F0FD34FF057
:109BC0009E03B3EB12620DD94FEA002343F000432A
:109BD00010F0004F23FA02F018BF404270474FF0D8
:109BE0000000704712F1610F01D1420205D110F05F
:109BF000004008BF6FF0004070474FF00000704712
:109C000042000ED2B2F1FE4F0BD34FF09E03B3EBE6
:109C1000126209D44FEA002343F0004323FA02F012
:109C200070474FF00000704712F1610F01D14202FE
:109C300002D14FF0FF3070474FF00000704700BF77
:109C400003460846194600F013B800210A2200F026
:109C500023BA00210A2200F01FBAFFFF0A46034977
:109C600003460868194600F084B800BF7488FF1FD7
:109C700070B5064C06460D4613462CB131462A46B1
:109C80000220AFF3008070BD204670BD00000000D0
:109C900070B50E4B0E4DED1AAD1000241E46AC42B1
:109CA00004D056F8242090470134F8E703F050FA26
:109CB000084D094BED1AAD1000241E46AC4204D0ED
:109CC00056F8242090470134F8E770BD5CD10000BD
:109CD0005CD1000074D100005CD10000024B014651
:109CE000186800F099B800BF7488FF1F024B014646
:109CF000186800F04DB800BF7488FF1F10B5C9B2D6
:109D000002449042034606D01C788C4200F10100C8
:109D1000F7D1184610BD002010BD10B500239342A6
:109D200003D0CC5CC4540133F9E710BD814270B557
:109D300001D300230EE08C18A042FAD285181346F6
:109D400013F1FF3305D3514266182944F65CCE5413
:109D5000F6E770BD934203D0CC5CC4540133F9E7FD
:109D600070BD02440346934202D003F8011BFAE798
:109D7000704738B502FB01F4214600F04DF8054666
:109D800018B100212246FFF7ECFF284638BDFFFF3F
:109D900030B500293CD051F8042C0B1F1D49002A76
:109DA000B8BF9B180A680C4612B95A600B6030BDE8
:109DB00093420DD219685818904203D15A58114451
:109DC000426819605A60236030BD994203D80A4640
:109DD00051680029F9D1146815199D420AD11B68F0
:109DE0002344D0188842136012D1086803441360DA
:109DF0004B680CE002D90C23036030BD18681C18B6
:109E00008C4203D10C684968204418605960536043
:109E100030BD00BFE091FF1F70B5CD1C25F00305DC
:109E200008350C2D38BF0C25002D06463FDB8D4232
:109E30003DD3214B1C6818462146A1B10B685B1B22
:109E40000ED40B2B03D90B60CC18CD501FE08C42E5
:109E500002D1626802601AE04B6863600C4616E04B
:109E60000C464968E9E7154C23681BB9304600F0F9
:109E700031F820602946304600F02CF8431C01469A
:109E800015D0C41C24F0030484420AD1256004F1D7
:109E90000B00231D20F00700C31A0BD05A42E250DA
:109EA00070BD3046611A00F015F80130EED10C2378
:109EB0003360002070BD00BFE091FF1FDC91FF1FE9
:109EC0000A46034903460868194600F001BA00BF74
:109ED0007488FF1F38B5064C0023054608462360EA
:109EE000FCF708FA431C02D1236803B12B6038BD8C
:109EF000FC91FF1FC9B2024610F8013B1BB18B4217
:109F0000F9D1104670470029FBD01846704710F869
:109F1000012B11F8013B012A28BF9A42F7D0D01A31
:109F20007047034611F8012B03F8012B002AF9D1E1
:109F30007047034613F8012B002AFBD1181A013889
:109F4000704770B592B10B4605461C7810F8016B4E
:109F5000B44201F1010101D1012A03D128781B7813
:109F6000C01A70BD013A002CEDD1F7E7104670BD64
:109F700010B5034632B111F8014B03F8014B013A19
:109F8000002CF7D11A44934203D0002103F8011B9F
:109F9000F9E710BD84463F482DE9F04FD0F8008026
:109FA0000E46344614F8015B08EB0500407800F0DB
:109FB000080000F0FF0708B12646F2E72D2D03D177
:109FC000B41C7578012703E02B2D04BF7578B41CF1
:109FD00033F010000DD1302D08D1207800F0DF00D3
:109FE000582851D165781023023402E0002B08BFB5
:109FF0000A23002F0CBF6FF0004A4FF0004ABAFB53
:10A00000F3F9002603FB19AA304608EB050B9BF871
:10A0100001B01BF0040F01D0303D0BE01BF0030B2F
:10A020001BD0BBF1010F14BF4FF0570B4FF0370B94
:10A03000CBEB05059D4210DAB6F1FF3F0AD048454B
:10A0400006D801D1554503DC03FB0050012601E091
:10A050004FF0FF3614F8015BD7E7731C0CD1002FCB
:10A060004FF022030CBF6FF000404FF00040CCF8DF
:10A0700000302AB9BDE8F08F07B1404242B106B1C5
:10A08000611E1160BDE8F08F002B08BF0823B0E708
:10A09000BDE8F08F7888FF1F30B51346044A0546A7
:10A0A0000C46106829462246BDE83040FFF772BFD3
:10A0B0007488FF1F2DE9F041ADF5047D1D464FF476
:10A0C00000730F4690460393044618B183690BB999
:10A0D00000F094F804AE00952046314603AA4346AA
:10A0E00000F05FF9054670B1204639462A46039BC9
:10A0F00000F01EF8B542039003D020462946FFF732
:10A1000047FE039801E04FF0FF300DF5047DBDE8F8
:10A11000F081FFFF30B51346044A05460C4610682F
:10A1200029462246BDE83040FFF7C4BF7488FF1FB0
:10A1300038B5074C054600202060084611461A46EF
:10A14000FEF726FD431C02D1236803B12B6038BD06
:10A15000FC91FF1FF8B5074600F1480494B1A568CB
:10A160006668013E0CD4AB89012B07D9B5F90E30D6
:10A17000013303D03846294600F0D6F96835F0E7B8
:10A180002468EBE7F8BDFFFF002310B50446036029
:10A190004360836081814366C2810361436183615F
:10A1A00019465C300822FFF7DCFD054B6362054B66
:10A1B000A362054BE362054B2462236310BD00BF1D
:10A1C0001DA300003FA3000077A300009BA3000095
:10A1D00070B54B1E68255D430E4605F17401FFF70F
:10A1E0001BFE044640B1002180E842000C30A06014
:10A1F00005F16802FFF7B5FD204670BD836910B513
:10A20000044633BB8364C3640365124B124A1B6864
:10A210008262984204BF0123836100F01FF86060EE
:10A22000204600F01BF8A060204600F017F804213B
:10A23000E06000226068FFF7A7FFA0680921012203
:10A24000FFF7A2FFE06812210222FFF79DFF012322
:10A25000A36110BDB4CF000055A10000F8B51B4BA1
:10A260001E68B369074613B93046FFF7C7FF483683
:10A27000B4687368013B04D4B4F90C5075B1683408
:10A28000F8E733682BB938460421FFF7A1FF3060A7
:10A2900008B13668ECE70C233B60F8BD4FF6FF735E
:10A2A000E3810123A38165662560A5606560256162
:10A2B0006561A56104F15C0029460822FFF751FDA4
:10A2C0006563A563A564E5642046F8BDB4CF0000CE
:10A2D000F8B5064614460D4621B91146BDE8F840CA
:10A2E000FFF79ABD1AB9FFF753FD2046F8BD00F0FD
:10A2F00057F9A0420ED230462146FFF78DFD0746A2
:10A3000050B129462246FFF708FD30462946FFF79F
:10A310003FFD01E02846F8BD3846F8BD10B50C46B3
:10A32000B1F90E1000F046F9002803DB636D034419
:10A33000636510BDA38923F48053A38110BD2DE96B
:10A34000F0411D468B89DB0507460C46164605D5B0
:10A35000B1F90E100022022300F010F9A389B4F91C
:10A360000E1023F48053A381384632462B46BDE8B5
:10A37000F041FFF7DDBE10B50C46B1F90E1000F04C
:10A38000FDF8431CA38903D123F48053A38110BD9E
:10A3900043F48053A381606510BDB1F90E1000F045
:10A3A0002FB830B515469BB0146829B124B14FF4CD
:10A3B000C162ADF80C2005E04FF422720024ADF824
:10A3C0000C202146002C0091049103DA8B230360BA
:10A3D000002012E04FF6FF72ADF80E2069461A46D3
:10A3E0001E9B0294059400F053F9031E4FF00000E9
:10A3F00003DB2B60009B187004981BB030BDFFFF7F
:10A4000038B5064C0023054608462360FBF77CFF61
:10A41000431C02D1236803B12B6038BDFC91FF1FA0
:10A420008A892DE9F041054610070C4657D44B6840
:10A43000002B02DC0B6C002B18DDE66AB6B102F4CF
:10A440008052002392B22F682B600AB1626D10E037
:10A45000216A28460123B047411C024609D12B68D6
:10A460003BB11D2B01D0162B46D12F600020BDE83B
:10A47000F081A3895B0705D56368D21A636B0BB1C2
:10A48000236CD21AE66A216A28460023B047461C8C
:10A49000A28905D12B681BB11D2B01D0162B19D118
:10A4A00000236360D1042369236004D5421C01D1D9
:10A4B0002B6803B96065616B2F600029D6D004F169
:10A4C0004403994202D02846FFF762FC00206063F3
:10A4D000BDE8F08142F04002A281BDE8F0810E6942
:10A4E000002EC3D00B680E60C6EB030893070CBFA9
:10A4F0004B6900238B6012E0A38943F04003A381E2
:10A500004FF0FF30BDE8F081A76A216A2846324645
:10A510004346B8470028EFDD0644C0EB0808B8F111
:10A52000000FF1DCA2E7FFFF38B50B6905460C46CA
:10A53000DBB118B183690BB9FFF760FE0C4B9C428D
:10A5400001D16C6808E00B4B9C4201D1AC6803E080
:10A55000094B9C4208BFEC68B4F90C302BB128467B
:10A560002146BDE83840FFF75BBF002038BD00BF83
:10A57000BCD00000DCD00000FCD0000038B5074C97
:10A58000054600202060084611461A46FBF7BFFE2C
:10A59000431C02D1236803B12B6038BDFC91FF1F1F
:10A5A00051F8040C002802DA04390B581844043816
:10A5B0007047FFFF38B5074C05460020206008466D
:10A5C00011461A46FBF79EFE431C02D1236803B1D5
:10A5D0002B6038BDFC91FF1F2DE9F0478D68AB4221
:10A5E00081460C4692461F4643D38B8913F4906FE5
:10A5F0003DD026680969C1EB06086669022206EBB0
:10A60000460696FBF2F608F101023A44964238BF3C
:10A6100016465B050FD53146FFF7FEFB054698B1A0
:10A6200021694246FFF779FBA38923F4906343F045
:10A630008003A38113E03246FFF74AFE054670B956
:10A6400048462169FFF7A4FB0C23C9F80030A38911
:10A6500043F04003A3814FF0FF30BDE8F087256150
:10A6600066614544C8EB06062560A6603D46AF42DC
:10A6700000D23D462A4620685146FFF757FBA368A3
:10A680005B1BA36023681D4425600020BDE8F087A4
:10A690002DE9F0439DB0074603938B891C060D46B8
:10A6A00016460CD50B6953B94021FFF7B5FB28605E
:10A6B000286110B90C233B60C8E040236B61002384
:10A6C000099320238DF8293030238DF82A30334622
:10A6D0001C4613F8012B1AB9B4EB06090FD002E09F
:10A6E000252AF5D1F8E73846294632464B46FFF78A
:10A6F00073FF013000F0A580099B4B440993237838
:10A70000002B00F09E8000234FF0FF32049307934C
:10A71000059206938DF853301A9304F101094C46C3
:10A720004D4E217830460522FFF7E8FA09F101097C
:10A73000049B28B1861B0120B04003430493EEE73D
:10A74000D90644BF20228DF853201A0744BF2B227C
:10A750008DF8532022782A2A02D0079B21460EE04A
:10A76000039A111D12680391002A01DB079204E08D
:10A77000524243F002030792049301340AE00C466C
:10A7800001312278303A092A03D80A2000FB03233A
:10A79000F5E7079323782E2B1AD163782A2B0AD159
:10A7A000039B1A1D1B680392002B04F10204B8BF1F
:10A7B0004FF0FF330BE0611C00230C46013122787F
:10A7C000303A092A03D80A2000FB0323F5E7059352
:10A7D000224E217830460322FFF790FA30B1861BD3
:10A7E000049B4020B04003430493013421781C486B
:10A7F0008DF828100622661CFFF780FA88B1194BE5
:10A8000033B9039B073323F007030833039314E0A2
:10A8100003AB0093384604A92A46134BAFF30080DC
:10A8200007E003AB0093384604A92A460E4B00F01C
:10A830008FF8B0F1FF3F804603D0099B4344099352
:10A8400045E7AB895B0601D4099801E04FF0FF3082
:10A850001DB0BDE8F08300BF1CD1000022D1000074
:10A8600026D1000000000000D9A500002DE9F84322
:10A8700015461F468A680B69DDF820809A42A8BFFA
:10A8800013462B6091F8432006460C460AB101336B
:10A890002B602368990602D52B6802332B6023684E
:10A8A00013F006091DD094F843302268003318BF16
:10A8B000012392061FD5E1185A1C302081F843006D
:10A8C000224494F8451082F84310023313E03046D6
:10A8D000394604F119020123C047013007D009F1BC
:10A8E0000109E2682B68D31A9945F0DBDBE74FF0EA
:10A8F000FF30BDE8F8833046394604F14302C047D3
:10A900000130F4D023682A68E16803F00603042BC1
:10A9100008BFC2EB01052369A2680CBF25EAE575F3
:10A9200000259A42C4BFC3EB0203ED184FF00009A3
:10A93000A9450ADA3046394604F11A020123C04714
:10A940000130D4D009F10109F2E70020BDE8F88315
:10A950002DE9FF470E7E0C9D6E2E80460C469146DB
:10A960009A4601F1430000F0A58011D8632E22D051
:10A9700009D8002E00F0AF80582E40F0BF8081F83B
:10A9800045607B4A4FE0642E1ED0692E1CD0B5E096
:10A99000732E00F0A48009D86F2E2BD0702E40F0BB
:10A9A000AD800B6843F020030B6038E0752E21D09A
:10A9B000782E34D0A2E02B681A1D1B682A6001F1A2
:10A9C000420781F842309DE022682B6812F0800F28
:10A9D00003D01A1D2A601D6805E05106F9D51A1D1D
:10A9E0002A60B3F90050002D39DA2D236D4284F826
:10A9F000433034E022682B6812F0800F03D01A1D18
:10AA00002A601D6804E05206F9D51A1D2A601D88C7
:10AA1000237E574A6F2B14BF0A2308231BE0782399
:10AA2000544A84F845302368296813F0800F01F1F7
:10AA300004062E6001D00D6802E05F06FBD50D888C
:10AA4000DE0744BF43F0200323601DB9236823F0D1
:10AA5000200323601023002184F8431001E0444ABE
:10AA60000A236668A660002E03DB216821F004013A
:10AA7000216005B96EB104F14201B5FBF3F603FBA9
:10AA800016550F46555D01F801593546002EF4D193
:10AA900000E00746082B0AD12368DD0707D5626866
:10AAA00023699A4203DC302307F8013C013FC01BB5
:10AAB00020612CE009682B68626911F0800F04D0D6
:10AAC000191D29601B681A6005E04906F8D5191D93
:10AAD00029601B681A8000232361074617E02B6852
:10AAE0001A1D2A601F683846FFF723FA6368206141
:10AAF000984288BF23612369636005E004F142073F
:10AB000084F8426001232361002384F84330CDF8A8
:10AB100000A04046214603AA4B46FFF7A7FE01309E
:10AB200002D14FF0FF301FE0404649463A462369C4
:10AB3000D0470130F5D023689B0705D4E068039B1C
:10AB40009842B8BF18460FE00025E268039BD31A6D
:10AB50009D42F3DA4046494604F119020123D047E9
:10AB60000130DED00135F0E704B0BDE8F08700BF6A
:10AB70002DD100003ED100004E4F54204150504C8A
:10AB80004945440045787465726E616C20566F6C5F
:10AB900074616765205B25735D0045787465726E2E
:10ABA000616C20566F6C74616765205B25642E258F
:10ABB000645D56000A427269646765206D6F646562
:10ABC00020666F7220496E7465726E616C204465F8
:10ABD0007669636520626F6F746C6F616465722063
:10ABE0006163636573733B2077616974696E672085
:10ABF000666F72207468652066697273742063687A
:10AC0000617261637465722E2E2E000A0A21212062
:10AC10005741524E494E4720212120496E73756697
:10AC200066696369656E742065787465726E616CBF
:10AC300020706F776572206170706C696564202187
:10AC40000A496E7465726E616C20736572766F73FB
:10AC500020617265206E6F7420706F776572656415
:10AC600020616E642077696C6C206E6F7420626561
:10AC700020726573706F6E736976652E0A4170700D
:10AC80006C7920706F77657220283E3D39562920F7
:10AC90007468726F75676820746865206D61696E8D
:10ACA00020636F6E6E6563746F7220706F72742EA6
:10ACB00000436F6E6E656374656420746F20455247
:10ACC0004F5320626F617264206174205B25645D64
:10ACD0006270732E20426F61726420465720766541
:10ACE0007273696F6E205B25645D2E20005B425499
:10ACF000204E4F542050524553454E545D00415410
:10AD00002B554152543D25642C302C30004F4B00C4
:10AD100041540D0A0041542B4E414D453F0D0A0050
:10AD200041542B505357443F0D0A005B4D41494E4F
:10AD30004252445F554E535550525445445D004174
:10AD4000542B4E414D453D25730041542B505357D4
:10AD5000443D2530346900636C735F43697263421C
:10AD600075666665725F3100636C73436972634236
:10AD700075666665725F320044756D70696E672036
:10AD800043697263756C6172206275666665725F95
:10AD9000006275666665725F2073697A6520697303
:10ADA0003A2025640A00252E32782000FFFFFFFF9D
:10ADB000000000000000000015630000891700007B
:10ADC000A1170000000000001801FFFFFFFFFFFFB8
:10ADD0000000000000000000C917000095170000E7
:10ADE000B5170000000000005B2254494D454F5547
:10ADF00054225D0A005B25645D205B25645D0A00CA
:10AE00005B22706172616D735F636F756E74202574
:10AE100064225D205B25645D0A00556E6B6E6F7762
:10AE20006E20737461746520696E2063616C6C625E
:10AE300061636B20696E20636C73436F6E736F6C1C
:10AE4000652121210A00496E69742064796E2070A1
:10AE500061636B6574005061727469616C6C792018
:10AE60006F70656E2068616E642066756E637469CC
:10AE70006F6E616C697479206973206E6F742079CC
:10AE8000657420696D706C656D656E7465642069AC
:10AE90006E2074686973206669726D7761726520CF
:10AEA00076657273696F6E2E20506C6561736520D4
:10AEB0007573652074686520636F6D6D616E6420C5
:10AEC000746F2073657420736572766F20706F7372
:10AED0006974696F6E7320696E64697669647561FF
:10AEE0006C6C792E0A00436C6F73652068616E6428
:10AEF0002066756E6374696F6E616C697479206920
:10AF000073206E6F742079657420696D706C656D47
:10AF1000656E74656420696E207468697320766557
:10AF20007273696F6E2E2055736520746865206397
:10AF30006F6D6D616E6420746F207365742073652E
:10AF400072766F20706F736974696F6E7320696EAB
:10AF5000646976696475616C6C792E0A005363616B
:10AF60006E6E696E6720696E2070726F67726573AE
:10AF7000732E2055736520636F6D6D616E6420279D
:10AF80007374617475732720746F206C69737420F7
:10AF900049447320666F756E642E00596573004EC8
:10AFA0006F005365656420526F626F74696373202C
:10AFB00045524F53204669726D776172650A00569B
:10AFC000657273696F6E2025642C20636F6D7069E4
:10AFD0006C6564206F6E204A616E203234203230FE
:10AFE00031392031393A30303A34350A002D0A48A7
:10AFF000415244574152453A0A2D0A00426F61724C
:10B0000064204D6F64656C203A20090925640A00AC
:10B01000485720436F6E66696775726174696F6E19
:10B020003A0925640A0053657269616C204E756D9A
:10B030006265723A0909252E3278252E3278252E3E
:10B0400032780A0050616C6D2049522053656E734E
:10B050006F723A0909004E6F7420696E7374616CE7
:10B060006C65640A005368617270204952207261F5
:10B0700074696F6D65747269632073656E736F7246
:10B080000A004D6963726F204952204469737461EC
:10B090006E63652053656E736F722028534D44298B
:10B0A0000A00436170616369746976652053656E57
:10B0B000736F72733A0900426C7565746F6F7468D0
:10B0C000206D6F64756C653A09496E7374616C6CC0
:10B0D00065640A00426C7565746F6F7468206D6FEB
:10B0E00064756C653A094E6F7420496E7374616CB7
:10B0F0006C65640A000A436F6E6669677572656401
:10B1000020566F6C74616765206F6E20496E742ED7
:10B110006275733A092564560A0043757272656E4A
:10B12000742073656E736F72207265736973746FC8
:10B13000722076616C75653A0925640A002D0A4310
:10B140004F4E46494755524154494F4E3A0A2D0AEF
:10B1500000426F61726420697320636F6E66696775
:10B160007572656420746F206F70657261746520FC
:10B1700077697468203132626974207265736F6C0C
:10B180007574696F6E2E0A00426F61726420697374
:10B1900020636F6E6669677572656420746F206FD7
:10B1A00070657261746520776974682031306269F6
:10B1B00074207265736F6C7574696F6E2E0A000A65
:10B1C00045787465726E616C2062757320636F6D73
:10B1D0006D756E69636174696F6E207365747469EF
:10B1E0006E67733A200A00426F6172642062757361
:10B1F000206465766963652049443A0925640A003C
:10B200004261756420726174652073657474696E3F
:10B21000673A092564203D202564204250530A00E6
:10B220005374617475732072657475726E206C65E9
:10B2300076656C3A0925640A005573696E67205477
:10B240005820456E61626C652070696E3A092573FD
:10B250000A000A496E7465726E616C206275732013
:10B26000636F6D6D756E69636174696F6E20736570
:10B270007474696E67733A20000A496E7465726E61
:10B28000616C20627573204261756420726174651F
:10B290002073657474696E673A09092564203D203E
:10B2A000256420425053000A496E7465726E616CC9
:10B2B000206275732070617273657220636F6E66B1
:10B2C00069677572656420666F723A0925730A0AA8
:10B2D00000426C7565746F6F746820434F4D4D204C
:10B2E000426175642073657474696E673A092564F8
:10B2F000203D202564204250530A00426C7565743D
:10B300006F6F746820646576696365206E616D6532
:10B310003A092573200A00426C7565746F6F746872
:10B320002064657669636520636F64653A0925303A
:10B330003464200A004E6F20426C7565746F6F7420
:10B3400068206D6F64756C652064657465637465F1
:10B35000642E0A0A004F6E004F66660053656564EE
:10B3600020526F626F746963732045524F532042BD
:10B370006F617264205374617475733A0A2D0A0008
:10B3800045585420566F6C746167653A0909004E40
:10B390004F54204150504C4945440A004552524FA9
:10B3A00052205B4F7574206F6620626F756E6473F8
:10B3B0002072656164696E672066726F6D20496EE8
:10B3C000742050535520666565646261636B3A2052
:10B3D0002564205D200A0025642E2564560A004954
:10B3E0004E542054656D703A0909256420646567E0
:10B3F000430A0046414E2053657474696E673A09EA
:10B400000925640A0046414E2050776D3A09092506
:10B41000640A0A0053454E532057416464756374AF
:10B42000696F6E3A0925640A0053454E532057460A
:10B430006C6578696F6E3A090925640A004F5054AB
:10B440004943414C2053454E532050616C6D3A099D
:10B4500000284F50544943414C2053454E532041FE
:10B460006D6269656E743A092564290A004341508A
:10B47000414349544956452053454E5320313A09DA
:10B4800025640A00434150414349544956452053DD
:10B49000454E5320323A0925640A000A494E544564
:10B4A000524E414C2042555320536572766F2049CD
:10B4B000447320286C6973743A2049442C205B45FE
:10B4C00052524F52204D41534B5D290A00253032D4
:10B4D00064095B4D41494E424F4152445D0A00258B
:10B4E000303264095B25645D0A000A504F525420D3
:10B4F00043555252454E542052454144494E4753BC
:10B500003A0A0023253032643A204F5645524C4FB8
:10B510004144204552524F52202825646D41290A4A
:10B520000023253032643A2025646D410A004254DC
:10B530006D6F64756C65207374617475733A092559
:10B54000730A000A434F4D4D204865616C746820B2
:10B5500053746174733A0A0055415254312028459E
:10B5600078742E436F6D6D29204275666665722072
:10B570004F76657272756E733A2025640A005541E4
:10B580005254322028496E742E436F6D6D2920422B
:10B590007566666572204F76657272756E733A20B5
:10B5A00025640A005541525433202842542E20432A
:10B5B0006F6D6D2920427566666572204F766572E3
:10B5C00072756E733A2025640A004C697374206F9B
:10B5D0006620616476616E63656420636F6D6D6182
:10B5E0006E64732E0A0A444953434C41494D4552F7
:10B5F0003A20546865736520636F6D6D616E647386
:10B600002061726520726573657276656420666F6D
:10B61000722074686520757365206F6620536565B8
:10B620006420526F626F7469637320746563686E1F
:10B630006963616C206167656E74732E0A496E637D
:10B640006F7272656374207573616765206D6179CF
:10B6500020636175736520696E6F706572617469CE
:10B660006F6E2C2064616D61676520616E64206D72
:10B67000617920766F696420796F757220776172C5
:10B6800072616E74792E0A55736520617420796F2A
:10B690007572206F776E207269736B2E0A0A0061D3
:10B6A00068700954686973206D6573736167652EEE
:10B6B0000A00696E697420656570726F6D0A0069B1
:10B6C0006E697420626F6172646D6F64656C205B7B
:10B6D0006D6F64656C5D0A00696E697420626F61EC
:10B6E00072646877636F6E666967205B636F6E660E
:10B6F0006967206D61736B5D0A00696E6974206310
:10B70000757272656E747265736973746F72205BA3
:10B710007265736973746F722076616C7565204F02
:10B72000686D735D0A00696E697420736E205B59E1
:10B73000595D205B4D4D5D205B434845434B535560
:10B740004D5D0A00696E69742073657269616C638E
:10B750006F6D6D205B6C6566747C72696768745D83
:10B760000A0A005573652027636F6E666967272094
:10B77000666F72207468652072656D61696E696EAE
:10B780006720636F6E66696775726174696F6E7347
:10B790002E2054797065202768656C702720666FAD
:10B7A0007220696E666F726D6174696F6E2E0A0A1F
:10B7B000004C697374206F6620617661696C616208
:10B7C0006C6520636F6D6D616E64732E20416C6CCF
:10B7D00020636F6D6D616E647320617265206361BB
:10B7E00073652073656E7369746976652E0A0A0045
:10B7F00068656C700954686973206D65737361675F
:10B80000652E0A0073746174757309446973706CF2
:10B8100061792063757272656E74207379737465D3
:10B820006D207374617475732E0A0061626F757494
:10B8300009446973706C617920696E7465726E6118
:10B840006C20696E666F726D6174696F6E2E0A008E
:10B850007363616E6275730952657363616E732001
:10B8600074686520696E7465726E616C20627573B0
:10B8700020666F722044796E616D6978656C206412
:10B880006576696365732E0A0073657466616E2060
:10B89000205B307E31305D095365747320746865B8
:10B8A00020756E69742066616E2073706565642012
:10B8B00028303D6F66663B2064656661756C742058
:10B8C00069732032292E0A00736574706F7320200B
:10B8D0005B6465766963652069645D205B706F7386
:10B8E0006974696F6E3A20302D25645D0953657463
:10B8F00020706F736974696F6E20666F7220737049
:10B9000065636966696564206465766963652E0AA6
:10B910000072657374617274205B7073757C616C06
:10B920006C5D095265737461727473206F6E6C790B
:10B930002074686520736572766F20505355206FB0
:10B9400072207468652066756C6C207379737465F9
:10B950006D2E0A00636F6E666967205B657874629E
:10B960006175647C65787469647C657874747865E5
:10B970006E61626C657C31326269746164636578A2
:10B98000706F7365647C6865617274626561747CF4
:10B99000696E74626175647C6274626175647C62F4
:10B9A000746E616D657C6274636F64657C627463E0
:10B9B0006F6D6D616E645D205B76616C75655D0AAF
:10B9C0000953797374656D207769646520636F6EC0
:10B9D00066696775726174696F6E206F7074696FE4
:10B9E0006E732E0A00636F6D6D6272696467652005
:10B9F0005B6269746D61736B5D09456E61626C6554
:10BA000020434F4D4D206272696467652E0A0942DA
:10BA100069746D61736B3A20313D5553422C20326D
:10BA20003D496E74204275732C20343D4578742056
:10BA30004275732C20383D42542C2031363D5553ED
:10BA40004220772F4454522052657365742E0A00A9
:10BA5000777262205B6465766963652069645D2046
:10BA60005B616464726573735D205B6279746520E9
:10BA700076616C75655D09577269746520627974C9
:10BA80006520746F206465766963652E0A0077729D
:10BA900077205B6465766963652069645D205B611E
:10BAA0006464726573735D205B696E742076616C8B
:10BAB00075655D09577269746520776F72642074CB
:10BAC0006F206465766963652E0A00726562205B8B
:10BAD0006465766963652069645D205B6164647296
:10BAE0006573735D095265616420627974652066CF
:10BAF000726F6D206465766963652E0A00726577E2
:10BB0000205B6465766963652069645D205B6164C0
:10BB100064726573735D095265616420776F726446
:10BB20002066726F6D206465766963652E0A0A006F
:10BB3000496E76616C696420636F6D6D616E642E11
:10BB400020436F6D6D616E64732061726520636167
:10BB500073652073656E7369746976652E0A54790E
:10BB60007065202768656C702720666F72206D6F86
:10BB7000726520696E666F726D6174696F6E2E0AF0
:10BB8000004944206E6F742070726573656E742076
:10BB9000696E2074686520696E7465726E616C20D0
:10BBA0006275732E205479706520277374617475E3
:10BBB000732720666F722061206C697374206F6632
:10BBC0002076616C6964204944732E0A00496E76C0
:10BBD000616C696420706F736974696F6E2E204D9B
:10BBE0006178696D756D206163636570746564204B
:10BBF000706F736974696F6E2069732034303935E2
:10BC00002E0A41637475616C206D6178696D756D84
:10BC100020646570656E6473206F6E206163747557
:10BC200061746F7220636F6E6669677572617469A3
:10BC30006F6E2E0A002564096D696C6C697365630B
:10BC40007309494409256409506F730925640D0A75
:10BC5000005B224E4F4944225D0A00707375004418
:10BC60006F6E6500616C6C00506172616D6574652A
:10BC70007220706173736564202822257322292045
:10BC8000697320696E76616C69642E204269746DF7
:10BC900061736B206D757374207365742074776F96
:10BCA00020696E74657266616365732E0A00446F65
:10BCB0006E652E005468697320626F617264206D36
:10BCC0006F64656C20646F6573206E6F742073758C
:10BCD00070706F72742066616E2073706565642089
:10BCE00073657474696E672E006578747478656E18
:10BCF00061626C6500796573006E6F003132626954
:10BD0000746164636578706F7365640068656172FF
:10BD10007462656174006F6E006F666600696E74B0
:10BD2000626175640062746261756400496E766177
:10BD30006C69642073657474696E672E2053657432
:10BD400074696E672073686F756C6420626520612A
:10BD5000204261756420706172616D657465722046
:10BD6000286578616D706C653A2031363D3131352A
:10BD700032303062707329005375636573732063CA
:10BD80006F6E6669677572696E67204254206D6FC9
:10BD900064756C652E0A004661696C656420636F8A
:10BDA0006E6669677572696E67204254206D6F64B4
:10BDB000756C652E0A005361766564207365747432
:10BDC000696E6720696E204D61696E20626F6172D5
:10BDD0006420656570726F6D2E0062746E616D65B2
:10BDE000005375636573730A004661696C0A0062EB
:10BDF00074636F646500496E76616C696420636F7B
:10BE000064652E20436F6465206D757374206265D0
:10BE100020612034206469676974206E756D6572D5
:10BE2000696320636F64652072616E67696E672065
:10BE300066726F6D203030303020746F20393939A0
:10BE4000392E0A00537563636573732E20425420A4
:10BE5000636F64652073657420746F2027257327D2
:10BE60002028616C776179732061203420646967D0
:10BE7000697420636F6465292E0A006274636F6DB4
:10BE80006D616E64005265706C793A0A25730A0020
:10BE9000656570726F6D00626F6172646D6F64656D
:10BEA0006C00626F6172646877636F6E66696700C9
:10BEB00063757272656E747265736973746F720004
:10BEC00073657269616C636F6D6D006C656674009B
:10BED000726967687400736E0068656C70006168F1
:10BEE00070007374617475730061626F75740073B0
:10BEF00063616E62757300636C6F7365007061726D
:10BF0000746F70656E00736574706F730072657323
:10BF10007461727400636F6D6D627269646765004D
:10BF200073657466616E0077726200777277007273
:10BF300065620072657700435249544943414C2081
:10BF40004552524F523A2074686973206669726D87
:10BF50007761726520636F6D70696C6174696F6E73
:10BF6000206973206E6F742064657369676E656401
:10BF700020666F72207468697320626F6172642E2C
:10BF8000202853455249414C315F4F4E455F574938
:10BF9000524520697320646566696E656420616E30
:10BFA000642073686F756C646E2774206265290065
:10BFB000435249544943414C204552524F523A2032
:10BFC00044696420796F7520696E7374616C6C20AC
:10BFD00074686520636F7272656374206669726D40
:10BFE000776172652076657273696F6E20666F7215
:10BFF00020796F757220626F617264206D6F646565
:10C000006C3F0A00466978656453697A6544786CC8
:10C01000436F6D6D616E6451756575650046697835
:10C02000656453697A6544786C436F6D6D616E64C5
:10C0300051756575655F6279746573617272617956
:10C0400000466978656453697A6544786C436F6D1E
:10C050006D616E6451756575655F62696469726C66
:10C06000697374000A44554D50204C4953540A00DA
:10C070004865616420616464722025702C205461DD
:10C08000696C20616464722025702C204974656D90
:10C0900020636F756E742025642C20707472206488
:10C0A00069666572656E63652025640A0041646493
:10C0B000722025702C20536572766F20494420250C
:10C0C000640A00636C735F4D61696E426F617264F4
:10C0D0005F696E6974000000010002000300040043
:10C0E00006000700080009000A000B000C000D0004
:10C0F0000E000F00100011001200130014001500B4
:10C100001600180019001A001B001C001D001E005C
:10C110001F0020002100220023002400250026000B
:10C120002700280029002A002B002C002D002E00BB
:10C130002F0030003100320033003400350036006B
:10C140003700380039003A003B003C003D003E001B
:10C150003F004000410042004300440044004500CD
:10C1600046004700480049004A004B004C004D0083
:10C170004E004F0050005100520053005400550033
:10C18000560057005800580059005A005B005C00E8
:10C190005D005E005F00600061006200630064009B
:10C1A0006500660066006700680069006A006B0051
:10C1B0006C006D006E006F00700071007200720004
:10C1C00073007400750076007700780079007A00BB
:10C1D0007B007C007C007D007E007F008000810071
:10C1E0008200830084008500860086008700880026
:10C1F00089008A008B008C008D008E008F008F00DC
:10C200009000910092009300940095009600970092
:10C210009700980099009A009B009C009D009E004A
:10C220009F009F00A000A100A200A300A400A50001
:10C23000A600A700A700A800A900AA00AB00AC00B8
:10C24000AD00AE00AF00AF00B000B100B200B3006F
:10C25000B400B500B600B600B700B800B900BA0027
:10C26000BB00BC00BD00BE00BE00BF00C000C100DE
:10C27000C200C300C400C500C500C600C700C80096
:10C28000C900CA00CB00CC00CD00CD00CE00CF004D
:10C29000D000D100D200D300D400D400D500D60005
:10C2A000D700D800D900DA00DB00DC00DC00DD00BC
:10C2B000DE00DF00E000E100E200E300E400E40073
:10C2C000E500E600E700E800E900EA00EB00EB002B
:10C2D000EC00ED00EE00EF00F000F100F200F300E2
:10C2E000F300F400F500F600F700F800F900FA009A
:10C2F000FB00FC00FC00FD00FE00FF00000101014E
:10C3000002010301040104010501060107010801FE
:10C3100009010A010B010C010D010D010E010F01B4
:10C320001001110112011301140115011601170169
:10C330001701180119011A011B011C011D011E0121
:10C340001F012001210121012201230124012501D6
:10C3500026012701280129012A012B012C012D0189
:10C360002D012E012F013001310132013301340141
:10C37000350136013701380139013A013B013B01F2
:10C380003C013D013E013F014001410142014301A9
:10C390004401450146014701480149014A014B0159
:10C3A0004C014D014E014F014F015001510152010D
:10C3B00053015401550156015701580159015A01C1
:10C3C0005B015C015D015E015F0160016101620171
:10C3D00063016401650166016701680169016A0121
:10C3E0006B016C016D016E016F01700171017201D1
:10C3F00073017401750176017701780179017A0181
:10C400007B017C017D017E017F0180018101820130
:10C410008301840185018601880189018A018B01DC
:10C420008C018D018E018F01900191019201930188
:10C43000940195019601970198019A019B019C0135
:10C440009D019E019F01A001A101A201A301A401E0
:10C45000A601A701A801A901AA01AB01AC01AD0188
:10C46000AE01B001B101B201B301B401B501B60131
:10C47000B701B901BA01BB01BC01BD01BE01C001D8
:10C48000C101C201C301C401C501C701C801C9017D
:10C49000CA01CB01CC01CE01CF01D001D101D20123
:10C4A000D401D501D601D701D801DA01DB01DC01C5
:10C4B000DD01DF01E001E101E201E401E501E60166
:10C4C000E701E901EA01EB01EC01EE01EF01F00106
:10C4D000F201F301F401F501F701F801F901FB01A3
:10C4E000FC01FD01FF01000201020302040205023A
:10C4F0000702080209020B020C020D020F021002D1
:10C500001202130214021602170219021A021B0267
:10C510001D021E02200221022302240226022702FB
:10C5200028022A022B022D022E023002310233028F
:10C5300034023602370239023A023C023E023F021E
:10C540004102420244024502470249024A024C02A9
:10C550004D024F0251025202540256025702590232
:10C560005B025C025E0260026102630265026602B7
:10C5700068026A026C026D026F0271027302740239
:10C58000760278027A027C027E027F0281028302B6
:10C590008502870289028B028D028E02900292022E
:10C5A0009402960298029A029C029E02A002A202A3
:10C5B000A402A602A802AB02AD02AF02B102B3020E
:10C5C000B502B702B902BC02BE02C002C202C40276
:10C5D000C702C902CB02CE02D002D202D502D702D4
:10C5E000D902DC02DE02E102E302E502E802EA022D
:10C5F000ED02F002F202F502F702FA02FC02FF027B
:10C600000203050307030A030D03100312031503B6
:10C6100018031B031E032103240327032A032D03EE
:10C6200030033303360339033D034003430346031A
:10C630004A034D035003540357035B035E03620335
:10C64000650369036D037103740378037C0380033E
:10C65000840388038C039003940398039D03A10330
:10C66000A503AA03AE03B303B803BC03C103C60307
:10C67000CB03D003D503DA03DF03E503EA03EF03BB
:10C68000F503FB03000406040C04120419041F0440
:10C6900025042C0433043A04400448044F0456048F
:10C6A0005E0466046E0476047E0487049004990494
:10C6B000A204AC04B604C004CA04D504E004EC042B
:10C6C000F804040511051E052C053A054905590510
:10C6D00069057A058C059F05B305C805DE05FFFFD2
:10C6E0000000000000000000F94800009141000037
:10C6F000C14100000000000044796E312070726F6B
:10C70000746F636F6C206465766963657300736C26
:10C710006176657061727365723A696E74206465E2
:10C72000766963657320646174610069735F726523
:10C730006164696E675F706172616D657465723A9C
:10C7400020726561642073746172743D25303258C3
:10C750003B207265616420656E643D253032583B34
:10C7600020706172616D5F6E616D65202530325899
:10C770000A00526573756C74206F6620746573745B
:10C780002072656164696E6720706172616D2069F5
:10C79000733A2025640A004552524F523A2052659E
:10C7A000717565737420746F206D6F64696679208C
:10C7B00061205245414420706172616D65746572FB
:10C7C00020627974652062757420746865207265D2
:10C7D000706C7920697320736D616C6C6572207464
:10C7E00068616E2074686520696E6465782077687A
:10C7F00065726520746865206E65772076616C755A
:10C800006520697320746F20626520696E7365729C
:10C810007465642100FFFFFF0000000000000000BD
:10C82000D14C000089490000B1490000C349000013
:10C83000114A00005D4A0000A54A0000554E000064
:10C8400025500000454B0000F54A0000A94B0000B0
:10C85000854900007D490000000000000000000044
:10C8600015630000FD510000255200001563000013
:10C8700015630000156300001563000015630000D8
:10C8800015630000156300001563000015630000C8
:10C8900015630000156300004D616C6C6F632066CA
:10C8A00061696C656420666F722025730A004944D3
:10C8B00025303264200057524954452000575249D0
:10C8C00054455F4E4F5F524554200052454144202D
:10C8D0000050494E472000494E535452204953209E
:10C8E0004E4F522052454144204E4F5220575249FC
:10C8F00054450A00205061636B65743A200030781B
:10C90000464620307846462049443D307800204C49
:10C91000454E3D30780020494E5354523D3078000A
:10C92000204552524F523D30780020504152414DE7
:10C93000533D002043484B3D307800205354415232
:10C94000543D25735B3078253032585D2056414C7C
:10C950005545533D003078464620307846462030D5
:10C960007846442030783030203078004D6F646550
:10C970006C204E756D626572284C29004D6F6465A0
:10C980006C204E756D626572284829005665727379
:10C99000696F6E206F66204669726D7761726500FF
:10C9A00049440042617564205261746500526574A7
:10C9B00075726E2044656C61792054696D65004321
:10C9C000435720416E676C65204C696D6974284C33
:10C9D000290043435720416E676C65204C696D699F
:10C9E000742848290074686520486967686573740D
:10C9F000204C696D69742054656D70657261747541
:10CA0000726500746865204C6F77657374204C699B
:10CA10006D697420566F6C74616765007468652079
:10CA200048696768657374204C696D697420566F36
:10CA30006C74616765004D617820546F7271756523
:10CA4000284C29004D617820546F72717565284813
:10CA500029005374617475732052657475726E2069
:10CA60004C6576656C00416C61726D204C454400EC
:10CA7000416C61726D2053687574646F776E004D00
:10CA8000756C7469205475726E204F666673657498
:10CA9000284C29004D756C7469205475726E204FB6
:10CAA0006666736574284829005265736F6C7574E7
:10CAB000696F6E204469766964657200546F7271A3
:10CAC000756520456E61626C650044204761696E42
:10CAD0000049204761696E0050204761696E004738
:10CAE0006F616C20506F736974696F6E284C2900F8
:10CAF000476F616C20506F736974696F6E284829A5
:10CB0000004D6F76696E67205370656564284C2907
:10CB1000004D6F76696E67205370656564284829FB
:10CB200000546F72717565204C696D6974284C29C9
:10CB300000546F72717565204C696D6974284829BD
:10CB40000050726573656E7420506F736974696FFD
:10CB50006E284C290050726573656E7420506F7397
:10CB60006974696F6E2848290050726573656E7428
:10CB7000205370656564284C290050726573656E9A
:10CB80007420537065656428482900507265736588
:10CB90006E74204C6F6164284C2900507265736577
:10CBA0006E74204C6F61642848290050726573656B
:10CBB0006E7420566F6C74616765005072657365A2
:10CBC0006E742054656D7065726174757265005283
:10CBD000656769737465726564004D6F76696E6729
:10CBE000004C6F636B0050756E6368284C290050D1
:10CBF000756E636828482900454550524F4D20778F
:10CC0000726974652064656E696564206279206963
:10CC10006E7465726E616C2070726F746563746996
:10CC20006F6E2E204E72206F662077726974657366
:10CC300020617474656D7074656420696E20746819
:10CC400069732073657373696F6E3A200041747461
:10CC5000656D7074696E6720746F20777269746592
:10CC6000206120424954206F6E2061206269746DFA
:10CC70006170206275742069742773206F75742049
:10CC80006F662072616E67653B2074686520616C19
:10CC90006C6F7765642072616E6765206973203000
:10CCA0007E372E00090AFFFFFFFFFFFFFFFFFFFF98
:10CCB000FFFFFF0D00060807FFFF0E0FFF0CFFFF31
:10CCC000FFFFFFFF0B05050E08090D0C06070F04FB
:10CCD000001303931A9217C585848687C4FF6FF0EB
:10CCE0007F030370037813F0800FFBD07047FFFFC2
:10CCF0004008FE4340A004404408FE4344A00440D2
:10CD00000018FE4300C004403000FE433090044051
:10CD10003400FE43349004401C18FE431CC0044001
:10CD20001018FE4310C004400818FE4308C0044019
:10CD30000C18FE430CC004400C10FE430CB0044021
:10CD40001010FE4310B004401810FE4318B0044009
:10CD50001C10FE431CB004401410FE4314B00440E9
:10CD60000418FE4304C004400010FE4300B0044019
:10CD70000008FE4300A004400408FE4304A0044051
:10CD80000C08FE430CA004400808FE4308A0044021
:10CD90001418FE4314C004401818FE4318C0044081
:10CDA0000410FE4304B004400810FE4308B00440E1
:10CDB0001400FE43149004404C08FE434CA0044071
:10CDC0000420FE4304D004402410FE4324B0044059
:10CDD0002010FE4320B004402810FE4328B0044039
:10CDE0002C10FE432CB004400020FE4300D0044031
:10CDF0004808FE4348A004401000FE431090044041
:10CE0000090AFFFFFFFFFFFFFFFFFFFFFFFFFF0D0F
:10CE100000060807FFFF0E0FFF0CFFFFFFFFFFFFDD
:10CE20000B05FFFFFFFFFFFF0000000000000000F8
:10CE3000ED86000005870000D5860000DD86000035
:10CE4000D9860000E1860000798600008B8600000C
:10CE5000AB860000AF860000B5860000C5860000E6
:10CE6000E5860000E986000049860000558600003E
:10CE7000618600006D86000015870000F9860000BD
:10CE80000000000000000000F18700000988000099
:10CE9000D9870000E1870000DD870000E5870000FA
:10CEA0007D8700008F870000AF870000B3870000F8
:10CEB000B9870000C9870000E9870000ED870000FE
:10CEC0004D870000598700006587000071870000CA
:10CED00019880000FD87000000000000000000002D
:10CEE000F58800000D890000DD880000E58800005D
:10CEF000E1880000E9880000818800009388000034
:10CF0000B3880000B7880000BD880000CD8800000D
:10CF1000ED880000F1880000518800005D88000065
:10CF200069880000758800001D89000001890000E3
:10CF30000D0AFFFFFFFFFFFF0000000000000000E0
:10CF4000478C00004D8C0000378C00003B8C0000AB
:10CF50003F8C0000438C00000015191500010000F3
:10CF60007487FF1F12000000000200009E87FF1F51
:10CF70004300000000030000F887FF1F00000000CE
:10CF8000010309048687FF1F000000000203090453
:10CF9000E287FF1F0000000003030904FC87FF1F56
:10CFA0000000000000000000000000000000000081
:10CFB0004300FFFF1488FF1F002020202020202096
:10CFC0002020282828282820202020202020202039
:10CFD0002020202020202020208810101010101049
:10CFE0001010101010101010100404040404040495
:10CFF000040404101010101010104141414141412F
:10D000000101010101010101010101010101010110
:10D010000101010110101010101042424242424220
:10D0200002020202020202020202020202020202E0
:10D030000202020210101010200000000000000088
:10D0400000000000000000000000000000000000E0
:10D0500000000000000000000000000000000000D0
:10D0600000000000000000000000000000000000C0
:10D0700000000000000000000000000000000000B0
:10D0800000000000000000000000000000000000A0
:10D090000000000000000000000000000000000090
:10D0A0000000000000000000000000000000000080
:10D0B000000000000000000000FFFFFF0000000073
:10D0C0000000000000000000000000000000000060
:10D0D0000000000000000000000000000000000050
:10D0E0000000000000000000000000000000000040
:10D0F0000000000000000000000000000000000030
:10D10000000000000000000000000000000000001F
:10D11000000000000000000000000000232D302B64
:10D120002000686C4C006566674546470030313228
:10D13000333435363738394142434445460030317F
:10D14000323334353637383961626364656600FFDF
:10D15000F8B500BFF8BC08BC9E4670473504000017
:10D160007D590000318700003588000039890000B2
:04D17000598C0000D6
:10D1740000000000010A04000092FF1F08000000E4
:10D18400FFFFFFFF1201000202000040C0168304EB
:10D1940000010102030118035400650065006E00DC
:10D1A400730079006400750069006E006F00090265
:10D1B4004300020100C03209040000010202010020
:10D1C400052400100105240101010424020605249C
:10D1D4000600010705820310004009040100020A49
:10D1E4000000000705030240000007058402400018
:10D1F4000000160355005300420020005300650050
:10D204007200690061006C00040309040C0300004F
:10D21400000000000000000000000000000000000A
:10D224000000000000000000BCD00000DCD00000C2
:10D23400FCD000000000000000000000000000001E
:10D2440000000000B0CF000000000000000000005B
:10D2540000000000000000000000000000000000CA
:10D2640000000000000000000000000000000000BA
:10D2740000000000000000000000000000000000AA
:0CD28400000000001488FF1FB8CF00005D
:00000001FF
